:020000040800F2
:100000000000012055400008E9270008EB27000800
:10001000ED270008EF270008F12700080000000086
:10002000000000000000000000000000F3270008AE
:10003000F527000800000000F7270008F92700084E
:10004000A5400008A5400008FD270008A5400008BD
:10005000A5400008A5400008A5400008A5400008EC
:10006000A540000821280008A5400008A540000878
:10007000A5400008A5400008092800081528000828
:10008000A5400008A5400008A5400008A5400008BC
:1000900000000000A5400008A5400008A540000899
:1000A000A5400008A5400008A5400008A54000089C
:1000B000A5400008A5400008A5400008A54000088C
:1000C000A5400008A5400008A5400008A54000087C
:1000D000A5400008A5400008A5400008A54000086C
:1000E000A5400008A540000829280008A5400008F0
:1000F000A54000080000000000000000A540000826
:10010000A5400008A540000835280008A5400008C3
:10011000A5400008A5400008A5400008A54000082B
:10012000A5400008A5400008A5400008A54000081B
:08013000A5400008A5400008ED
:1001380010B5054C237833B9044B13B10448AFF319
:1001480000800123237010BDBC08002000000000BF
:10015800183A010808B5034B1BB103490348AFF32C
:10016800008008BD00000000C0080020183A0108FF
:1001780014214160704714207047406A704700009E
:10018800790100087F01000883010008990100082F
:1001980010B5044604F1100000F05CFCC4F8F80047
:1001A8000148C4F87C0110BD88010008F8B5E6B024
:1001B80004460D4616461F460A4906A800F0CAFE20
:1001C80070996F9A05910492009733466E996D9ACB
:1001D800039102922A466C990191214600F060F839
:1001E80067B0F0BD94010008F8B5E6B004460D46C6
:1001F80016461F46094906A800F0ACFE6F996E9A8C
:100208000491039200976D996C9A0291019233467A
:100218002A46214600F087F867B0F0BD940100082F
:1002280038B500281CBF01680029184A23D1184B8B
:100238001C684FF6F0710C404CF24025AC421FBFD1
:100248001B6819404CF27024A14212D1114D296843
:1002580079B911490B68C3F30B03B3F58A6F1FBF54
:100268000968C1F30B0140F28343994204BF01219D
:10027800117028B905E0094B994204BF012111709A
:100288004068BDE8324001F099BE00BFD8080020A0
:1002980000ED00E0002004E00010005C000037489A
:1002A8002DE9F04104460D46216816464A681F4666
:1002B80090478046B8F5403F2ED122680A99936846
:1002C800204698478046B8F5403F25D12368089ACC
:1002D8000799D3F80CC02046E0478046B8F5403F60
:1002E8001AD12368069A39461F692046B8478046BE
:1002F800B8F5403F10D1236829465D69324620464B
:10030800A8478046B8F5403F06D123680B9A09995B
:100318009D692046A847804621680A68204690477C
:100328004046BDE8F0812DE9F04104460D462168BC
:1003380016464A681F4690478046B8F5403F2ED17A
:1003480022680A999368204698478046B8F5403F46
:1003580025D12368089A0799D3F80CC02046E047AE
:100368008046B8F5403F1AD12368069A39461F6976
:100378002046B8478046B8F5403F10D12368294643
:100388005D6932462046A8478046B8F5403F06D109
:1003980023680999DD6900222046A847804621681C
:1003A8000A68204690474046BDE8F0814FF4403047
:1003B80070470000F0B50C4685B0114600281A4673
:1003C8001CBF0568002D0B4B11D082B104B971B95F
:1003D8000D9860B10F9E0E9F0A9B0290049603979A
:1003E8000B980C9E009001962046A8470346184695
:1003F80005B0F0BD020003002DE9F04F0646D0B06D
:100408000868F56DD6F860E0726EB76EF36E00BAE4
:1004180000906C46486800BA60600DF14008886832
:1004280000BAA060C86800BAE060086900BA206134
:10043800486900BA6061886900BAA061C86900BAF1
:10044800E061086A00BA2062486A00BA6062886A95
:1004580000BAA062C86A00BAE062086B00BA2063FA
:10046800486B00BA6063886B00BAA063C86B00BAB7
:10047800E063402058F80C1C58F820CC58F838ACE9
:100488008CEA010158F840CC8AEA01018CEA01099A
:100498004FEAF979401E48F8049BEBD187EA02003D
:1004A80000EA0E00784010EBF5610098DFF824C4EC
:1004B80041186144C81882EABE032B404FEAF06134
:1004C80053405918636859186144CF194FEAB50366
:1004D80083EABE01014081EABE0111EBF765A1681C
:1004E8004D196544A91883EAB0023A404FEAF1650C
:1004F8005A405519E26855194FEAB70282EAB0071F
:1005080065440F4005EBBE0E97EAB00717EBFE6592
:1005180027697D194FEAB10782EA0701654401EAB4
:100528000E01EB18514011EBF36561694D194FEA63
:10053800BE0187EA010E65440EEA030E15EBB00012
:100548008EEA070E0EEBF065D4F818E075446544A2
:10055800AA1881EAB30505404FEAF26E4D40AE4451
:10056800E569AE44E64477444FEAB00080EAB30E4A
:100578000EEA020E8EEAB30E0EEBF765D4F820E011
:1005880075446544691880EAB2053D404FEAF16E4A
:100598004540AE44656AAE44E6440EEBB3034FEA09
:1005A800B70787EAB20E0EEA010E8EEAB20E0EEB1C
:1005B800F365D4F828E075446544281887EAB1053E
:1005C8001D404FEAF06E7D40AE44E56AAE44E64415
:1005D8000EEBB2024FEAB30383EAB10E0EEA000E45
:1005E8008EEAB10E0EEBF265D4F830E0754465443E
:1005F800EF1983EAB00515404FEAF76E5D40AE4447
:10060800656BAE44E6440EEBB1014FEAB20282EAF2
:10061800B00E0EEA070E8EEAB00E0EEBF165D4F8B6
:1006280038E075446544EB1882EAB7050D404FEA97
:10063800F36E5540AE44E56BAE44E6440EEBB000B5
:100648004FEAB10181EAB70E0EEA030E8EEAB70E41
:100658000EEBF065D4F840E07544654481EAB30ECA
:10066800AA180EEA000E4FEAF2658EEA010E7544EA
:10067800DDF844E04FEAB000754480EAB30E654403
:100688000EEA020E15EBB7078EEAB30E0EEBF7650E
:10069800DDF848E04FEAB202754480EA020E65448C
:1006A8000EEA070E69188EEA000E0EEBF165DDF80A
:1006B8004CE07544654405EBB3034FEAB70E1427C5
:1006C8000DF1500CDFF810528EEA010B82EA0B0B89
:1006D8000BEBF36A5CF804BBDA44AA44504483EA9F
:1006E800B10B4FEAF06A8EEA0B0BDA445CF804BBF4
:1006F800DA44AA44524480EAB30B4FEAF26A8BEA1E
:10070800B10BDA445CF804BBDA444FEAB000AA44FF
:1007180080EA020BD6448BEAB30B0BEBFE6A5CF85B
:1007280004BBDA444FEAB202AA4482EA0E0B0AEB8F
:10073800B10180EA0B0B0BEBF16A5CF804BBDA44FD
:100748007F1DAA44282F0AEBB3034FEABE0EBBD382
:100758003C2F61D3502F4DD204EB870CC7F15407BF
:100768005E4CA7FB04A504465D4FA8088EEA010A63
:1007780082EA0A0A5CF804BB0AEBF3655D447D195A
:100788002C1983EAB10A4FEAF4658EEA0A0A55443D
:100798005CF804AB5CF804BB55447D19AA1884EADC
:1007A800B30A4FEAF2658AEAB10A55445D444FEA52
:1007B800B4047D1984EA020AAE448AEAB30A0AEB51
:1007C800FE655CF804AB55444FEAB2027D1982EA33
:1007D8000E0A15EBB10184EA0A0A5CF804BB0AEBBD
:1007E800F1655D447D1915EBB303401E4FEABE0E5B
:1007F800BCD12046F46D1B19F365336EC9183166F8
:10080800716E71447166B36ED218B266F16E40189B
:10081800F06650B0BDE8F08F4EEA010B0EEA010A0F
:100828000BEA020B4BEA0A0A0AEBF36554F827A015
:10083800DFF8B0C0554443EAB10B654403EAB10A96
:100848000BEA0E0B28184BEA0A0A7F1C0AEBF06524
:1008580054F827A0554440EAB30B654400EAB30AAC
:100868000BEAB10BAA184BEA0A0A7F1C0AEBF265DD
:1008780054F827A055444FEAB00040EA020B6544FB
:1008880000EA020A0BEAB30BAE444BEA0A0A7F1CE1
:100898000AEBFE6554F827A055444FEAB20242EA33
:1008A8000E0B654402EA0E0A0BEA000B15EBB101C8
:1008B8004BEA0A0A7F1C0AEBF16554F827A0554455
:1008C8007F1C65443C2F05EBB3034FEABE0EA3D350
:1008D80040E700BF9979825AA1EBD96ECDCCCCCC38
:1008E800D6C162CADCBC1B8F00B581B00168074A5B
:1008F800914200D110B9064801B000BD7C2112F028
:10090800F1FF4FF4003001B000BD00BFFC09000842
:10091800030002002DE9F0410B4A92E8F85188B033
:10092800694681E8F8510268084B9A4200D118B923
:10093800074808B0BDE8F0811422083000F04FFBEA
:1009480008B0BDE8F08100BFDC090008FC09000818
:1009580003000200152904D20268044B9A4200D110
:1009680008B903487047083000F048BBFC09000884
:100978000300020010B481B013460268074CA2427B
:1009880000D118B901B010BC0548704701B000F19A
:10099800240210BC083000F035BB00BFFC09000879
:1009A8000300020010B481B013460268074CA2424B
:1009B80000D118B901B010BC054870470A4601B00B
:1009C80000F1240110BC083000F070BBFC090008DD
:1009D800030002000123456789ABCDEFFEDCBA981E
:1009E80076543210F0E1D2C300000000000000008D
:1009F80000000000F10800081D0900085D09000852
:100A08007D090008AD09000801040008790F0008F5
:100A1800C50F0008810F0008F0B5A3B004460B48C5
:100A280002900D4616461F46094B0822402104A88D
:100A380000F0D1FA28980190009733462A462146BB
:100A480002A800F01BF823B0F0BD00BFFC090008A5
:100A5800100A000810B5040008BF002408D0054893
:100A6800054B20600822402104F1080000F0B3FA89
:100A7800204610BDFC090008100A00082DE9F041C5
:100A880004460E46216817464A681D469047804628
:100A9800B8F5003F19D1226806999368204698470F
:100AA8008046B8F5003F10D123683146DE683A46E3
:100AB8002046B0478046B8F5003F06D12368079A1C
:100AC80029461D692046A847804621680A682046AD
:100AD80090474046BDE8F08110B500F033FA4FF476
:100AE800403400280EBF034C4FF4C07112F0FAFED8
:100AF800204610BD0200030010B5044600F022FA9B
:100B080008B9054810BD0021A160D0F87C21116802
:100B180088474FF4403010BD0200030070B504460A
:100B28000D4600F00FFA064E40B1D0F87C0141683E
:100B38008847A84224BF65604FF44036304670BDF0
:100B4800020003002DE9FF4715000C4600D02CB128
:100B5800064600F0F7F95FEA000801D16448C3E0EF
:100B6800D8F8F80001684A689047B0F5003F17D1F7
:100B7800D8F87C118A68404690478146B9F1810FC0
:100B880080F09E80A94508F1FC0A17D2D8F8F80031
:100B98000368D3F80CC02A462146E047B0F5003F69
:100BA80040F08E80D8F8F8000368D3F810C06A4681
:100BB8005146E047B0F5003F76D10AE0002004E056
:100BC800215C0AF800100098401C00900098A84288
:100BD800F6D34FF0000C4749474A484B01AC009800
:100BE800844558D2D3E9007001ADC5E9007010788A
:100BF80000281ABF042086464FF0000E085854F803
:100C08000E5028443E4D05600127D0F800E087606B
:100C1800019D4F681AF80C007D408EEA050585F0A5
:100C2800040E65680F687D4085F0FC05754485F005
:100C3800A30568400AF80C000CF1010CCFE7D3E9D2
:100C4800004501A8C0E9004510782E4D002814BFC2
:100C58004FF0040E4FF0000E01A8744651F80EE054
:100C68000459A6440127CEF80050DEF80040CEF81B
:100C780008704D68019F40687D406C400D68684071
:100C880084F0040480F0FC00041984F057040AF886
:100C98000C400CF1010CCC45D1D3D8F8F800016810
:100CA8004A689047B0F5003F0AD1D8F8F8000368C1
:100CB800D3F80C804A465146C047B0F5003F01D0F2
:100CC800114811E0002006E05AF8201081F06A313E
:100CD8004AF82010401CB0EB990FF5D3B06840F0EB
:100CE8000100B0604FF4403004B0BDE8F08700BFA9
:100CF80002000300B03A0108D8080020240F0008B9
:100D0800ADBE4ED70DBE75A10100030038B50C4627
:100D1800017A1546CA0702D500F014F908B908483F
:100D280032BDD0F8F80003682146DC682A46A0479F
:100D3800B0F5003F01D0034832BD4FF4403032BD1A
:100D480002000300010003002DE9F84191B00546B7
:100D58000E461746402101A812F0C4FD297AC8079B
:100D680004D5284600F0EEF8040002D1DFF8A4808C
:100D78004BE0D4F8F800DFF8A0800368D3F810C07F
:100D88006A4601A9E047B0F5003F3ED1D4F8F80023
:100D980001684A689047B0F5003F36D1D4F87C1115
:100DA8008A6820469047D4F8F830024618461B68EF
:100DB800D3F80CC004F1FC01E047B0F5003F24D1A2
:100DC800D4F87C0141688847D4F8F83002461846C0
:100DD8001B68D3F80CC001A9E047B0F5003F14D157
:100DE800D4F8F8000268696893689847B0F5003F3E
:100DF8000BD1D4F8F80003681C693A463146A0477D
:100E0800B0F5003F08BF4FF44038404612B0BDE887
:100E1800F08100BF02000300010003002DE9F84142
:100E2800A5B0074688461646402115A812F05AFD77
:100E380000220492402105A812F054FD387AC10717
:100E48005ED5384600F07EF8050059D0D5F8F80090
:100E58002D4C0368D3F810C06A4605A9E047B0F5E1
:100E6800003F3CD1D5F8F80001684A689047B0F5D2
:100E7800003F34D1D5F87C118A6828469047D5F8C8
:100E8800F830024618461B68D3F80CC005F1FC017F
:100E9800E047B0F5003F22D1D5F87C01416888478A
:100EA800D5F8F830024618461B68D3F80CC005A9D7
:100EB800E047B0F5003F12D1D5F8F800026879682C
:100EC80093689847B0F5003F09D1D5F8F800036852
:100ED8001D6904AA15A9A847B0F5003F01D020460E
:100EE8000FE00A4B0A490B4A0396029101924046C9
:100EF8001C68049B009415AA796800F0E5F900E0E5
:100F0800054826B0BDE8F08101000300B83A0108A1
:100F1800936E030026C703000200030004B001011A
:100F280000170145E10A0008010B0008250B00081D
:100F3800B50300084D0B0008150D0008510D0008F9
:100F4800250E00080168024A914218BF0020704728
:100F58002C0F000810B5040008BF002404D0034873
:100F68002060204609688847204610BD2C0F0008DD
:100F780020225C3012F0B4BCF0B58468A3080022CB
:100F880004F0030407E000F15C0555F8226035BA67
:100F980041F82250521C9A42F5D300220BE000F18E
:100FA8005C0502EB830755F82360D500C5F11805E9
:100FB800EE40CE55521CA242F1D3F0BD30B5C46804
:100FC80003690022E31AD5188C5C0544521C082AD0
:100FD8002C77F8D330BD0360C1600261704738B523
:100FE800044615460022626023685A68904700202C
:100FF8006061A061A5604FF4003032BD81604FF49C
:10100800003070472DE9F84304462079D4F80C8065
:10101800450748BF244845D466691D46A8F1010024
:1010280000EAD60306EBC506B6EBC50F666102D229
:10103800A669761CA6611746A66906EB5576A661D1
:101048000E46E918884225D2A8EB03094A463146DC
:10105800F81812F045FC2268136839460FE042463A
:10106800384612F03DFC23681A68394620469047F6
:1010780007E0311811F00300F1D122681368204607
:101088009847484600EB0809A9F10101A942F0D3A5
:10109800002300E000202A1A3118F81812F020FC6A
:1010A8004FF40030BDE8F283040002002DE9FC4F44
:1010B800024685B0D0681369DFF86CC1DFF86C812F
:1010C800A0EB030A506840F004005060002703A812
:1010D80002900DF10C0ED8E9003403A8544DC0E974
:1010E80000342878534D00280CBF00230423994668
:1010F8005CF803305EF80940234401261D601C6833
:101108009E60DCF80430039DDCF80090DEF8046093
:101118005D406540484C654089EA0606474C664094
:101128007519474C6540D8E9006B03AC0028C4E941
:10113800006B0EBF002404200424029E5CF800000B
:10114800345920183F4C04600126046886600398CF
:10115800029E43406340384C7068634089EA00004F
:10116800364C6040034438484340280018BF0120EB
:101178005B1E9B41042F2CBFC0B2D80F02F1140391
:1011880053F8200007F00303C3F10303DB00D84042
:101198000DF807007F1C082F9DD315460C466A6979
:1011A800AB69E868D20842EA4372401E00EA0207C7
:1011B800002302409B420AD8524508D28020E055BD
:1011C8007F1C574516D2AAEB0701E01910E08020D2
:1011D800E05500E0E355E8687F1C8742FAD32A68A7
:1011E800136828469847BAF1000F03D051462046A5
:1011F80012F078FB2A68069E059F93686946284680
:1012080098472A68D2F8009021462846C8472B6894
:10121800DA683946284690470EB1A86830604FF41E
:10122800003007B0BDE8F08FB03A0108541200084A
:10123800D80800205FC5109304850012FC68017A65
:10124800C0F524FF24AF33D426AF698B04B0010165
:1012580000170145F8B501240094002300240DE08F
:10126800009D065D0F5D7E40F643761CF60F86F006
:10127800010635400095641C009DEB189442EFD39D
:101288001846F2BDF8B5002301240094002A11E0A5
:10129800009C85188F1815F8016C17F8015C6E40D2
:1012A800F643761CF60F86F0010634400094009C45
:1012B800E318521EECD11846F2BD00005D1200087A
:1012C8008D120008010000002DE9F84F1D46DDF8D9
:1012D80028900B9F0D9C4FF0FF3300930E469246CB
:1012E800D9F800B0804632465146D847834664B3A1
:1012F800D9F8043032465146404698476FEA0B0207
:10130800521C42EA0B0200996FEAD2735B1C194027
:10131800C2430091521C024300996FEAD2735B1CCE
:101328001940009186F05531484087EA000181F064
:101338005531216080F05531C943491C0843009A52
:101348006FEAD070401C82430092D9F80800012847
:1013580009D17540E943491C0D4300986FEAD572DD
:10136800521C90430AE0F11C85EA9102D243521CB8
:10137800154300986FEAD5735B1C984386F0AA362C
:10138800009086EA0B0686F0AA33F243DB430C98FA
:10139800C2F3C0725B1C42EAD3720099D243521C5A
:1013A80091430091774000998843009987F0AA37C4
:1013B8000F403843BDE8F28F034613F8012B002A8B
:1013C800FBD1181A0138704781F0004102E000BFD4
:1013D80083F0004330B54FEA41044FEA430594EAED
:1013E800050F08BF90EA020F1FBF54EA000C55EA28
:1013F800020C7FEA645C7FEA655C00F0E2804FEAF9
:101408005454D4EB5555B8BF6D420CDD2C4480EADA
:10141800020281EA030382EA000083EA010180EA0A
:10142800020281EA0303362D88BF30BD11F0004F58
:101438004FEA01314FF4801C4CEA113102D040428E
:1014480061EB410113F0004F4FEA03334CEA1333C9
:1014580002D0524263EB430394EA050F00F0A780E1
:10146800A4F10104D5F1200E0DDB02FA0EFC22FADC
:1014780005F2801841F1000103FA0EF2801843FAD0
:1014880005F359410EE0A5F120050EF1200E012AC1
:1014980003FA0EFC28BF4CF0020C43FA05F3C018FF
:1014A80051EBE37101F0004507D54FF0000EDCF178
:1014B800000C7EEB00006EEB0101B1F5801F1BD321
:1014C800B1F5001F0CD349085FEA30004FEA3C0C25
:1014D80004F101044FEA445212F5800F80F09A801B
:1014E800BCF1004F08BF5FEA500C50F1000041EB1F
:1014F800045141EA050130BD5FEA4C0C404141EB23
:101508000101013C28BFB1F5801FE9D291F0000F1D
:1015180004BF01460020B1FA81F308BF2033A3F1CC
:101528000B03B3F120020CDA0C3208DD02F1140CC3
:10153800C2F10C0201FA0CF021FA02F10CE002F1FE
:101548001402D8BFC2F1200C01FA02F120FA0CFCF7
:10155800DCBF41EA0C019040E41AA2BF01EB045140
:10156800294330BD6FEA04041F3C1CDA0C340EDC3E
:1015780004F11404C4F1200220FA04F001FA02F381
:1015880040EA030021FA04F345EA030130BDC4F13F
:101598000C04C4F1200220FA02F001FA04F340EA34
:1015A8000300294630BD21FA04F0294630BD94F0E5
:1015B800000F83F4801306BF81F480110134013DCC
:1015C8004EE77FEA645C18BF7FEA655C29D094EA3D
:1015D800050F08BF90EA020F05D054EA000C04BFBB
:1015E8001946104630BD91EA030F1EBF00210020A6
:1015F80030BD5FEA545C05D14000494128BF41F045
:10160800004130BD14F580043CBF01F5801130BDA8
:1016180001F0004545F0FE4141F470014FF0000033
:1016280030BD7FEA645C1ABF194610467FEA655CE4
:101638001CBF0B46024650EA013406BF52EA033586
:1016480091EA030F41F4002130BD00BF90F0000F74
:1016580004BF0021704730B54FF4806404F13204B0
:101668004FF000054FF0000150E700BF90F0000F69
:1016780004BF0021704730B54FF4806404F1320490
:1016880010F0004548BF40424FF000013EE700BF60
:1016980042004FEAE2014FEA31014FEA02701FBFF0
:1016A80012F07F4393F07F4F81F06051704732F022
:1016B8007F4208BF704793F07F4F04BF41F4002179
:1016C800704730B54FF4607401F0004521F00041D7
:1016D8001CE700BF50EA010208BF704730B54FF061
:1016E80000050AE050EA010208BF704730B511F062
:1016F800004502D5404261EB41014FF4806404F19A
:1017080032045FEA915C3FF4D8AE4FF003025FEA1F
:10171800DC0C18BF03325FEADC0C18BF033202EBA3
:10172800DC02C2F1200300FA03FC20FA02F001FAFD
:1017380003FE40EA0E0021FA02F11444BDE600BFA0
:101748004FF0FF3C06E000BF4FF0010C02E000BF85
:101758004FF0010C4DF804CD4FEA410C7FEA6C5C68
:101768004FEA430C18BF7FEA6C5C1BD001B050EA0B
:10177800410C0CBF52EA430C91EA030F02BF90EAF6
:10178800020F0020704710F1000F91EA030F58BFB5
:10179800994208BF90422CBFD8176FEAE37040F017
:1017A800010070474FEA410C7FEA6C5C02D150EAB5
:1017B800013C07D14FEA430C7FEA6C5CD6D152EA70
:1017C800033CD3D05DF8040B704700BF8446104635
:1017D80062468C461946634600E000BF01B5FFF734
:1017E800B7FF002848BF10F1000F01BD4DF808ED04
:1017F800FFF7F4FF0CBF012000205DF808FB00BFD5
:101808004DF808EDFFF7EAFF34BF012000205DF82E
:1018180008FB00BF4DF808EDFFF7E0FF94BF01207B
:1018280000205DF808FB00BF4DF808EDFFF7CEFF7C
:1018380094BF012000205DF808FB00BF4DF808EDBB
:10184800FFF7C4FF34BF012000205DF808FB00BF8C
:101858004FEA410212F5001215D211D56FF47873D0
:10186800B3EB625212D94FEAC12343F0004343EA73
:10187800505311F0004F23FA02F018BF404270474E
:101888004FF00000704750EA013005D111F00040D8
:1018980008BF6FF0004070474FF00000704700BF6E
:1018A80080F0004002E000BF81F0004142001FBF0D
:1018B8005FEA410392EA030F7FEA226C7FEA236C16
:1018C8006AD04FEA1262D2EB1363C1BFD21841400B
:1018D80048404140B8BF5B42192B88BF704710F0A1
:1018E800004F40F4000020F07F4018BF404211F044
:1018F800004F41F4000121F07F4118BF494292EAAC
:10190800030F3FD0A2F1010241FA03FC10EB0C00D7
:10191800C3F1200301FA03F100F0004302D5494264
:1019280060EB4000B0F5000F13D3B0F1807F06D311
:1019380040084FEA310102F10102FE2A51D2B1F109
:10194800004F40EBC25008BF20F0010040EA0300FE
:101958007047490040EB0000013A28BFB0F5000F7E
:10196800EDD2B0FA80FCACF1080CB2EB0C0200FA34
:101978000CF0AABF00EBC25052421843BCBFD04083
:101988001843704792F0000F81F4000106BF80F4FD
:1019980000000132013BB5E74FEA41037FEA226CC0
:1019A80018BF7FEA236C21D092EA030F04D092F08B
:1019B800000F08BF0846704790EA010F1CBF0020BF
:1019C800704712F07F4F04D1400028BF40F000401C
:1019D800704712F100723CBF00F50000704700F03C
:1019E800004343F0FE4040F4000070477FEA226263
:1019F80016BF08467FEA23630146420206BF5FEA34
:101A0800412390EA010F40F4800070474FF0000333
:101A180004E000BF10F0004348BF40425FEA000CFA
:101A280008BF704743F0964301464FF000001CE0A2
:101A380050EA010208BF70474FF000030AE000BFF8
:101A480050EA010208BF704711F0004302D5404236
:101A580061EB41015FEA010C02BF844601460020A8
:101A680043F0B64308BFA3F18053A3F50003BCFAC3
:101A78008CF2083AA3EBC25310DB01FA02FC634470
:101A880000FA02FCC2F12002BCF1004F20FA02F277
:101A980043EB020008BF20F00100704702F120026A
:101AA80001FA02FCC2F1200250EA4C0021FA02F2CB
:101AB80043EB020008BF20EADC7070474FEA40029F
:101AC800B2F1FE4F0FD34FF09E03B3EB12620DD964
:101AD8004FEA002343F0004310F0004F23FA02F0CE
:101AE80018BF404270474FF00000704712F1610F75
:101AF80001D1420205D110F0004008BF6FF000404C
:101B080070474FF00000704753B94AB9002908BF21
:101B180000281CBF4FF0FF314FF0FF3000F06AB9CA
:101B2800ADF1080C6DE904CE00F006F8DDF804E02C
:101B3800DDE9022304B070472DE9F047089D0C4603
:101B4800002B4ED194468C458646B2FA82F262D971
:101B58004AB1C2F12003914020FA03F30CFA02FCC7
:101B6800194300FA02FE4FEA1C471FFA8CF6B1FB34
:101B7800F7F44FEA1E4307FB141143EA014304FB41
:101B880006F199420AD91CEB030304F1FF3080F0F7
:101B98001281994240F20F81023C6344591A1FFA9C
:101BA8008EF3B1FBF7F007FB101143EA014300FB8A
:101BB80006F69E420AD91CEB030300F1FF3180F0C0
:101BC800FC809E4240F2F980634402389B1B40EA45
:101BD800044000211DB1D3400022C5E90032BDE810
:101BE800F0878B4205D90DB1C5E9000100210846EF
:101BF800F5E7B3FA83F1002946D1A34202D3904214
:101C0800C0F0F080861A64EB03030120002DE6D0B3
:101C1800C5E90063E3E7002A40F09080A1EB0C04DB
:101C28004FEA1C481FFA8CF70121B4FBF8F64FEA7B
:101C38001E4308FB164443EA044307FB06F0984298
:101C480008D91CEB030306F1FF3402D2984200F2D4
:101C5800CD8026461C1A1FFA8EF3B4FBF8F008FB59
:101C6800104443EA044300FB07F79F4208D91CEBE2
:101C7800030300F1FF3402D29F4200F2B0802046F5
:101C8800DB1B40EA0640A5E7C1F120068B4022FA9B
:101C980006F71F4320FA06FC04FA01F343EA0C0393
:101CA800F44000FA01F8380C4FEA1349B4FBF0FE8F
:101CB8001FFA87FC00FB1E4449EA04440EFB0CF99A
:101CC800A14502FA01F20AD93C190EF1FF3A80F057
:101CD8008480A14540F28180AEF1020E3C44A4EB21
:101CE80009041FFA83F9B4FBF0F300FB134449EA33
:101CF800044403FB0CFCA44507D93C1903F1FF304D
:101D080067D2A44565D9023B3C4443EA0E40A0FB98
:101D18000293A4EB0C049C42CE469C4651D34ED071
:101D280055B1B8EB0E0364EB0C0404FA06F6CB408D
:101D38001E43CC40C5E90064002150E7C2F12003EE
:101D480020FA03F10CFA02FC24FA03F394400C4342
:101D58004FEA1C4800FA02FE1FFA8CF7B3FBF8F0B2
:101D680008FB1031230C43EA014300FB07F19942B9
:101D780008D91CEB030300F1FF362CD299422AD96B
:101D8800023863445B1AA4B2B3FBF8F108FB1133C1
:101D980044EA034401FB07F3A34208D91CEB0404FB
:101DA80001F1FF3613D2A34211D902396444E41A6F
:101DB80041EA004139E70446F0E6084606E7C84527
:101DC800AED2B9EB020E63EB070C0138A8E7314637
:101DD800EDE7034699E73046D4E7D6467FE7634404
:101DE80002384DE70646234608460FE7023E63449D
:101DF80030E700BF704700BF1348144A08B54FF0DA
:101E08000043C0E900230422426101220023C26189
:101E18004FF480510722C0E90233C0E90933C0E911
:101E28000C1203610383837680F8203080F82C300D
:101E3800826380F83C30C36404F0DEFE18B1BDE86C
:101E4800084000F0F5BB08BDDC0800200024014074
:101E58000268084B9A4282B00AD14FF0B0431A6E1A
:101E680042F400721A661B6E03F400730193019B1F
:101E780002B07047002401400268054B9A4201BF36
:101E88004FF0B042136E23F400731366704700BF1F
:101E98000024014030B585B000240546CDE9014451
:101EA8000394FFF7A9FF144805F03AFA08B100F0C7
:101EB800BFFB1148039401A9CDE9015404F0FAFFCE
:101EC80008B100F0B5FB0C4805F054F908B100F072
:101ED800AFFB4FF0FF31084804F08EFF064805F0CD
:101EE80001FA054804F0E2FF0446034805F0A4F9A6
:101EF800204605B030BD00BFDC080020014B024A77
:101F08001A607047DC0800200024014008B5094821
:101F1800FFF7C0FF68B1084BB3F8AA304FF6FF725D
:101F2800934216BF40F6E442044B5343B3FBF0F32D
:101F380098B208BD002000B40075FF1FD8084C00F7
:101F480013B50023ADF80630FFF7E0FF0446194843
:101F5800FFF7A0FF184BB3F8C820B3F8A8108A42BF
:101F680004FB00F018D040F6E443B0FBF3F3642020
:101F78005B1A4343521A93FBF2F31E331BB2ADF8BC
:101F88000630BDF806305BB21B02ADF80630BDF86E
:101F9800060000B202B010BD4FF47A7240F6FF732B
:101FA800B0FBF3F35343A3F53923A3F50C6340F6D1
:101FB800C412E0E7001000B00075FF1F4FF0B043F7
:101FC80082B09A6A22F480529A629A6C42F48052E1
:101FD8009A649B6C03F480530193019B002002B028
:101FE80070474FF0B04307B59A6C42F004029A6408
:101FF8009A6C02F004020192019A9A6C42F0010272
:102008009A649B6C002203F00103114600930E2092
:10201800009B05F023FA0E2005F052FA0022114623
:102028000F2005F01BFA0F2003B05DF804EB05F054
:1020380047BA000008B505F01DFC10B16FF00400A8
:1020480008BD064B9A6942F040429A614CF2FA3256
:102058001A6105F021FC0028F2D0EFE70040005893
:10206800F0B585B000230D4600930646A8B3FFF7E8
:10207800E1FF044670BB05F0FDFB88BB1A481B4A0C
:1020880002230193D0F8E01506F1784302EA812192
:10209800B3FBF1F701FB1733DB0A0293D0F8E00535
:1020A80005F178410139314402EA8022B1FBF2F0AE
:1020B80002FB1011C3EBD1230133694601A8039336
:1020C80005F06AFC20B1022814BF6FF00104012456
:1020D80005F0E2FB204605B0F0BD6FF00504F9E716
:1020E8006FF00404F6E700BF0070FF1F00FCFF0359
:1020F800014B186000207047400900202DE9F04F7F
:10210800B0F1006F89B006460F469046C0F0C08017
:10211800DFF89091644DD9F8E03505EA832303F19F
:102128000063013B984200F2B380002900F0B380BD
:1021380040EA02035B0740F0AE80FFF77BFF0446EE
:1021480090BB05F097FB002840F0A880D9F8E0156F
:10215800009705EA812106F17842B2FBF1F301FB11
:10216800132208F17843013B3344B3FBF1F001FB40
:102178001033DB0A01334FEAD22AA3EBD222012A19
:10218800039388BFC6F30A050AF58037C6F108032A
:102198008CBFC5F500654546FF02B3460693039B11
:1021A8009A4505D305F078FB204609B0BDE8F08FC5
:1021B800A6F10803069A1A4495421CD8009B049578
:1021C8000193CDF814B04FF00009059B09EB03010A
:1021D800049B99453DD3009BAB442B44A8EB0505D4
:1021E800B5F5006F009328BF4FF400650AF1010AA6
:1021F80007F50067D3E753F8081F5A68B2F1FF3FA5
:1022080008BFB1F1FF3FD5D0284B186810B96FF05F
:102218000504C7E727B14FF40062394610F0F0FE15
:10222800DFF888900099D9F80030CBF30A001844F9
:10223800AAB210F0E5FE4FF400613846FFF710FF30
:1022480000BBD9F8003001934FF40063059704935D
:10225800B9E7019B07914B4402930120D3E900237E
:1022680005F054FB88B90799019BD1E9000259F898
:102278000310029B5B689A4208BF884205D109F1A6
:102288000809A2E76FF001048CE76FF0030489E7FF
:102298004FF0FF3488E76FF0050485E76FF004041A
:1022A80082E700BF0070FF1F00FCFF034009002009
:1022B800B1F1006F70B510D30B4BD3F8E0650B4B41
:1022C80003EA862303F10063013B994205D838B13C
:1022D80092B210F095FE002070BD4FF0FF30FBE782
:1022E8006FF00500F8E700BF0070FF1F00FCFF0358
:1022F800B0F1006F10B40DD3084BD3F8E045084B8C
:1023080003EA842303F10063013B984202D810BC1E
:10231800FFF7A6BE4FF0FF3010BC70470070FF1FDC
:1023280000FCFF034FF0B04382B0DA6C0243DA647A
:10233800DB6C03400193019B02B07047F0B50120AC
:1023480087B00024364DCDE90444FFF7EBFF0220A7
:10235800FFF7E8FF0420FFF7E5FF0DEB00014FF65C
:10236800FF7203232846CDE90123039405F062FB9D
:1023780001A92C4805F05EFB01A94FF0904005F03B
:1023880059FB4FF0B0422846D36C23F00403D364C2
:102398002021012205F074FC0220FFF7C3FF082763
:1023A8004FF4041601A92846CDE90176039405F0F7
:1023B80041FB01A92846CDE901760394012605F0E1
:1023C80039FB202301A92846CDE90136CDE903646C
:1023D80005F030FB4FF4007301A94FF09040CDE9B0
:1023E8000136CDE9036405F025FB102301A9284631
:1023F800CDE90136CDE9034405F01CFB2246214610
:10240800092005F02BF8092005F05AF82246214644
:10241800092005F023F8092005F052F807B0F0BDAF
:10242800000400480008004808B51248124A134B37
:10243800C0E9002300230122C0E90232C0E90433C5
:10244800C0E90633036205F08FFD08B100F0F0F82B
:102458000848002105F008FF08B100F0E9F8054830
:10246800002105F027FF18B1BDE8084000F0E0B8EA
:1024780008BD00BF040A0020005800405D3E30201F
:1024880070B596B005461422002103A811F0F4F99E
:102498003822002108A811F0EFF92A68304B9A4237
:1024A8005BD18023089308A84FF440230E9306F0CD
:1024B8006FFC08B100F0BCF84FF0B0444FF4C050C6
:1024C800E36C43F00103E364E36C03F0010302935C
:1024D800029B12230026CDE903030323CDE90563FC
:1024E8004FF09040042303A9079305F0A3FAA36DC6
:1024F800DFF870C043F48003A365A36D1A4C03F49E
:1025080080030193019B26620D23C4E900C3204682
:102518008023C4E90266C4E90436C4E9066605F006
:102528002FF808B100F084F8104AEC63A562104C4B
:102538000E23C4E900231021002380222046C4E989
:102548000213C4E90423C4E90633236205F018F82A
:1025580008B100F06DF8AC63A56216B070BD00BF9D
:102568000058004044000240A409002058000240DE
:102578004409002000B59BB04822002108A811F0AA
:102588007BF91822002102A811F076F905F0B8FEAF
:102598004FF0B0420120D2F8903023F01803C2F86F
:1025A8009030D2F8003423F4C06343F40073C2F8C7
:1025B8000034D2F8003403F4C0630193019B242350
:1025C800089381230B930023CDE91003B02208A8B8
:1025D800CDE9122306F01EF808B172B6FEE74F23C4
:1025E800CDE90230CDE90400CDE90600022102A8B8
:1025F80006F0AAFA08B172B6FEE71BB05DF804FB54
:1026080008B504F0BFFAFFF7B5FFFFF797FEFFF72D
:10261800E8FCFFF709FF00F04EFD044807F0B2F9A7
:1026280000F07AFC00F04EFDFCE700BF340B002000
:1026380072B6FEE70F4808B50F4B03601F2383608F
:102648004FF080420023C0E90433C0E907238361C7
:102658004FF48073436206F01DFD08B1FFF7E8FFF1
:10266800044806F043FE18B1BDE80840FFF7E0BF94
:1026780008BD00BF580A00200028004010B50446D5
:1026880090B03822002102A811F0F6F82268194B00
:102698009A422CD14FF48033029302A84FF48073EE
:1026A8000F9306F075FB08B1FFF7C2FF4FF0B04378
:1026B8000220D3F8902042F40042C3F890209A6D8B
:1026C80042F480629A659B6D002203F48063114690
:1026D8000193019B04F0C2FE022004F0F1FE0022E7
:1026E8002A20114604F0BAFE2A2004F0E9FE10B0B0
:1026F80010BD00BF0028004010B50E4C0022204637
:10270800102105F0BDFA4FF6FF714FF0904005F02B
:102718003DFA20464FF6FF7105F038FA06484FF6A5
:10272800FF7105F033FA04F043FABDE8104005F0F4
:102738000FBE00BF000400480008004808B5044860
:102748000122102105F09CFABDE8084004F037BAD0
:102758000004004804F033BA10B5104C002220469B
:10276800102105F08DFA4FF6FF714FF0904005F0FB
:102778000DFA20464FF6FF7105F008FA08484FF6A3
:10278800FF7105F003FA04F013FA064B0120BDE8C7
:102798001040C3F8880005F01DBE00BF00040048C3
:1027A800000800480004005808B504F008FA064874
:1027B8000122102105F064FAFFF7C0FDFFF711FCB4
:1027C800BDE80840FFF730BE0004004808B504F033
:1027D800EFF9BDE808400121002005F099BD7047D8
:1027E800FEE7FEE7FEE7FEE7FEE770477047704743
:1027F80070470000014806F09FBD00BF580A00203E
:10280800014804F0C9BF00BFA4090020014804F032
:10281800C3BF00BF44090020082005F037BA0000F4
:10282800014806F0BDBB00BF580A0020014806F069
:10283800ACBF00BFBC0A00202DE9F04389B0804638
:102848000020109E0790894615461F46FDF7E8FCB4
:10285800F0B9104CCDE90090CDE9020407AB0E4861
:102868000593142304933A46434629460068FDF726
:10287800A1FD2346324604F1140153F8044B42F8F3
:10288800044B8B42F9D1079B337509B0BDE8F0833F
:102898000120FAE7A60A0020AC3A01081FB50E4C41
:1028A80000233C2202A8CDE902336275237500F0AB
:1028B800B7F8042303AA009412210848FFF7BCFFC5
:1028C80007491422204610F0C7FFB0FA80F35B09CD
:1028D800637504B010BD00BF900A0020D43A010807
:1028E800E50D0020054808B50823036006F06AFDD9
:1028F80018B1BDE80840FFF79BBE08BDBC0A002020
:102908004FF0B04307B55A6E42F001025A665B6E4B
:10291800002203F00103019311463220019B04F0C9
:102928009DFD322003B05DF804EB04F0C9BD000042
:102938000CB407B5054A05AB1021019310F06AFEE7
:1029480003B05DF804EB02B0704700BFE63A010837
:1029580030B585B0044602A80D4610F087FCBDF9D5
:102968000C30064A00931021029B2046FFF7E0FF37
:102978002046FEF721FD288005B030BDE63A010863
:102988004FF0B04210B5936823F40043936010F001
:10299800F5FC0D4B01241C7010F0C2F90B4810F027
:1029A800D9F90B4B4FF400421A61002010F0D8F906
:1029B800FFF7A4FA00F0B4F810F0CCFA214620464C
:1029C800BDE8104010F0E6BAC80A002059290008EE
:1029D8000040005810F0F4BA08B5FFF797FA40F62F
:1029E800B83398420CD8B0F5E16F0BD3FE23A0F5AD
:1029F800E16058434FF49663B0FBF3F0C0B208BDF2
:102A0800FE20FCE70020FAE77FB5684600F06CF886
:102A18000198FFF753F800B207B05DF804FB000017
:102A2800194A38B5D2F88035591C044619D104F032
:102A3800CDF8054604F0D6F8054404F0CDF82B0E81
:102A4800E3712B0CA3712B0A6371030EE370C0F3BF
:102A58000742C0F307232571C0B2A27063702070CB
:102A680038BD190AC3718171190C1B0E41710371AC
:102A7800D2F88435C370D2F88405C0F30722C0F3B6
:102A88000743000EE9E700BF0070FF1F38B5094B88
:102A9800D3F8803503600133054609D104F096F870
:102AA800044604F099F8444004F09CF844402C6033
:102AB80038BD00BF0070FF1F0121022010F054BA7A
:102AC8000021022010F050BA00207047024B1878FD
:102AD80008B100F05DB87047C80A002082B00190C4
:102AE800019802B000F0F0B810B50446FFF728FAD4
:102AF800074BA36040F30F20FEF78CFF054B064AF7
:102B08002360064B6060C4E90323002010BD00BFAA
:102B18000000484200007A440D093E00AB0305005E
:102B280000207047014B1868704700BFCC0A00208E
:102B38000320704708B501464FF47A7200238002DB
:102B4800890DFEF7E1FF08BD4FF47A73A0FB03037C
:102B5800800A40EA83507047034B98689A6890420D
:102B6800FBD1C043704700BF0028004008B5FFF7FD
:102B7800F3FF014B186008BDCC0A002008B5FFF729
:102B8800EBFF024B1B68C01A08BD00BFCC0A00202F
:102B9800024B187808B1FFF7DFBF7047D00A002052
:102BA80010B5074B074C0122DA654FF480712046B7
:102BB80006F0BCF94FF0FF332363002010BD00BFBF
:102BC80000280040580A002002460021014806F06B
:102BD800C4BB00BF580A002002460121014806F084
:102BE800BCBB00BF580A002010B58CB02C220021B5
:102BF800044601A810F040FEFFF7D2FF0C4B0D4829
:102C08001B681C440023089306934FF00053E443C9
:102C1800079301224FF4807301A902940B9306F0E5
:102C280099FA08B1FFF704FD00200CB010BD00BFF1
:102C3800CC0A0020580A002038B50546FFF78CFF5B
:102C480002210446074806F08FFBC4F309024FF43B
:102C58007A71A2FB0121920AA30A2A8043EA8050D2
:102C680038BD00BF580A00200148002106F07CBB8F
:102C7800580A00200148012106F076BB580A0020B6
:102C8800F8B50F4D2E78CEB90E4C4FF0FF372763AD
:102C9800FFF7D0FCFFF784FF4FF48071204606F061
:102CA80045F92046276306F003FB324620460221F9
:102CB80006F053FBFFF75AFF01232B700020F8BDE5
:102CC800D00A0020580A0020014610B54FF47A7245
:102CD80000238002890DFEF717FF0146FFF73CFF2E
:102CE8000446FFF739FF031B8B4200D310BD00BF1A
:102CF800F7E710F04BBC000010B5064C0221204647
:102D080006F032FB0221421C2046BDE8104006F0C6
:102D180024BB00BF580A00201348144A08B54FF4D2
:102D2800E133C0E9002300230C22C0E90233C0E9E3
:102D38000523C0E90733C0E90933036107F03DFB08
:102D480008B1FFF775FC0848002107F0ABFC08B193
:102D5800FFF76EFC044807F085FC18B1BDE8084091
:102D6800FFF766BC08BD00BF340B002000440040DC
:102D780070B596B006461422002103A810F07CFD19
:102D88003822002108A810F077FD32682C4B9A42AF
:102D980053D10223089308A82A4B0A9305F0F8FF99
:102DA80008B1FFF745FC4FF0B04300259A6D42F497
:102DB80000329A659A6D02F400320292029ADA6C35
:102DC80042F00102DA64DB6C03F001030193042290
:102DD800019B0223CDE903230324072303A94FF012
:102DE8009040CDE90554079304F024FE082303A975
:102DF8004FF09040CDE903340595134C04F01AFECA
:102E0800124925621423C4E900131023C4E90235CA
:102E180020468023C4E90435C4E9065504F0B0FB14
:102E280008B1FFF705FC2520F46700220221A662FD
:102E380004F014FB252004F043FB16B070BD00BF5E
:102E48000044004004000C00D40A00208000024026
:102E580002680C4B9A4210B5044612D14FF0B042AA
:102E68000C21936D23F4003393654FF0904004F0E8
:102E78008DFEE06F04F0F6FBBDE81040252004F05D
:102E88002DBB10BD0044004008B50A460146024863
:102E980006F098FD002008BD340B002013B5114B37
:102EA800114C18604FF40013009302AB13E90600AD
:102EB800204607F07BFB2368DA69D103FCD4DA6982
:102EC8005202FCD59A68084842F480029A6007F0DA
:102ED800B3FB06490448012207F024FB002002B096
:102EE80010BD00BFC80B0020340B0020D00B002001
:102EF80008B5074B1860FFF774F8FFF70DFF054A90
:102F0800D2F8803043F00063C2F88030002008BD5A
:102F1800CC0B00200008005808B54FF0B043084813
:102F28009A6B42F400329A639A6B22F400329A63E5
:102F3800FFF78EFF112004F0D1FA002008BD00BF72
:102F4800340B00200268044B9A4203D1034B002043
:102F58001B681847704700BF00440040CC0B002096
:102F680002680B4B9A4210B504460FD1094B1B68F7
:102F78002BB1D0F8902012B9074801219847204674
:102F88000549BDE81040012207F0CCBA10BD00BFCA
:102F980000440040C80B0020D00B0020024801224A
:102FA800102104F06DBE00BF000400480248002252
:102FB800102104F065BE00BF0004004810B50A4C9B
:102FC80023780BB9E37C6BB1FFF768FC0038074B3B
:102FD80018BF0120400018701B78022B02BF002385
:102FE8002370E37410BD00BFE50D0020D80B00204E
:102FF80038B5114C2378F3B9E37CE3B90F4D2B684E
:10300800012B07D92B68042B04D80D4A0421012071
:1030180000F00EFA2B68042B0DD9FFF73FFC00389F
:10302800084B18BF0120400018701B78022B02BF04
:1030380000232370E37438BDE50D0020D40B002075
:10304800403B0108D80B002008B5FFF7A7FF01F0A7
:1030580021FABDE80840FFF7A9BF022801D8FFF709
:103068009DBF7047022801D8FFF7A0BF7047000036
:10307800022808B51BD8012210210D4804F000FED3
:103088003220FFF72BFD0A480022102104F0F8FD3A
:1030980001221021064804F0F3FD3220FFF71EFD3F
:1030A800BDE8084002480022102104F0E9BD08BD2F
:1030B80000040048704708B5FFF762FCBDE8084007
:1030C80000F056BB4FF0FF300FF0DEBF704770477F
:1030D80070470000014BD870704700BF0C000020FB
:1030E800014B1874704700BF0C00002008B502207F
:1030F80000210FF091FFBDE80840014810F0F4B935
:10310800480D0020002101200FF086BF10B542F2C3
:103118001073084C002818BF03460748236010F0B6
:1031280095F92168044810F019FABDE810400248E2
:1031380010F0DAB908000020480D002010B5094C3D
:10314800206023680BB9084B2360084810F07EF90B
:103158002168064810F002FABDE81040034810F054
:10316800C3B900BFB4000020A0860100DC0B00201A
:1031780010B5044680B190F906306BB9094810F0D3
:1031880065F9094BE2791A70084B1868FFF7D6FF02
:10319800074B1868FFF7BAFFBDE81040002102206E
:1031A8000FF03ABFF40B0020E20D0020B40000201D
:1031B800080000200A460149FFF77AB800F0030822
:1031C80038B50C4810F042F907F0CCFE60B90A4C4B
:1031D8000A480125257007F059FD2078294607F08F
:1031E800ADFA044810F080F9BDE83840044810F002
:1031F8007BB900BF480D0020700000200C000020A3
:10320800300D002007F04CBF30B585B0FFF7E4FB68
:10321800044607F08DFB054688B100243C4810F0B1
:1032280015F93C4B3A481B689C42214638BF194661
:1032380010F094F9364810F057F905B030BD014642
:103248004FF480700FF0E8FE684601F007F823B2EB
:1032580003EB4303FE2203EB4313B3FBF2F32E4AC3
:10326800392111702D4950680978DBB28DF80C307E
:103278000170506845705068272484705068012494
:10328800C47050680371264B187818B31D705368C2
:1032980061F07F0119703A23137005232149224CEC
:1032A8000978012988BF00235370637A33B107F086
:1032B8002BFB012802D1204610F0C8F81B4B1648FA
:1032C800D978002207F04AFB0630A6D107F016FB92
:1032D8000446A3E7164B1748197811B90178002955
:1032E800DBD0002101701970536804215971BDF8B1
:1032F80000305168180A88715168CB71BDF80830E0
:1033080051681B0A0B72BDF808304B720A23C5E7D7
:10331800480D002008000020000000203C0C002080
:10332800E10D0020D80B0020F40B00200C00002039
:10333800600D0020E30D002020B1037813B102488E
:1033480010F0D2B8704700BF240C002008B5104B0D
:103358000122002102201A700FF05EFE0D4810F0C5
:10336800C3F80D4B1B788BB10C4B1A7872B9DB7C08
:1033780063B90B4B1A68042A9EBF1A6801321A6097
:103388000021BDE8084010200FF046BE08BD00BF70
:10339800E10D0020DC0B0020E20D0020E50D0020EF
:1033A800D40B0020044B1B78022B03D100210820EA
:1033B8000FF032BE704700BF7000002008B507F05C
:1033C800DAFD80B907F0A0FA01280CD1BFF34F8FBE
:1033D8000549064BCA6802F4E0621343CB60BFF3A9
:1033E8004F8F00BFFDE708BD00ED00E00400FA05BF
:1033F80038B504460D4607484FF40061FEF778FFDC
:1034080030B92A4621460348BDE83840FEF776BE63
:1034180038BD00BF00F00308704770477047704719
:10342800082802BF014B01221A707047600E002065
:1034380070B505460C46164607F07AFA034600288A
:1034480035D000241B4810F001F81B4B19481B68A5
:103458009C42214638BF194610F080F8BDE87040FC
:10346800144810F041B84A68F05CD0540133DAB21D
:103478009442F8D8114B0D701B78012B88BF00249B
:103488004C700F4C637A33B107F03EFA012802D131
:1034980020460FF0DBFF0B4B0B48D978002207F0D2
:1034A8005DFA0630CDD107F029FA0446CAE7064985
:1034B800DDE700BF480D002008000020D80B0020E1
:1034C800F40B00200C00002000000020044B1B78A7
:1034D80023B9044A05210120FFF7AABF704700BF9E
:1034E800D80B0020453B010810B5002490B03C22C1
:1034F800214601A8009410F0BFF92F4B2022DA7260
:1035080019788DF8001059788DF8011099788DF890
:103518000210D9788DF8031019798DF804105979AB
:103528008DF8051099798DF80610D9798DF807105E
:10353800197A8DF80810597A8DF80910997A8DF84A
:103548000A108DF80B2021460DF10B025818013195
:10355800007B02F8010F1C29F8D193F828208DF878
:10356800282093F829208DF8292093F82A208DF80F
:103578002A2093F82B208DF82B2093F82C206AB161
:1035880093F83F2052B10DF12B0100229818013217
:1035980090F82C0001F8010F142AF7D107484FF4CE
:1035A8000061FEF7A5FE20B9044840226946FEF7EF
:1035B800A5FD10B010BD00BF7100002000F8030881
:1035C800014940220FF01CBD00F8030870B52A4DD0
:1035D80028796B794D2BC0B233D1C0EB0010800035
:1035E8000A2838BF0A204FF47A735843234BAC7922
:1035F8001860EB794D2BE4B22BD1C4EB0414A40072
:1036080095F82C301E4E63BB95F83F304BBB42F209
:103618001070FFF77BFD3068FFF790FD2B7A194A91
:103628001949DBB213706B7A184ADBB213700023A6
:10363800EA1892F82C20D2B2CA540133142BF7D1CD
:1036480070BD6B79482B0ABF4FF461636B7958439F
:10365800C6E7EB79482B0ABF4FF46163EB795C430B
:10366800CEE7FFF753FD012C38BF01244FF47A73DE
:103678005C433460CFE700BF7100002008000020E1
:10368800B4000020E40D0020E50D0020D80B002038
:1036980010B590B000213C2201A8009110F0ECF880
:1036A8004022314968460FF0ABFC9DF800203AB93A
:1036B8009DF80100272803D19DF80210012909D09F
:1036C800FFF712FF4FF47A70FFF708FAFFF77EFF53
:1036D80010B010BD254B1A70587099709DF80310E2
:1036E800D9709DF8041019719DF8051059719DF84D
:1036F800061099719DF80710D9719DF80810197274
:103708009DF8091059729DF80A1099729DF80B10CE
:1037180001F03F01D972D87AD1B288421BD89DF8FE
:10372800282083F828209DF8292083F829209DF84F
:103738002A2083F82A209DF82B2083F82B200DF1CE
:103748002B0100229818013211F8014F80F82C4003
:10375800142AF7D1BAE701F140006844194410F877
:10376800340C08730132D6E700F803087100002012
:103778001FB5002403A92046039407F0E1FB03A921
:10378800012007F0DDFB384B3848009422464FF4FF
:10379800FA710FF0FDFD364B3648009422464FF47F
:1037A800FA710FF0F5FD344B3448009401224FF4C0
:1037B800FA710FF0EDFD2046FEF79AFC08B1FEF70E
:1037C80037FF2F4B009400224FF4FA612D480FF079
:1037D800DFFD2D4A002101200FF0DAFC2B4A0021E1
:1037E80002200FF0D5FC2A4A002104200FF0D0FC5B
:1037F800284A002108200FF0CBFC00F0ABFB26493B
:10380800264807F053FB264807F040FA1B480FF0FC
:103818006BFE244B0021187806F090FF2249009493
:10382800224B0968224800220FF0B2FD20480FF011
:103838005BFEFFF72DFF1F4A002110200FF0A8FCA8
:103848001D4A00214FF480700FF0A2FC1B4B1C484E
:1038580019681C4B009400220FF09AFD18480FF0CD
:1038680043FE04B010BD00BF25340008240C00201E
:10387800273400080C0C002021340008F40B002029
:10388800AD330008300D002099AA00081132000855
:103898000D320008C931000800000301240000208F
:1038A8000C0000207000002008000020F5300008FF
:1038B800480D0020F92F000851300008B4000020FE
:1038C800DC0B00205533000810B50024A2B07C2280
:1038D800214603A802940FF0CFFF53238DF8083038
:1038E80040F22713ADF80A3001238DF80C30ADF8FB
:1038F8000440FFF771F800B200EB400000EB401005
:10390800FE23B0FBF3F08DF80D0001A800F0B6FC23
:10391800A0B958238DF80E3007243022802114488E
:103928000FF0AAFF224602A911480FF0DEFF104A45
:1039380021460120FFF77CFD22B010BD4300013372
:103948008DF80E308DF80F0000F0A4FD094B1A68B1
:1039580012128DF810201A688DF811205A685B68C9
:103968008DF8133012128DF812200C24D5E700BF01
:10397800610D0020640E002030B50378592B91B0FA
:10398800044640F00082052959D84378443B162B59
:1039980055D8DFE813F03D0154002D0154003501DE
:1039A800540054005400540094005400180154006A
:1039B80054005400A70154005400B00054005400AF
:1039C800540017008578482D11D1BC4A14210120D4
:1039D800FFF72EFD41F28830FFF780F840F6B83047
:1039E800FFF77CF811B0BDE83040FFF7E7BC532D76
:1039F8000ED130228021B2480FF03EFFFFF764FF5E
:103A080041F28830FFF76AF8AD4A1521012086E0B7
:103A1800432D16D1002468468DF8004007F0AEF813
:103A2800A74A4C231370272393709DF800305470D5
:103A380001204133D07013710521FFF7F9FC11B053
:103A480030BD442DFBD19E4C592323705A236370FB
:103A5800A57000F0F5FB2B228021601D0FF00CFFF4
:103A680000232570637001252723A370E570257155
:103A7800FEF7B2FF9349FE23B0FBF3F00B68642214
:103A88009BB2B3FBF2F3A3710B6800EB400000EBB1
:103A980040109BB26071B3FBF2F002FB1033E3718C
:103AA8004B689BB2B3FBF2F323724B689BB2B3FB38
:103AB800F2F102FB1133637222460A21A6E78378EA
:103AC800303BDBB2092BBAD87F49804A0B700B78A0
:103AD800DBB253727A4A592313704D2353700B7813
:103AE8000120303303219370FFF7A2FC11B0BDE829
:103AF8003040FFF7F9BC8578482D15D1704A562318
:103B08001370002353702723937003231821012077
:103B18001371937107235171D070D371082111B0BB
:103B2800BDE83040FFF784BC432D88D100213C22FA
:103B380001A800910FF0A0FE6846FFF741FD644B15
:103B48002322802118460FF097FE9DF8002000F8E8
:103B58000C2C9DF8012000F80B2C9DF8022000F891
:103B68000A2C9DF8032000F8092C9DF8042000F881
:103B7800082C9DF8052000F8072C9DF8062000F871
:103B8800062C9DF8072000F8052C9DF8082000F861
:103B98000D5C00F8042C9DF80B509DF8092000F8E6
:103BA800032C9DF80A2000F8022C03A92A46A0F14C
:103BB8000D0400F8015C0FF098FE05F10D01224696
:103BC800C9B2012039E7807839280CD83038C0B21A
:103BD800FFF743FA3A4A2378137063785370A3784F
:103BE8009370032112E711B0BDE83040FFF76EBCB7
:103BF80080783928F7D83038C0B2FFF733FAE9E7C8
:103C080080783928EFD83038C0B2FFF731FAE1E7C9
:103C18008378303BDAB2092AE5D8C0783038C2B2A6
:103C2800092AE0D82179A1F14802D2B20B2ADAD8C0
:103C3800284D45FA02F2D507D5D40A224D2902FBB0
:103C4800030036D13C2358434FF47A735843224B30
:103C58001860224B1860FFF759FA194A2378137035
:103C680063785370A3789370E378D3700521237930
:103C780013710120FFF7DCFB144B00221A70272276
:103C88005A7001229A70DA70A278303A02EB8201F7
:103C9800E278303A02EB4102D2B21A7122795A71B3
:103CA8000F4A1278D2B21A72074A1278D2B25A72EE
:103CB8001CE74829C8D14FF46163C4E74B3B0108AE
:103CC800610D0020640E0020D80B00207100002038
:103CD8006E0D0020DEF7FFFF08000020B400002072
:103CE800E40D00208278303AD3B2092B3FF67BAF3F
:103CF800C378303BD9B209293FF675AF0079A0F1F6
:103D08004801C9B20B293FF66EAF624D45FA01F181
:103D1800C9073FF568AF0A214D2801FB02332DD1B1
:103D28003C2253434FF47A7253435B4A1360106842
:103D3800FFF704FA594A2378137063785370A3780D
:103D48009370E378D3700521237913710120FFF76D
:103D58006FFB534B00221A7027225A7001229A7067
:103D6800DA70A278303A02EB8201E278303A02EB5C
:103D78004102D2B29A712279DA7191E74828D1D1F9
:103D88004FF46162CDE7502B48D102297FF657AE38
:103D98004378303B012B3FF652AE8378312B7FF4CA
:103DA8004EAE0B2904D8FFF791FB00213B4A2DE6C4
:103DB8003B4D0234002214F8013FA918303B013270
:103DC800DBB20C2A0B73F6D1FFF774F9334B502290
:103DD80027211A709970002201215A70D97003F8AE
:103DE800041FA9180132097B0C2A01F1300103F8DC
:103DF800011FF6D100232B7027236B700123AB70B2
:103E0800EB70284B1B78DBB22B72274B1B78DBB28D
:103E18006B72EA72FFF768FB1121C7E7412B7FF449
:103E28000EAE4378432B7FF40AAE16297FF407AE13
:103E38001E4D421C002312F8011FE9540133142BB4
:103E4800F9D1FFF7BBF81A4B5B7D012B1DD1144943
:103E58000023EA5CC8180133D2B2142B80F82C2056
:103E6800F7D1114B00221A701B78DBB24B72FFF7A7
:103E78003BFB0A4A631E153413F8011F02F8011BA5
:103E8800A342F9D1054A1621C0E5074B02221A7050
:103E9800EFE700BFDEF7FFFFB4000020610D002050
:103EA80071000020E40D0020D80B0020E50D002053
:103EB800900A002037B504460D46002939D022481B
:103EC8000FF012FB2B78A3B39CB36068237880B300
:103ED800032B0DD0392B2ED0022B2AD16178012942
:103EE80027D00B0625D403B0BDE83040FFF744BD0A
:103EF8006378012B07D10078012802D0022800D06E
:103F080008B906F0F5FD00240DF107008DF807400B
:103F180006F034FE0D4A4C231370272393709DF846
:103F280007305470012041330521D0701371FFF719
:103F38007FFA03B030BD6378012BFAD10378044AC5
:103F480003F001031370F4E70C0C0020610D00204E
:103F58003C0C0020034B0022C3E902220122C3E9E2
:103F680000227047FC0D002000487047FC0D00201F
:103F78004FF0B04382B0DA6C0243DA64DB6C034082
:103F88000193019B02B070472DE9F04186B00024EF
:103F98000220154D0594FFF7EBFF0420FFF7E8FF1B
:103FA800124F03944FF4807601230DEB0001CDE905
:103FB80001632846032304934FF4005803F03AFDA5
:103FC80001A93846CDF8048003F034FD2246414665
:103FD800384603F055FE28462246314603F050FE87
:103FE800204606B0BDE8F0810004004800080048FB
:103FF800032810B50ED8012810D868B902460B4816
:104008004FF4807103F03CFE002209484FF4005140
:1040180003F036FE002010BD0122F0E7002203481D
:104028004FF4807103F02CFE0122EEE700040048F3
:1040380000080048022070470020704701207047A0
:10404800002814BF16200F20704700000D48854631
:1040580002F096FD0C480D490D4A002302E0D458A1
:10406800C4500433C4188C42F9D30A4A0A4C0023BA
:1040780001E013600432A242FBD30FF005FCFEF707
:10408800BFFAFEE70000012000000020BC08002065
:1040980054460108BC080020602C0020FEE74FF0C1
:1040A800B04382B0DA6C42F00102DA64DB6C03F0F0
:1040B80001030193019B02B07047000030B587B03F
:1040C800FFF7EDFF4FF4805101224FF0904003F0CD
:1040D800D7FD01224FF400614FF0904003F0D0FD6E
:1040E8004FF4C0551123CDE9015301A901234FF025
:1040F8009040039303F09EFC08240A2500224FF405
:1041080080514FF0904003F0BBFD0120FEF7E6FC24
:1041180001224FF480514FF0904003F0B1FD01208F
:10412800FEF7DCFC013DE9D14FF400614FF090400F
:1041380003F0A0FD08B9013CDFD14FF400614FF056
:10414800904003F097FD68BBFFF7A9FF0424012303
:10415800039001A92A48CDE9014303F06BFC284CE0
:1041680001220421204603F08BFD2120FEF7B6FC36
:1041780000220421204603F083FD2120FEF7AEFC37
:1041880001220421204603F07BFD2120FEF7A6FC36
:1041980020460022042103F073FD4FF42570FEF73A
:1041A8009DFCDDE7FFF77BFF4FF0B04300249A6DDD
:1041B80042F480029A659B6D03F4800300934FF4E8
:1041C800C052009B1223CDE901230323CDE9034309
:1041D80004230DEB03014FF09040059303F02AFCF4
:1041E80008480949094B8460C0E900130123C0E964
:1041F8000334C0E90744446103F0B6FE07B030BD9C
:10420800000400480C0E0020005800401A09102035
:10421800FFF754BF10B1012809D0704701394A424D
:104228004A414FF090404FF4007103F029BD4B1EF6
:104238005A4202485A412021F7E700BF00040048CB
:1042480008B50120FEF709FF6420FEF747FC00F0DF
:1042580021F9BDE808400120FEF704BF054B1A68A4
:1042680002805A689B684381034B028101221A70BD
:10427800704700BF640E0020E30D002010B504460F
:1042880000F008F810F0FF001CBFEE232370AA23EB
:10429800637010BD2DE9F7430024304E304D346073
:1042A80021462046FFF7B6FF21460120FFF7B2FF5F
:1042B80021460220FFF7AEFF5227A046012195F8BC
:1042C800640185F86071C5F86881FFF7A3FF0320D2
:1042D800FEF704FC00228821284602F0BFFB0DF1FE
:1042E8000602C021284602F009FC88BBBDF806205A
:1042F8004EF6AA639A422BD14FEA440909F15409B0
:104308005FFA89F94946284600F032F900BB85F87A
:1043180060910DF10602C021284602F0EFFBB8B902
:10432800284600F0E1FA98B9326801231A4432604D
:104338000C4AC5F868311168A3400B431360013477
:10434800032C05F5C875B9D1306803B0BDE8F08312
:104358000021E0B2FFF75EFFF1E700BF780E002012
:10436800B8000020740E00202DE9F74F344C0546A4
:1043780004F5966B4FF00A0A4FF00E0948F2E80868
:104388004FF490174FF48046D4F86831002B50D082
:10439800204600F099FD0DF102020DF101012046C1
:1043A80000F05AFB0DF1030201A9204600F08EFE31
:1043B8000021204600F0E0F801220021204600F00C
:1043C800A0F901221146204600F09BF9022D0ED8D3
:1043D8001C4B33F815601C4B53F825701B4B53F8D6
:1043E80025801B4B13F805901A4B13F805A032468D
:1043F8000121204600F0CEF93A460021204600F07F
:10440800C9F94146204600F0D1F84A460021204625
:1044180000F0CEF852460121204600F0C9F80DF10F
:1044280002020DF10101204600F016FB0123C4F839
:104438007C3104F5C874A345A6D103B0BDE8F08F5C
:10444800B8000020803B0108743B0108683B010864
:10445800633B0108603B010810B50B7E9BB9D0F89F
:104468007C21098912B1C0E95E1310BD084BD0F850
:1044780078411A68C2F580734B4304FB02331B1260
:10448800C0F87831F1E70123C0F87C31EDE700BFCF
:10449800680500202DE9F84FDFF8BCA02F4DFFF785
:1044A800B7FEDAF800300BB12B6813B9FFF7F2FE4C
:1044B80028602B682A4E0024A34234607460B460DC
:1044C80044DDDFF8A080284D0220FFF74DFF88F873
:1044D8000040D5F86831012B2ED1DFF890B003FAEF
:1044E80004F90A272149284600F04EFCB0B959467C
:1044F8002846FFF7B1FF9BF818307BB9D5F878311B
:1045080046F82430DAF8003043EA0903CAF80030E4
:1045180098F8003043F0010388F800300120FEF7D6
:10452800DDFA9BF818309BB1013F17F0FF07D9D18E
:104538004FF47A7346F8243001200134FEF7CEFA9E
:10454800032C05F5C875C4D198F80030BDE8F88F7C
:10455800D5F87831EEE700BF740E0020700E002009
:10456800640E0020E30D0020B80000207C0E00201F
:104578004A088A2102F072BA152906D8044BCB40A2
:10458800DB0702D50174002070476FF00700704701
:104598000B00300010B50A460C46092102F080FADB
:1045A80018B9237803F00103237010BD01F051BE40
:1045B80001F02EBD01F033BEF7B500230F461446B7
:1045C80001210DF1070206468DF8073002F068FA5E
:1045D8000546D0B9012C9DF8073025D1042F39D8CC
:1045E800DFE807F00316191C1F0043F010049C4273
:1045F8000BD022460121304602F030FA68BB7169BF
:1046080086F830413046FFF7D1FF284603B0F0BDA9
:1046180043F02804EBE743F00404E8E743F04004E0
:10462800E5E743F08004E2E7042F13D8DFE807F05A
:104638000306090C0F0003F0EF04D8E703F0D704D2
:10464800D5E703F0FB04D2E703F0BF04CFE703F09C
:104658007F04CCE76FF00305D7E70546D5E713B528
:1046680000230C460DF1070201218DF8073002F0F6
:1046780017FA78B99DF80730C3F300122270C3F314
:10468800C002A270C3F380026270C3F38012DB0918
:10469800E270237102B010BD37B50D460DF102026C
:1046A800F821044602F02AFA70B901AA042120462A
:1046B80002F042FA40B9BDF802201AB1019BB3FBDF
:1046C800F2F32B602B68A36103B030BD037F0B703E
:1046D8000020704737B50D460DF10602202104462B
:1046E80002F00CFA28B9BDF8063023B9236A2B600A
:1046F800207703B030BDDB002B60236201232377D2
:10470800F7E70529F8B504460E46154633D862B1D1
:1047180000EB810301215A6B0023701E042807D87F
:10472800DFE800F010191C1F260011460123F4E7EA
:1047380084F82810003D344418BF012584F8285017
:10474800002007E0C2F34F224421204602F096F9E8
:104758000028EFD0F8BD84F82A10EBE784F82B1076
:10476800E8E75B00FE226021204602F0B0F9EFE79F
:104778001B01EF22F7E76FF00300EBE7052996BF6F
:104788004018002390F82830137094BF00206FF071
:104798000300704770B54318044693F828300E4656
:1047A80015463BB105291BD8DFE801F003091214AF
:1047B8001616426304EB86040020656307E0C2F323
:1047C8004F224421204602F059F90028F2D070BD4A
:1047D800C263EFE70264EDE7C2F34F226421F1E719
:1047E8006FF00300F3E737B50446154605292AD8C4
:1047F800DFE801F0030614161818436B2B601FE05E
:104808000DF10602442102F079F9D0B9BDF806206D
:1048180053028AB12B60A36301230FE0C36BEDE75A
:10482800036CEBE70DF10602642102F067F940B969
:10483800BDF806305B02E1E7A26B2A6084F82930F4
:10484800002003B030BD6FF00300FAE737B50D461E
:104858000DF107020121044602F022F938B99DF84A
:10486800073084F83031DB092B7084F84C3003B002
:1048780030BD2DE9F843037C0C4601F8083B05469A
:10488800FFF70AFF40BB207304F110012846FFF729
:1048980021FF08BB04F11401284600F019FCD8B91F
:1048A80004F1240705F1270904F1170806463A46DA
:1048B800B1B22846FFF797FF70B9013619F8013FE2
:1048C80008F8013F062E07F10407F0D104F13C0176
:1048D8002846FFF7BBFF08B1BDE8F883211D28462D
:1048E800BDE8F84301F01DBDF0B50022054693B0C0
:1048F800882102F0B3F84FF47A72A5F852214FF4E8
:10490800C872A5F85421514AC5F858210023504AC5
:1049180085F8F030C5F8D4202B6202A92846FFF7A5
:10492800A8FF044670B9ADF8080002AE0FCE05F135
:1049380010070FC70FCE0FC70FCE0FC796E80F008F
:1049480087E80F00434BC5F834314FF4FA7301265A
:10495800A5F838314FF42063A5F83C313246802160
:1049680085F85061284602F079F832460746FF215B
:10497800284602F073F8002211460743284602F041
:104988006DF83C4364B204430DF1070291212846B7
:1049980002F086F864B29DF8073085F83A3104438E
:1049A80032460021284602F059F864B20443002236
:1049B800FF21284602F052F864B204430022802105
:1049C800284602F04BF864B2204340B200283BD09E
:1049D80013B0F0BD0028FBD1A1B201222846013452
:1049E800FFF78FFE062CF5D10028F1D10446688523
:1049F800024604212846FFF784FE0028E8D1024633
:104A080005212846FFF77DFE0028E1D14FF49013D9
:104A18006B634FF4804201212846FFF7BBFE002854
:104A2800D6D14FF40C13FF22C5E90F3085F8302199
:104A38000121284602F012F8012385F832310028B6
:104A4800C6D185F81541C3E70446C5E7856B010063
:104A5800A470090064008403012300F069BD2DE9F6
:104A6800F0428EB00C460C2304AA1421054601F02E
:104A7800DDFF8446002860D1BDF81620BDF8183047
:104A8800A075BDF81210206052BA5BBA6060BDF81C
:104A98001A60B5F8520192B29BB249BA5B0252024F
:104AA8002361A18276BAE260B0F57A7F8BB295F87D
:104AB80031719DF81010B6B20AD0704300F5FA7043
:104AC8004FF47A76B0FBF6F02E7F002E39D186B2FD
:104AD800002F40D0B001C0B2B608E0750DF10F004C
:104AE8002681CDE90040284601F072FE844620BBAD
:104AF8009DF80FE084F818E005F150060FCE07AFD7
:104B08000FC796E80700E37D87E80700D4E90301AB
:104B1800A28AADF83020D4E90149CDE90A01CDE9EE
:104B2800084907AC8DF833308DF834E00FCC503598
:104B38000FC597E8070086E8070060460EB0BDE895
:104B4800F0822E8C5E43B2EB262F4FEA262C04D13E
:104B580057B948F6E0260020BFE780B25043A2EBE1
:104B68000C06B0FBF6F0B2E742F2B826B2E7000056
:104B7800F7B517460E210DF106021D460B4C0646E9
:104B880001F0BCFFBDF8063004EA43433B6050B96E
:104B98000DF106020C21304601F0B0FFBDF80630D9
:104BA80004EA43442C6003B0F0BD00BF0000FE1FC0
:104BB80073B590F8DA30013B022B06460C4634D820
:104BC80001AB6A460121FFF7D3FF009BB3F57F0FC6
:104BD800054603D8019BB3F57F0F23D915BB34B124
:104BE8001349304602B0BDE8704001F0FFBB042213
:104BF800FF21304601F032FF2A4604467021304634
:104C080001F02CFF2A460443FF21304601F026FF1D
:104C180064B204432A468021304601F01FFF64B283
:104C2800044365B2284602B070BD0025FAE700BF0C
:104C38006C05002037B5044601228021057C01F06F
:104C48000DFF0122FF21204601F008FF0022114636
:104C5800204601F003FF94F83A219121204601F003
:104C6800FDFE01220021204601F0F8FE0022FF216E
:104C7800204601F0F3FE00228021204601F0EEFEDE
:104C8800012D24D0032D32D0C5BB01222946204650
:104C980001F0E4FE01238DF80730B0B905469DF810
:104CA8000730DB0705F101050AD548B9B5F5FA6FF4
:104CB80027D001460DF10702204601F0F1FEEEE78C
:104CC800B5F5FA6F08BF6FF0060003B030BD18B92C
:104CD80029462046FFF76CFF02220021204601F0FA
:104CE800BDFE0028F1D1042384F83231EDE718B96C
:104CF80001212046FFF75CFF0422EEE76FF0070072
:104D0800E3E76FF00600E0E738B5057C044625B117
:104D1800204600F03BFD28B138BDFFF78BFF002887
:104D2800F6D0F9E7002DF7D1032384F83231F3E701
:104D380073B50646002501220B21304601F08EFE90
:104D4800002204460B21304601F088FE0DF10702CF
:104D580004431321304601F0A3FE9DF8073064B2E6
:104D6800044301355B0760B2EDB205D0032D08D0CE
:104D78000028E0D002B070BD032D08BF6FF00B0013
:104D8800F8E76FF00B00F5E738B500230374044625
:104D98000D46FFF7B9FF50B929462046FFF75FFED9
:104DA80028B901462046BDE83840FFF7C1BF38BDE5
:104DB800152970B5054616461C4667D10122FF2104
:104DC80001F04CFE002211460446284601F046FE3A
:104DD80000220443FF21284601F040FE64B2044348
:104DE80001228021284601F039FE64B204430222E0
:104DF8008521284601F032FE64B204430422FF21D3
:104E0800284601F02BFE64B204430022CD21284637
:104E180001F024FE64B204431122CC21284601F09B
:104E28001DFE64B204430722FF21284601F016FE46
:104E380064B204430022BE21284601F00FFE64B28A
:104E480004430622FF21284601F008FE64B2044309
:104E58000922CC21284601F001FE64B20443002255
:104E6800FF21284601F0FAFD64B204430122FF2124
:104E7800284601F0F3FD64B2002204431146284697
:104E880001F0ECFD64B2204340B270BD042A17D88B
:104E98000A2101F0E3FD0028F7D1231E18BF0123E2
:104EA8001B01EF228421284601F011FE0028ECD1D5
:104EB80085F8DA6001462846BDE87040FFF738BF3C
:104EC8006FF00A00E1E7000070B594B00546402293
:104ED800002104A80EF0D0FC002301212846ADF8DB
:104EE80006308DF803308DF80430029300F0A0FCF2
:104EF80095F8142195F81311012A04D840F0AD80D3
:104F0800202940F2AC8001AA02A9284600F02BFB18
:104F18000446002840F09E8095F85031002B40F060
:104F2800A280D5F84C11284601F060FA0446002802
:104F380040F090800346014604222846FFF738FFD8
:104F48000446002840F086800122FF21284601F00F
:104F580085FD0DF1060206468421284601F0CEFDA6
:104F680022460643FF21284601F078FD76B2064323
:104F780074B2002C6ED1BDF806301B01C5F8D430D0
:104F880004A92846FFF775FC0446002862D10DF1F4
:104F980003012846FFF7FEFA044600285AD19DF877
:104FA800033085F8313104AC0FCC05F110060FC67B
:104FB8000FCC0FC60FCC0FC694E80F0086E80F0081
:104FC8000DF103020121284601F06AFD044600287C
:104FD80040D19DF8033085F8303102460146284615
:104FE800FFF7EAFA0446A8BB024602212846FFF763
:104FF800E3FA044670BB0323014685F832310DF10C
:105008000502284601F00BF9044618BB9DF8053047
:1050180085F8E8300DF105020121284601F0FFF876
:105028000446B8B99DF8053085F8E03003AA032195
:10503800284600F0E7FE044660B9039BC5F8E43053
:1050480003AA0421284600F0DDFE044610B9039B9C
:10505800C5F8DC30204614B070BD0C2951E728464D
:1050680000F013F954E701495DE700BF220700206B
:1050780013B50C460DF10702132101F011FD9DF83F
:10508800073013F0180F03F0070218BF6FF0050080
:10509800226002B010BD13B590F8DA30042B0C462C
:1050A80009D101A9FFF7E4FF019B1A1F534253419D
:1050B800237002B010BD01AA142101F0F1FC0028F0
:1050C800F7D19DF8043003F00103F1E700F04BBA83
:1050D80013B50C460DF10602282101F00FFD78B931
:1050E800BDF80620C2F30B0312F4006F18BFA3F536
:1050F80080534FF0FA0214BF13FB02F353432360AB
:1051080002B010BDF0B54FEAD20C4FF0FF341C606E
:1051180002F00702664600278E4200D207B1F0BDB2
:10512800845D664503BF1441E4B215463D4614F05C
:10513800010705D005EBC6051D6001270136EBE721
:105148000135082D4FEA5404F8D014F0010FF0E7A8
:10515800034B800953F82000003818BF012070471E
:105168001808002010B5B1EBD20F4FEAD20402F0B4
:10517800070381BF01229A40035D13438ABF035589
:105188006FF03100002010BD0A460623B02101F05F
:105198002FBC0A460623B02101F048BC2DE9F04F88
:1051A80085B00546109F0E9E01978A4693461C4679
:1051B8004FF00009119B994508D10023129A1760F6
:1051C80013B36FF0310005B0BDE8F08F01AB3A467C
:1051D80031465846FFF796FFDDF80480B8F1FF3FE7
:1051E8000FD00F9B08EB0300FFF7B2FF504508D123
:1051F80042462046FFF7B6FF08F1010709F1010909
:10520800D8E76FF03103D9E721462846FFF7BCFFFE
:105218000028D8D102A92846FFF7BBFF02ABA21984
:105228009442D0D014F8015B13F8011B8D42F7D0DB
:10523800C7E770B5C02288B00E46012190F83051FA
:10524800044601F00BFCF0B901A92046FFF79CFDCC
:10525800C8B90122FF21204601F000FC98B9324666
:10526800B621204601F04AFC68B90246FF212046D3
:1052780001F0F4FB38B92A460121204601F0EEFB83
:1052880008B984F8305108B070BDF0B50F4689B040
:105298001646FF210122044601F0E0FB0246A8B9A8
:1052A8004F21204601F0DAFB80B92C224E212046FE
:1052B80001F0D4FB024648B9FF21204601F0CEFB9D
:1052C80020B9B422B621204601F0C8FB0025C4F855
:1052D8002451A4F82851DEB9354607ABB422CDE9EC
:1052E80003730623CDE90032029504F5927304F5A1
:1052F800957231462046FFF751FF30B9012384F8F3
:10530800153184F8137184F8146109B0F0BD0135C2
:1053180005F1B400FFF71CFF0028DED12C2DF6D1D3
:10532800DBE710B541F001020021044601F096FBCD
:1053380078B9204600F02AFA58B901462046FFF706
:10534800F7FC30B9024601462046BDE8104001F09E
:1053580085BB10BD2DE9F74F4FF0000B8846174667
:10536800FF21012205461E469DF838A09DF83C9075
:105378008DF807B001F072FB5A4604465946284694
:1053880001F06CFB5A460443FF21284601F066FBF6
:1053980064B2044364B2B8F1000F32D0BAF1000F1E
:1053A80006D00C9ACB21284601F07AFB204344B260
:1053B800B9F1000F07D00DF10702EE21284601F0E0
:1053C8006FFB204344B20122FF21284601F046FB2F
:1053D800012204430021284601F040FB64B2044343
:1053E8000022FF21284601F039FB64B29DF80730FE
:1053F8000D9A204323F0100340B2137003B0BDE8A8
:10540800F08FBAF1000F06D03A46CB21284601F0BA
:1054180025FB204344B2B9F1000FD4D03346802293
:10542800EE21284601F053FBCBE72DE9F04387B086
:105438009146002205460E468DF817201F4653B3A5
:1054480090F8308101221146284601F007FB0446F6
:1054580048BB40212846FFF764FFF0B9B9F1010FB6
:1054680024D10DF11703CDE90294CDE9006322465A
:10547800234649462846FFF76DFF044678B947B1E9
:1054880042460121284601F0E9FA044638B985F870
:105498003081002403E09846D4E73470044620465F
:1054A80007B0BDE8F08300233370F8E73070E6E713
:1054B8002DE9F043054687B00E4691461F4653B383
:1054C80090F8308102220121284601F0C7FA0446EB
:1054D80048BB01462846FFF724FFF0B9B9F1010F90
:1054E80024D10DF11703CDE9024900932246234642
:1054F800019649462846FFF72DFF044678B947B17B
:1055080042460121284601F0A9FA044638B985F82F
:105518003081002403E09846D4E7347004462046DE
:1055280007B0BDE8F08300233370F8E73070E6E792
:10553800F8B51D46164600232A4690F830710446F1
:10554800FFF773FF70B903462A4631462046FFF736
:10555800AFFF38B93A460121204601F07FFA08B971
:1055680084F83071F8BD2DE9F04F002393B0CDE9F0
:105578000A12C0F82431A0F828310122FF21CDE910
:105588000E33B0F83C818DF8343004468DF8353050
:1055980001F064FA002840F0F08002464F212046CE
:1055A80001F05CFA002840F0E8802C224E212046C9
:1055B80001F054FA002840F0E0800246FF2120461E
:1055C80001F04CFA002840F0D880B422B6212046D9
:1055D80001F044FA002840F0D0800246802120469D
:1055E80001F03CFA002840F0C88003460DF135026E
:1055F8000DA92046FFF79CFF002840F0BE8004F567
:10560800957307930323CDE90203B421062304F518
:1056180092790EAECDE90031049601464B4604F569
:1056280095722046FFF7BAFD002840F0A6800DF1DC
:10563800360120460E9DFFF7FCFD002840F09D80B6
:10564800BDF83630434541D9C4F82401A4F82801EF
:1056580005F1B400FFF77CFD08B92B2D1FD90623EF
:10566800B42204960326CDE90032CDE90256079A02
:105678004B4601212046FFF791FD00287DD10DF111
:10568800360120460E9DFFF7D4FD002875D1BDF8E0
:105698003630434574D901274FF0010A19E0013526
:1056A800D6E7089E099324E0089E0A9B1E600B9B80
:1056B8001F70012384F815310A9B1B6884F8133185
:1056C8000B9B1B7884F81431002056E000273E46D7
:1056D800BA46BDF836304345E7D2A3EB080383EA60
:1056E800E372A2EBE3725FFA8AF70992032604F5E4
:1056F800927BDBF80000BBF804301090ADF8443022
:105708002A460FAB07980621FFF7FCFC0F9D6B1C80
:1057180039D005F1B400FFF71BFD5045C5D1731C06
:105728002A4648460893FFF71DFD30BB49462046E8
:105738000135FFF729FD00BB0DF136012046FFF7C3
:1057480078FDD0B9BDF83620A2EB0803002BB8BF0E
:105758005B424245A5D9099A9342A5D910A920468A
:10576800FFF712FDBDF8442003461098C4F8240141
:10577800ABF804201846002B97D013B0BDE8F08F83
:105788000746064688E76FF03100F6E737B500238D
:1057980004468DF807304FF4FA650DF107012046ED
:1057A800FFF779FC58B99DF80730012B07D0013D68
:1057B80003D0204601F0DEF9EFE76FF0060003B0F2
:1057C80030BD02464FF08043934202D8002013B9FF
:1057D80070479B08F8E7C11891424FEA50009CBFF8
:1057E800C018521A9B08F2E773B5002283210546B8
:1057F80001F034F9044690B906460DF107028321F9
:10580800284601F04DF99DF807300343DBB2044602
:105818002BB90136B6F5FA6FEFD16FF00604012205
:105828008321284601F01AF9204340B202B070BD26
:105838002DE9F04F90F8F06091B04FF00009072E75
:10584800CDE9079904460F4600F0A2820122802183
:1058580001F004F901228046FF21204601F0FEF8FC
:105868004A4648EA00084946204601F0F7F84FFA48
:1058780088F848EA00080622FF21204601F0EEF8E1
:105888004FFA88F848EA00080DF1150283212046EE
:1058980001F006F99DF815204FFA88F848EA000843
:1058A80042F004028321204601F0D8F84FFA88F824
:1058B80048EA00080722FF21204601F0CFF84FFAF6
:1058C80088F80122812148EA0008204601F0C6F83C
:1058D8004FFA88F848EA0008204601F04BF94FFAD9
:1058E80088F848EA000801228021204601F0B6F82D
:1058F8004FFA88F848EA000517F0010B6DB200F07E
:105908001E82F20700F11E826B229421204601F0CC
:10591800A5F880462046FFF767FF06AA48EA000870
:105928009021204601F008F945EA0805069B6DB26A
:105938002422942105432046C3F3062AC3F3C03921
:1059480001F08CF86DB205432046FFF74DFF6DB2AC
:10595800054306AA9021204601F0EEF8069B6DB299
:105968001BBA2522942105432046099301F076F8B5
:105978006DB205432046FFF737FF6DB2054306AA0F
:105988009021204601F0D8F8069B6DB21A0E054307
:105998001B0C6DB28DF828208DF8293017F0020302
:1059A800029300F0DB8016F0020840F0D780022254
:1059B8009421204601F052F801902046FFF714FF89
:1059C800019B0DF116020343902120461D4301F06F
:1059D80067F86DB27B2294210543204601F03EF81A
:1059E8006DB205432046FFF7FFFE6DB205430DF18A
:1059F80017029021204601F053F86DB277229421C6
:105A08000543204601F02AF86DB205432046FFF70A
:105A1800EBFE6DB2054306AA9021204601F08CF8F2
:105A2800069B5A0E8DF82C20C3F386428DF82D2044
:105A3800C3F3C6228DF82E206DB2C3F30612DB0025
:105A480003F07803942105438DF82F20204678220F
:105A58008DF8153001F002F86DB205432046FFF7C6
:105A6800C3FE6DB2054306AA9021204601F064F8F2
:105A7800069B9DF8152002EB53728DF83020C3F376
:105A880086528DF83120C3F3C6328DF83220C3F325
:105A980006228DF833206DB2C3F346029B0103F052
:105AA8004003942105438DF83420204679228DF84F
:105AB800153000F0D3FF6DB205432046FFF794FE82
:105AC8006DB2054306AA9021204601F035F8069BE1
:105AD8009DF8152002EB93628DF83520C3F3C6427A
:105AE8008DF83620C3F306328DF837206DB2C3F334
:105AF80046129B0003F07C03942105438DF838205F
:105B080020467A228DF8153000F0A8FF6DB20543C3
:105B18002046FFF769FE6DB2054306AA902120468C
:105B280001F00AF8069B9DF815208DF83E8002EBDF
:105B380093728DF83920C3F3C6526DB28DF83A20AE
:105B4800C3F3064205438DF83B20C3F34622C3F353
:105B580086036DB28DF83C208DF83D3017F00403B4
:105B6800019300F0F180730700F1EE807B2294210D
:105B7800204600F073FF80462046FFF735FE07AA4F
:105B880048EA00089021204600F0D6FF45EA0808B8
:105B98004FFA88F848EA00057C229421204600F054
:105BA8005DFF6DB205432046FFF71EFE6DB205434B
:105BB80008AA9021204600F0BFFF6DB273229421FD
:105BC8000543204600F04AFF6DB205432046FFF723
:105BD8000BFE6DB2054306AA9021204600F0ACFFEB
:105BE800069B6DB21B0274229421054320461FFABE
:105BF80083F800F033FF6DB205432046FFF7F4FD4C
:105C08006DB2054306AA9021204600F095FF6DB2BB
:105C18009DF81B30752294210543204643EA080865
:105C280000F01CFF6DB205432046FFF7DDFD6DB2A5
:105C3800054306AA9021204600F07EFF069B6DB220
:105C48001B029BB27622942105432046039300F061
:105C580005FF6DB205432046FFF7C6FD6DB205434B
:105C680006AA9021204600F067FF6DB29DF81B2020
:105C7800039B05436DB21343002281212046039301
:105C880000F0ECFE06220543FF21204600F0E6FE68
:105C98006DB205430DF115028321204600F000FF87
:105CA8009DF815206DB2054302F0FB0283212046C2
:105CB80000F0D4FE6DB205430122FF21204600F01A
:105CC800CDFE6DB2054301220021204600F0C6FE3C
:105CD8006DB205430022FF21204600F0BFFE6DB2E1
:105CE800054300228021204600F0B8FE6DB205432E
:105CF8006DB2039BFDB9BBF1000F29D1029AAABB73
:105D0800019AAAB1720713D4079AC4F81821089AFD
:105D1800C4F81C214FEA4822C4F820213BB1A3F55E
:105D2800C8534FF47A7253431B095B421BB2E360BA
:105D38003E4384F8F060284611B0BDE8F08FD9469C
:105D4800DA462BE6CA4629E64FF00008434693E7B1
:105D5800F007D3D40998BDF8282084F813A184F853
:105D68001491C4F82A01A4F82E21C7E7B107C7D4B3
:105D78009DF8162084F8F1209DF8172084F8F22069
:105D88000BA904F1F30002930DF0A2FD029BB7E703
:105D98004D46D0E740B101380023FF2803F1010246
:105DA80003D800EB032080B2704740081346F4E79D
:105DB800C3B2000A03FA00F001307047084B5A4397
:105DC8004FF47A7302F5FA724FF4FA60B2FBF0F00E
:105DD800B2FBF3F203FB0100B0FBF2F0704700BF27
:105DE800002F3A00064B5A434FF47A7002F5FA72C4
:105DF800B2FBF0F24A4302F5FA72B2FBF0F07047D8
:105E0800002F3A002DE9FF4102294FF0000507460F
:105E180016468DF80350ADF804501CD80DF1020257
:105E28002946FEF7C7FB044630B90DF103024621A7
:105E3800384600F035FE04469DF80300FFF7B8FF2A
:105E480081B29DF802203846FFF7CCFF306020462B
:105E580004B0BDE8F081032918D10DF102022946EA
:105E6800FEF7A8FB0446002846D101460DF10202C0
:105E78003846FEF79FFB044628B901AA5121384647
:105E880000F03CFE0446BDF80400D7E7042935D1EC
:105E980002A9FEF7E4FB9DF80B304BB30DF10202AB
:105EA80029463846FEF786FB044618BB01AA51214D
:105EB800384600F023FE0446BDF80400FFF778FFDB
:105EC80085B2BCB90DF1020201213846FEF772FB1A
:105ED800044678B90DF106027121384600F00EFE2D
:105EE8000446BDF80600FFF763FF80B2401BA7E732
:105EF8001D46E7E70020F9E72846A7E728462C468D
:105F0800A4E7F0B5022985B0054616461ED80DF15E
:105F180005020021FEF74EFB0446A0B99DF80520B6
:105F280031462846FFF74AFF83B2B3F5807F9ABF10
:105F380000F1FF32D2B2FF22A5F8D8204621284628
:105F480000F08CFD0446204605B0F0BD032920D1A1
:105F58000DF105020021FEF72DFB9DF805200446F2
:105F680031462846FFF72AFF80B2FFF713FF0246A3
:105F7800ADF80600A5F8D800002CE4D15121284638
:105F880000F07CFD04460028DDD1C5F8E46000245B
:105F9800D9E7042939D102A9FEF761FB9DF80B70F6
:105FA800B7B10DF1050200212846FEF703FB0446B0
:105FB8000028C8D10DF106025121284600F09EFDA7
:105FC80004460028BFD1BDF80600FFF7F1FE87B2EE
:105FD8000DF1050201212846FEF7ECFA04460028D7
:105FE800B1D19DF8052031462846FFF7E7FE384431
:105FF800FFF7D0FE71210246284600F03FFD044617
:106008000028A0D1C5F8DC60C1E76FF003049AE767
:10601800F0B585B000238DF80330D30705460F4649
:10602800164605D441B9A2F10C03DAB2062A12D9F0
:106038006FF0030005B0F0BD012920D1A2F10803DB
:10604800DAB2062AF4D8062B19D8DFE803F0371895
:10605800651886189900062B11D8DFE803F004109C
:1060680029102B102D0018225721284600F0F6FC85
:1060780008225621284600F0F1FC0028DAD17408DD
:10608800013CE4B2002F00F08E80012FD0D101AA8C
:1060980004212846FFF7B6FE38B922467021284663
:1060A80000F0DCFC002800F0B28085F8E060C1E771
:1060B8003022D9E74022D7E75022D5E710224821DD
:1060C80000F0CCFC08224721284600F0C7FC022239
:1060D80004463221284600F0C1FC0C22044330213A
:1060E800284600F0BBFC64B204430122FF21284685
:1060F80000F0B4FC64B2044364B230223021284674
:1061080000F0ACFC00220443FF21284600F0A6FC66
:1061180064B2204340B2B0E72822482100F09EFC38
:1061280008224721284600F099FC03220446322120
:10613800284600F093FC044364B209223021284623
:1061480000F08CFC01220443FF21284600F086FC65
:1061580064B2044364B22022D0E73822482100F018
:106168007DFC08224721284600F078FC03220446DB
:106178003221284600F072FC044364B20822DDE7AD
:106188004822114600F06AFC08224721284600F000
:1061980065FC032204463221284600F05FFC0443D4
:1061A80064B20722CAE702AA03212846FFF72AFE9B
:1061B80088B903AA02212846FFF724FE58B92246C7
:1061C8005021284600F04AFC28B9029A03212846A3
:1061D800FFF797FE10B185F8E8602BE7039A0221D4
:1061E8002846FFF78EFE85F8E86000287FF422AF86
:1061F80069692846FEF7DAF900287FF41BAF0246E2
:1062080001230DF103012846FFF752F912E7019A1D
:1062180004212846FFF775FE85F8E060E5E713B529
:10622800144629B1012910D06FF0030002B010BD47
:106238000DF10702502100F033FC0028F6D19DF83B
:10624800073001335B002370F0E70DF1070270217E
:10625800F1E7F0B5002385B04FF4FA62CDE90023E9
:1062680044F61F63994206460F4604D86FF00305AB
:10627800284605B0F0BD02A9FEF7F1F90546002849
:10628800F6D19DF809209DF8083013439DF80A209F
:106298001343A7F636341BD06A4602213046FFF76F
:1062A800B1FD00283BD19DF808302BB1009B03F2CB
:1062B8004E239C42DAD9E41A9DF80A3023B3009B96
:1062C80003F2B223B4EB430F4FEA4302CED9A41A28
:1062D8009DF80B305BB101AA03213046FFF792FD10
:1062E800019B03F525739C42C0D9C0B9E41A9DF8F7
:1062F8000C30002BBCD0A4F2262204213046FFF734
:1063080000FE77610546B3E79DF80930002BDFD022
:10631800009B03F525739C42A8D9E41AD8E70546E3
:10632800A6E770B54FF4FA6286B00023CDE90223E0
:1063380040F636330B600C4604A90646FEF78FF983
:106348000546002836D19DF811209DF810301343DA
:106358009DF81220134319D002AA02213046FFF7F4
:1063680051FD002840D19DF810302BB1029B03F25B
:106378004E222368134423609DF81230EBB1029B30
:1063880003F2B222236803EB420323609DF8133023
:10639800EBB99DF814305BB101AA04213046FFF730
:1063A80031FD019B03F22622236813442360D8B9E8
:1063B80023687361284606B070BD9DF81130002B24
:1063C800E4D0029B03F5257223681344DDE703AA92
:1063D80003213046FFF716FD039B03F5257223685A
:1063E800134423600028D4D00546E3E72DE9F7439A
:1063F800002406460D46204615F80480B8F1000F23
:1064080000D010B103B0BDE8F083671CB8F1FF0FEE
:1064180015F8079029D1A71CEB5DB9F1030F36D801
:10642800DFE809F0020B131B271D2C44E27802EB6E
:106438000323A6F834313C46DEE7271D2C44E278D6
:1064480002EB0323A6F83631F5E7271D2C44E27842
:1064580002EB0323A6F83831EDE7271D2C44E27838
:1064680002EB0323A6F83C31E5E7B8F1040F0ED898
:1064780002344246291901A80DF037FA434601AA09
:106488004946304604EB080700F0B2FAD3E76FF04C
:106498000300D0E773B500230E4613600DF1070122
:1064A80005461446FEF712F940B99DF807302BB19E
:1064B800B38A2A6A534380331B0A236002B070BD33
:1064C80013B5CB681360144601AAFFF7E3FF18B9A8
:1064D8002368019A1344236002B010BDF8B5B0F8E0
:1064E8005451D0F8580168438030000A0E4645439D
:1064F800DDE90717144652B1B60206EB5202B2FBA9
:10650800F4F202EB4202524302F50042140C069ADE
:10651800534301F50042120C06200332B2FBF0F29D
:10652800C2EBC202B2F5803F38BF033103F5004326
:106538003EBFB1FBF0F1C1EBC10101F500414FEAEB
:10654800134334BF090C1B4903FB03F338BF49430A
:1065580003EB57030B44B3FBF7F39B03FE2205F150
:1065680020007F33B3FBF2F35C434FF47A7704F5F2
:10657800FA748009B4FBF7F42401FFF722F904F553
:10658800FA74BC4228BF4FF4FA63064629BFB4FB2D
:10659800F3F300205B19B4FBF7F428BFB3FBF4F066
:1065A800FFF70FF9099B864294BF1E601860002010
:1065B800F8BD00BF0000F0FF2DE9F04F91B005468F
:1065C80007930B6908930F46CB680B9393460FAA62
:1065D800FFF776FF0EAA39462846FFF75BFF48BB50
:1065E8000F9C95F8E0A0D5F8DC3005934FF47A7647
:1065F80006FB04F101F50041049180340E990991DC
:1066080024F0FF010A910F910499D5F8E43006931C
:10661800BAF1080F0CBF02230323090C95F8E820F0
:10662800DFF898810C9108D1079BCBF80080C5F85A
:106638004081186011B0BDE8F08F06990D93284687
:10664800FFF7BCFB5246059981462846FFF7B6FB83
:106658000D9B5B490C9A814403FB09F94FEAC92950
:1066680040F2776309F5FA79240AB9FBF6F903FBD6
:1066780009F909F5FA79B9FBF6F909FB04F404F10B
:106688008003089C74430C40B4FBF2F44D4A1B0A87
:10669800944228BF1446012B38BF01230C204FF425
:1066A800167258435443FFF78CF83B7E3A894FEAF9
:1066B800400A002B7FD14249049B0B4003F5FA7135
:1066C800414B5A4341F25C23B2FBF3F2099B7343FB
:1066D800B3F5481F28BF4FF44813A1EB4303B1FBA0
:1066E800F6F1B3FBF6F31B02B3FBF1F63602C6F57F
:1066F8008036564306F50046360C06F58036760891
:106708007643B60B4FF44873734303F5004304F51F
:1067180000401B0C5B43000C00FB0030FFF751F8F6
:1067280003046422323341F28837B3FBF2F340F6B4
:10673800B532B3FBFAF302FB0377244B9F429CBFAD
:1067480042F21073B7FBF3F7DDE90532134403F5A2
:10675800FA734FF47A7A4FF4FA62B3FBFAF0B3FBA8
:10676800F2F202F5C812B2FBF0F088BF4FF470479E
:10677800FFF727F8000200F5FA70B0FBFAF0404383
:1067880007FB0700FFF71DF80AFB00F0079B4045D1
:1067980028BF4046CBF80000C5F84001CDE9029378
:1067A8004FF448730093DDE90A12019433462846F2
:1067B800FFF794FE3EE74FF48036A3E7AE878F02DB
:1067C8000000FFFF666666009A9906000F279F245F
:1067D8002DE9F04F11F0780F8BB018BF4FF2A009D8
:1067E800C1F3C30B18BF29FA0BF990469A460DF16D
:1067F8000E024FF000034FF00001159F8DF80E3088
:1068080004468DF80F308DF810308DF81130ADF842
:106818001230099314BF09F001094FF00109FDF77F
:10682800ADFF9DF80E500646D5B1002840F09A807D
:10683800149909AB05AA2046FFF7BEFE002840F0D0
:106848009380149A099B5381014606AA2046FDF7B6
:10685800CAFF069D25B1059B9D422CBF0025012539
:1068680020B904AA02212046FDF788FF9DF8106090
:1068780026B300287AD107AA02212046FDF7B3FFE4
:1068880088B90122FF21204600F0E8F858B90DF137
:106898001202B621204600F031F920B90246FF2144
:1068A800204600F0DBF8BDF81230079E5B02C4F802
:1068B80048311EB19E422CBF0026012628B90DF191
:1068C800110203212046FDF759FF9DF8113093B1BD
:1068D80000286CD1BAF1000F03D04FEA0828B8FBA2
:1068E800FAFA08AA03212046FDF77DFF089B5345C5
:1068F80094BF0023012320B9B9F1000F38D0FF223B
:106908003A703A780AB914994A810DF10F020121B7
:1069180020460193FDF732FF08BB9DF80E20019B2E
:10692800002A08BF0125BBF1040F18BF9DF80F20EE
:1069380084F82E501ABFB2FA82F25209012284F862
:106948002F209DF81020002A9DF8112008BF01264D
:10695800002A08BF012384F8306084F831300BB076
:10696800BDE8F08F002581E735467FE70026ACE7D4
:106978000BF1FF32092A0AD8DFE802F005050509FC
:106988000907090B070B0522BAE70422B8E7012E0D
:1069980001D10322B4E7BBF1040F01D0012B01D1CF
:1069A8000222ADE7012D16BF00233D703B70002386
:1069B800A7E707B502F10A03009393B20A4690F8D5
:1069C8006011D0F85C0101F021FB03B05DF804FB15
:1069D80013B502F10A0390F860410093D0F85C0106
:1069E80093B20A4644F0010101F0A6FB02B010BDC3
:1069F8003F2BF8B50E46054611461C4611D80A4FDE
:106A080038461A4600F8016B0CF06FFF621C3946D5
:106A18002846FFF7CEFF002814BF6FF013000020B0
:106A2800F8BD6FF00300FBE7980E002073B515461C
:106A38008DF8071001220DF1070104461E46FFF7E5
:106A4800B8FF18B16FF0130002B070BD3246294686
:106A58002046FFF7BDFF0028F6D0F3E708B5064B40
:106A680019705A7019460222FFF7A3FF002814BFB5
:106A78006FF01300002008BD980E002008B5074BE2
:106A88001970110A59709A7019460322FFF791FF7D
:106A9800002814BF6FF01300002008BD980E0020D6
:106AA80037B515468DF8071001220DF10701044688
:106AB800FFF77FFF18B16FF0130003B030BD01225C
:106AC80029462046FFF784FF0028F6D0F3E7F7B5FC
:106AD80015460DF1070206460F461C46FFF7E0FF74
:106AE80050B99DF807301D4044EA05023946304642
:106AF8008DF80720FFF7B2FF03B0F0BD73B5144659
:106B08008DF8071001220DF107010546FFF751FF27
:106B180018B16FF0130002B070BD064E0222314664
:106B28002846FFF755FF0028F3D133885BBA238046
:106B3800F1E700BF980E002073B514468DF80710D2
:106B480001220DF107010546FFF733FF18B16FF079
:106B5800130002B070BD064E042231462846FFF7E6
:106B680037FF0028F3D133681BBA2360F1E700BF71
:106B7800980E002008B50220FBF7B0FF002008BDE2
:106B88007047000010B5032000F056FC01F032FDFC
:106B9800064B18600F20FBF797FF044618B9FBF760
:106BA8001EFE204610BD0124FBE700BF2808002078
:106BB8004FF0E022136923F00203136170474FF08E
:106BC800E022136943F0020313617047014BD3F8C5
:106BD800900570470070FF1F014BD3F8940570476C
:106BE8000070FF1F014BD3F8980570470070FF1F16
:106BF8008068C0F380007047F7B50023019304460E
:106C0800002800F0E980856D25B9FBF721F9E565D5
:106C180084F8545023689A68D00040F1A1809A689B
:106C2800D10000F1B480A26D42F01002A265E26DBD
:106C380042F00102E26501251846FFF7D9FFA26D6F
:106C480002F01002024340F0C980A26D206922F4CC
:106C5800817242F00202A2659A68D2075DD4226B63
:106C6800A67E94F82CC0003A18BF01221703D4E975
:106C780002120A43217E42EA8132617E42EAC1322F
:106C880042EA4632002842EA4C02B4BF20F00041F2
:106C98004FF400113A430A4394F82010012903D114
:106CA800002E76D142F48032616A21B1A66A01F4DD
:106CB800E07131430A43D968E66C21F4FE3121F4CE
:106CC800FF711143D96094F83C206168012A01F0F2
:106CD800404C4CEA060609D1D4E910273A4332431E
:106CE800A66C324342EA0C0242F001061F693E4A92
:106CF8003A4032431A6121F00042B2F1804F0CD081
:106D0800B1F1004F09D0394ED6F8082701F47011B7
:106D180022F470120A43C6F808275A69666BA16BF9
:106D280022F0070232435A615A6922F0700242EA9D
:106D380001125A61002835D19A6A62F00F029A62EC
:106D48005B6903F007039E423CD10023E365A36D12
:106D580023F0030343F00103A365284603B0F0BD05
:106D68009A68234922F0104222F0170242F080521A
:106D78009A60204A1268B2FBF1F201325200019285
:106D8800019A002A3FF44BAF019A013AF7E7002530
:106D980052E7A16D41F02001A165E16D41F00101CB
:106DA800E16581E7B0F5001FCAD19A6AE269013A44
:106DB80092006FF00F0102F01C0201FA02F2216E3C
:106DC8000A43BCE7A36D23F0120343F01003A36545
:106DD800E36D43F00103E3650125BEE7A36D43F0CE
:106DE8001003A365F8E700BF02FCFF1F0020014065
:106DF800400D030028080020F8B54569082D044611
:106E08000E460AD00368DB68D80705D5A36D43F0A2
:106E18002003A3650120F8BD0425FBF757FE0746AC
:106E280023681A682A4220D0A26D42F40072A26533
:106E3800DA6812F4406F14D1A27E92B91A68120768
:106E48000FD51846FFF7D4FE20BB5A6822F00C0273
:106E58005A60A26D22F4807222F0010242F001020F
:106E6800A265227EFAB10020D5E7711CD9D0FBF7C4
:106E78002DFEC01BB04201D8002ED1D123681B685B
:106E88002B40CDD1A26D84F8543042F00402A265A3
:106E98000320C0E7A26D42F02002A265E26D42F035
:106EA8000102E265DDE70C221A60DCE70368186C72
:106EB80070470000F7B50023019390F85430012B78
:106EC800044600F0C08005680269012380F8543048
:106ED8002846FFF78DFE002840F0AF80D1E900304A
:106EE800022822F004027ED0B2F1004FC3F3110E43
:106EF80035D1AA6A42EA0E02AA628A68686902EA79
:106F0800032222F07C4222F0FF0220EA03210A43F6
:106F1800002B6A611DDA4D4A4D4DD2F80817AB4275
:106F280001F0E07043D10D0213D4D2F8083723F0F2
:106F3800E073034343F40003C2F80837454B1A686B
:106F4800454BB2FBF3F20C2302FB03330193019B85
:106F580053BB0020002384F8543003B0F0BD226EE8
:106F680000F01F074FF00F0C0CFA07FC6FEA0C0635
:106F780022EA0C0CBEF1000F11D1C3F38462BA40AF
:106F880042EA0C0222668008E26901309042B4D8D5
:106F9800A86AC3F38362BA4006403243ACE793FA67
:106FA800A3F2B2FA82F2EAE7019B013BCEE72B4D4E
:106FB800AB420BD1C901CCD4D2F8083723F0E07327
:106FC800034343F08073C2F80837C2E7244DAB424D
:106FD800BFD14B02BDD4D2F8083723F0E073034386
:106FE80043F48003EFE7B2F1004F01BFAA6AC3F38D
:106FF80011018A43AA62002BABDA15481349834270
:10700800D1F8082709D1D1F8083702F0A07223F087
:10701800E0731A43C1F808279BE71048834204D15C
:10702800D1F8083702F44002F1E70D48834290D1C5
:10703800D1F8083702F0C072E9E7A26D42F02002E9
:10704800A265184686E7022087E700BF00200140B6
:10705800001000B028080020400D0300004000B8D0
:10706800002000B4026838B504461046FFF7C0FD9A
:1070780008B9002038BD9368990707D4936823F0AE
:10708800004323F0170343F010039360FBF71EFD42
:10709800054623689B685B07EBD5FBF717FD401B8C
:1070A8000228F6D923689B685A07F2D5A36D43F0E6
:1070B8001003A365E36D43F00103E3650120D9E7FD
:1070C80073B50023026801939368DD07044602D56F
:1070D800002002B070BD9168214B194209D0A36D00
:1070E80043F01003A365E36D43F00103E36501205A
:1070F800EFE7936823F0004323F0170343F00103FD
:107108009360184BD3F8083718021CD4637E012B00
:10711800DED0FBF7DBFC144E054622681368DB075C
:10712800D6D49368D9075FBF9368334043F001030F
:107138009360FBF7CBFC401B0228EED923681B6841
:10714800DA07EAD4CBE7094B094A1B68B3FBF2F329
:1071580001330193019B002BD8D0019B013BF8E739
:107168001700008000200140E8FFFF7F280800206A
:10717800400D030038B504460068FFF739FD0546A1
:1071880020BB94F85430012B20D0012384F85430CC
:107198002046FFF795FFB0B9A36D226823F470630A
:1071A80023F0010343F48073A3651C23E065136097
:1071B80084F85400936823F0004323F0170343F046
:1071C8000403936038BD84F85450FBE70220F9E7C4
:1071D800026838B5936891680446C80701D400204E
:1071E80038BD9907FBD4936803F00503012B19D127
:1071F800936823F0004323F0170343F002039360DE
:1072080003231360FBF762FC054623689B68DB07D2
:10721800E5D5FBF75BFC401B0228F6D923689B6881
:10722800DA07F2D5A36D43F01003A365E36D43F0CD
:107238000103E3650120D3E770B5044600284BD06D
:10724800836D43F002038365FFF70CFF054668B9B9
:107258002046FFF7BDFF054608B90123A36522684C
:10726800936823F0104323F01703936023685A6848
:1072780022F4677222F003025A6040F29F321A60C9
:10728800D968164A0A40DA601A6922F040421A613F
:107298005A6922F007025A611A6A02F0F0221A6249
:1072A8005A6A02F0F0225A62DA6A02F0F022DA62CE
:1072B8009A6A0B4A00269E62D2F8083723F0FE73BA
:1072C800C2F808372046FAF7D7FDE6652666A665B0
:1072D80084F85460284670BD0125FBE700023E8310
:1072E8000020014010B590F85430012B044615D009
:1072F800012380F85430FFF7B5FE58B92046FFF750
:1073080067FF38B9A36D23F4807323F0010343F0BA
:107318000103A365002384F8543010BD0220FCE764
:10732800F7B50023019390F85430012B04467FD021
:10733800012380F85430FFF74BFF23689A6812F056
:107348000102054607D0A36D43F01003A36500238F
:1073580084F854302DE0A16D364F21F4817141F04D
:107368000201A165DE68D96826F4FF4626F07C068E
:1073780021F40041360421F00301360CD9600820BD
:107388009968394041F0004199609968002913DAF9
:107398000199013101910199B1F52E3FF5D3A36D02
:1073A80023F0120343F01003A365002384F854303C
:1073B8000125284603B0F0BDD3F8B410013801F018
:1073C8007F010A44DCD199681A48014041F0010163
:1073D8009960D3F8B41021F07F0141EAD202C3F8D2
:1073E800B4209A68024042F002029A60FBF76EFBF2
:1073F800074623689A68D20708D4DA683243DA6005
:10740800A36D23F0030343F001039FE7FBF75EFB43
:10741800C01B0228EDD923689B68D907E9D5A36D5D
:1074280043F01003A365E36D43F00103E365BFE791
:107438000225BEE7E8FFFF7F0749CA6822F4E06239
:107448000302120403F4E063120C134343F0BF6316
:1074580043F40033CB60704700ED00E0164B30B5C5
:10746800DC68C4F30224C4F10703251D042B28BFDC
:107478000423062D4FF0FF358CBF033C002405FA8A
:1074880003F321EA0303A54022EA0502A3400028EA
:1074980043EA0203ACBF00F16040084A4FEA031315
:1074A800B8BF00F00F00DBB2AABF00F5614013546B
:1074B80080F8003330BD00BF00ED00E014ED00E0BF
:1074C800002807DB044A4109012300F01F0083401C
:1074D80042F82130704700BF00E100E000280CDBD3
:1074E8004309064900F01F0020330122824041F879
:1074F8002320BFF34F8FBFF36F8F704700E100E089
:1075080070B5D0E913456560446D14B1D0E91645EE
:107518006560D0E9105404F01C060124B4406C6086
:10752800046863608368102B0BBFA260A160E160F0
:10753800E26070BD0268416CD3B210B5083B1424F8
:10754800B3FBF4F30B4CA24288BF0B4A21F00301B2
:1075580099BF01F1804202F5023252180733826462
:10756800064AC26403F01F03012202FA03F303650B
:1075780010BD00BF070402401C08024080080240FA
:1075880038B500285CD002682E4B9A424FF014019F
:107598004AD82D4B1344B3FBF1F32C499B00C0E9A7
:1075A8001013022380F825301368056923F4FF437C
:1075B80023F070031360D0E9024323432B4345694A
:1075C80011682B4385692B43C5692B43056A2B43F7
:1075D8000B431360FFF7AEFFB4F5804F04BF0023E1
:1075E80043604368816C03F07F020A60D0E913149A
:1075F800013B032B4C601ED8154B1649816513447B
:107608009B000121013A01FA02F200214365C2659B
:107618001960114B5A6400230122C36380F8243097
:1076280080F82520184638BD0C4B1344B3FBF1F302
:107638000B499B00B3E70023C0E91533C365EAE7AC
:107648000120F0E707040240F8FFFDBF00000240F8
:107658003F8200104009024000090240F8FBFDBFCC
:107668000004024038B5002841D00268136823F0AE
:10767800010313601F4B9A424FF0140130D81E4B80
:107688001344B3FBF1F31D499B00C0E91013012417
:1076980003F01C0304FA03F3002515604B60FFF7A1
:1076A80049FF836C41681D60D0E913325A604A1E55
:1076B800032A06D8124B0B449B0094401D60114BC3
:1076C8005C640023C363C0E91533C0E90B33C0E928
:1076D8000D33C36580F8253080F82430184638BD4E
:1076E800094B1344B3FBF1F308499B00CDE7012094
:1076F800F5E700BF07040240F8FFFDBF00000240A5
:107708003F82001000090240F8FBFDBF0004024060
:1077180070B590F82450012D04463BD090F82560B0
:107728000125AE4280F824504FF000062CD10225E6
:1077380080F825500568C6632E6826F001062E607D
:10774800FFF7DEFE036BBBB12B6843F00E032B6023
:10775800A36C1A68D20342BF1A6842F480721A6096
:10776800636D1BB11A6842F480721A602B6843F08B
:1077780001032B60002070BD2B6823F004032B60ED
:107788002B6843F00A03E2E78023C36380F8246090
:107798002846F0E70220EEE770B4426C046C0368F8
:1077A80026681D6802F01C020421914031420FD066
:1077B80015F0040F0CD01A6892065EBF1A6822F002
:1077C80004021A60036B6160002B33D070BC184749
:1077D80002219140314217D015F0020F14D01A68D7
:1077E800940606D41A6822F00A021A60012280F868
:1077F8002520114A93428CBF104B114B596000232E
:1078080080F82430C36ADFE708219140314211D063
:1078180029070FD5196821F00E011960012303FA11
:1078280002F26260C36380F82530002380F82430B8
:10783800436BC9E770BC70478000024000040240F7
:10784800000002400A4A536943F4802330B553616B
:10785800EFF3108472B60023CD58C5500433B3F546
:10786800807FF9D11369DB03FCD484F3108830BD21
:1078780000400058064B5A69002ABFBF054A9A6063
:1078880002F188329A60BABF5869C00F0020704769
:107898000040005823016745044B5A6942F00042F2
:1078A8005A615869C043C00F704700BF0040005874
:1078B80070B50546FBF70AF9124E04463369D90339
:1078C80013D43369DA0744BF012232614CF2FA3229
:1078D800134011D10B4E306910F480200BD0FBF708
:1078E800F5F8001BA842F6D304E0FBF7EFF8001BFD
:1078F800A842E3D3032070BD024A1361024A012063
:107908005360F8E700400058D80E00202DE9F041F8
:10791800184D98462B78012B06460C46174626D05C
:1079280001232B704FF47A7000236B60FFF7C0FFC0
:10793800A0B9012E16D1104A536943F001035361CF
:107948002760BFF36F8FC4F804804FF47A70FFF795
:10795800AFFF094A536923EA0603536100232B70DA
:10796800BDE8F08139462046FFF76CFFEDE70220BD
:10797800F6E700BFD80E002000400058054A5369BA
:1079880023F47E7343EAC00040F4803040F00200E4
:1079980050617047004000582DE9F041234F3B7873
:1079A800012B054688463FD001233B704FF47A707F
:1079B80000237B60FFF77CFF044688B92B68042B03
:1079C80013D11B4A536943F4803343F004035361D2
:1079D8004FF47A70FFF76CFF0446154B1A681B6862
:1079E80000233B702046BDE8F0814FF0FF33C8F814
:1079F80000306E68D5E901321344B3420AD93046E3
:107A0800FFF7BCFF4FF47A70FFF752FF50B1C8F888
:107A180000600446064A536923F47E7323F0020388
:107A28005361DAE70136E5E70224DBE7D80E0020E8
:107A3800004000582DE9F04F524C00234FF00F0939
:107A48000A6832FA03F501D1BDE8F08F012505FA7D
:107A580003F818EA020200F08E804E68032706F049
:107A680003054FEA430E07FA0EFC6F1E012F6FEA5B
:107A78000C0C32D8876807EA0C0ACF6807FA0EF7A9
:107A880047EA0A078760476827EA0808C6F3001725
:107A98009F4047EA08074760C76807EA0C088F68ED
:107AA80007FA0EF747EA0807022DC76017D14FEA11
:107AB800D30800EB880803F0070AD8F820704FEACB
:107AC8008A0A09FA0AFB27EA0B0B0F6907FA0AF771
:107AD80047EA0B07C8F8207001E0032DDCD10768DE
:107AE80005FA0EF507EA0C073D4316F4403F05601A
:107AF80041D023F0030707F1804707F5803703F0EB
:107B0800030CBD684FEA8C0C4FF0070E0EFA0CFE02
:107B1800B0F1904F25EA0E0E2FD01B4DA8422ED063
:107B280005F58065A84214BF0725022505FA0CF55E
:107B380045EA0E05BD602568D74316F4801F0CBFC3
:107B48003D4015432560656816F4001F0CBF3D4095
:107B580015436560D4F8805016F4803F0CBF3D4053
:107B68001543C4F88050D4F88450B60354BF3D4040
:107B78001543C4F88450013362E70025D6E7012590
:107B8800D4E700BF0008005800040048374A2DE930
:107B9800F04F00234FF0010A4FF0070B4FF00F0989
:107BA80031FA03F401D1BDE8F08F0AFA03FC1CEAAC
:107BB800010654D023F0030404F1804404F5803412
:107BC80003F00307A568BF000BFA07F8B0F1904F60
:107BD80008EA050E45D0264DA84244D005F5806533
:107BE800A8420CBF02250725BD40754517D1D2F81C
:107BF800805025EA0605C2F88050D2F8845025EA5C
:107C08000605C2F88450156825EA0605156055680A
:107C180025EA06055560A56825EA0805A5600568F2
:107C280003265C0006FA04F423FA06F6254300EB63
:107C38008606056003F00705376AAD0009FA05F501
:107C480027EA05073762856825EA040585604568DF
:107C580025EA0C054560C56825EA0404C4600133BB
:107C68009EE70025C0E70125BEE700BF00080058D1
:107C7800000400480369194214BF0120002070471E
:107C88000AB181617047816270470000044AD16877
:107C9800014208B502D0D060FBF7C2FB08BD00BFA7
:107CA8000008005803689A69910744BF00229A6245
:107CB8009A69D2075EBF9A6942F001029A617047D9
:107CC80030B5039D04682B4343EA0243064A6068C3
:107CD800C1F309010B4342EA555223F0004320EA5D
:107CE80002000343636030BDFF63FF0303682DE9AF
:107CF800F0419C6914F0100405460F4616466FD0F3
:107D080010220024DA61A0462B689A69900661D493
:107D1800B8F1000F35D044F0040401202E68B3698F
:107D2800D90541BF4FF48072F26144F0010401208B
:107D38005A0541BF4FF4806244F00804F261012003
:107D48009B054FD54FF4007344F00204F3612846B5
:107D5800FFF7A8FF736823F0FF7323F48B3323F432
:107D6800FF7323F0010373606B6C23436B64202360
:107D780085F84130002385F8423085F840300120ED
:107D880032E07A1CC1D0FAF7A1FE801BB84201D8B4
:107D9800002FB9D12B68596895F8422098690004DA
:107DA800D2B20AD5490408D4202A06D05A6842F427
:107DB80080425A60FAF78AFE06462B689B699B0642
:107DC800A2D4FAF783FE801B1928F6D920244FF095
:107DD800010899E7B8F1000F9DD12022DA619AE7EE
:107DE80020469BE70028B2D1BDE8F08170B5044673
:107DF8000D46164623689B699B0701D500201BE0AA
:107E0800324629462046FFF771FFA0B96A1CF1D017
:107E1800FAF75CFE801BA84201D8002DEAD1636CFA
:107E280043F020036364202384F84130002384F85E
:107E3800423084F84030012070BD70B504460D46CC
:107E4800164623689B699B0601D5002019E0324637
:107E580029462046FFF74AFF90B9FAF737FE801BFC
:107E6800A84201D8002DECD1636C43F02003636471
:107E7800202384F84130002384F8423084F84030CD
:107E8800012070BD70B504460D46164623689B69EF
:107E98005B070ED4324629462046FFF727FF38BB3A
:107EA80023689A69910625D59A69520703D5228DC8
:107EB8000AB1002070BD9A6912F010021CBF10228E
:107EC800DA614FF0200118BF04226264D9615A6850
:107ED80022F0FF7222F48B3222F4FF7222F00102A8
:107EE8005A60002384F8411084F8423084F8403006
:107EF8000120DFE7FAF7EAFD801BA84201D8002D30
:107F0800C4D1636C43F020036364202384F84130B8
:107F18000023EBE72DE9F041069F04468846164604
:107F28001D462268936938EA03030CBF0123002326
:107F3800B34201D0002015E06B1CF3D0FAF7C6FD60
:107F4800C01BA84201D8002DEBD1636C43F020037D
:107F58006364202384F84130002384F8423084F895
:107F680040300120BDE8F08110B5044600284AD011
:107F780090F8413003F0FF021BB980F84020FAF76F
:107F88007FFA242384F8413023681A6822F001021A
:107F98001A60626822F070621A619A6822F40042DC
:107FA8009A60D4E90221012924D142F400429A605E
:107FB8005A6842F0007242F400425A60DA6822F4C9
:107FC8000042DA60D4E904210A43A16942EA0122A5
:107FD800DA60D4E907210A431A601A6842F00102FC
:107FE8001A6000202023606484F84130206384F8FC
:107FF800420010BD42F4044202299A6004BF4FF4C3
:1080080000625A60D4E70120F3E700002DE9F34746
:10801800984690F841300A9F202B04460E46914618
:1080280040F0868090F84030012B00F081804FF0BE
:10803800010A80F840A0FAF749FD19230546009087
:1080480052464FF400412046FFF764FF18B1012063
:1080580002B0BDE8F087212384F84130102384F86A
:1080680042306064A4F82A80638DC4F824909BB2DF
:10807800FF2B60632F4B26D9FF22228500934FF0F8
:10808800807331462046FFF71BFE638D9BB22A465C
:1080980039462046FBB9FFF7D0FE0028D7D1236820
:1080A8002021D9615A6822F0FF7222F48B3222F41F
:1080B800FF7222F001025A6084F8411084F84000EF
:1080C80084F84200C4E7628D92B2228500934FF093
:1080D8000073D2B2D5E7FFF789FE0028B7D1636AEB
:1080E800226813F8011B91626362638D228D013B44
:1080F8009BB26385638D013A92B29BB22285002BB5
:10810800C3D0002AC1D100953B4680212046FFF705
:1081180001FF00289BD1638D9BB2FF2B03D9FF225F
:1081280022850090ABE7628D92B222850090CEE75F
:1081380002208DE7002000802DE9F347984690F84B
:1081480041300A9F202B04460E46914640F0878016
:1081580090F84030012B00F082804FF0010A80F83F
:1081680040A0FAF7B3FC19230546009052464FF495
:1081780000412046FFF7CEFE18B1012002B0BDE84D
:10818800F087222384F84130102384F84230606459
:10819800A4F82A80638DC4F824909BB2FF2B6063F7
:1081A800304B26D9FF22228500934FF08073314649
:1081B8002046FFF785FD638D9BB22A463946204647
:1081C800FBB9FFF73AFE0028D7D123682021D961EF
:1081D8005A6822F0FF7222F48B3222F4FF7222F0E6
:1081E80001025A6084F8411084F8400084F8420083
:1081F800C4E7628D92B2228500934FF00073D2B229
:10820800D5E7FFF73FFE0028B7D123685A6A636AAB
:108218001A70636A228D01336362638D013B9BB2DE
:108228006385638D013A92B29BB22285002BC2D03E
:10823800002AC0D100953B4680212046FFF76AFE00
:1082480000289AD1638D9BB2FF2B03D9FF22228588
:108258000090AAE7628D92B222850090CDE70220B5
:108268008CE700BF0024008010B590F84120202A38
:108278000346D4B21CD190F84020012A18D02422F9
:1082880080F841200268106820F001001060106832
:1082980020F48050106010680143116011680020BC
:1082A80041F00101116083F8414083F8400010BD9E
:1082B8000220FCE710B590F84120202A0346D4B2EA
:1082C8001BD190F84020012A17D0242280F84120A1
:1082D8000268106820F001001060106820F47060D7
:1082E80040EA012111601168002041F0010111608C
:1082F80083F8414083F8400010BD0220FCE70000ED
:10830800024A136843F480731360704700040058EE
:108318000D4B10B55B690C4628B99A0507D500F0D6
:1083280039F820B110BD9B0501D400F02BF8074A9D
:108338001369012C23F00403136101D130BFF1E765
:1083480040BF20BF20BFEDE70004005800ED00E06B
:10835800064A136823F0070343F003031360044A33
:10836800136943F00403136130BF704700040058D9
:1083780000ED00E0024B186800F4C060704700BFD1
:1083880000040058024A136843F48043136070479E
:10839800000400580C4A136823F4804313600B4B05
:1083A8001B6832214B430A49B3FBF1F35169890534
:1083B80000D533B9536913F4007F14BF032000209C
:1083C8007047013BF2E700BF00040058280800206E
:1083D80040420F000B4A136823F0070343F00203DF
:1083E8001360094B1A69012842F004021A6105D189
:1083F80030BF1A6922F004021A61704740BF20BFDB
:1084080020BFF6E70004005800ED00E04FF0B0434D
:108418001868C0F3404070474FF0B0431868C0F385
:10842800400070474FF0B042536823F47F4343EA5B
:108438000023536070474FF0B0431868C0F34060A2
:10844800704700007FB54FF0B0432C4AD3F808318D
:10845800C0F3031003F00F0352F82040284A52F8E3
:108468002330B4FBF3F4FFF785FF264B054693E86A
:108478000700B5F5007F04AB03E9070010D0224BD5
:108488009C4218D303F5B70303F67F539C4229D9BE
:1084980003F5741303F510639C4225D802230BE0FF
:1084A8001A4B9C4207D91A4B9C421BD903F5370338
:1084B80003F5D853F0E7002304AA02EB830353F82B
:1084C8000C4C144D2B6823F0070323432B60FAF759
:1084D800FDFA06462B6803F007039C4206D10020EC
:1084E80004B070BD0123E7E70024EAE7FAF7EEFAE3
:1084F800801B0228EED90320F2E700BF883B010861
:10850800E83B0108303A0108C0CF6A00BFEA210100
:108518003F933402004000584FF0B04310B59A68BA
:10852800D96812F00C0205D00C2A4AD101F00303D5
:10853800012B51D14FF0B0412B480B6813F00803C1
:1085480006D00B6813F0080337D1D1F8941007E070
:108558000C68240756BFD1F894300968C3F3032385
:1085680050F82330002A0CBF184600204FF0B041C5
:108578008A6802F00C020C2A1ED1CA6802F00302B3
:10858800022A2ED0032A06D10B68184A13F4801F3A
:10859800174B18BF13464FF0B042D068D168D26865
:1085A800C0F306205843C1F302130133B0FBF3F0C4
:1085B800530F0133B0FBF3F010BD0B68C3F3031383
:1085C800CEE7042A05D0082A06D11B6813F48013C5
:1085D80005D006480023C9E700231846C6E7044823
:1085E800C4E7024BD7E700BF883B01080024F4002A
:1085F8000048E80108B5FFF78FFF4FF0B043044A81
:108608009B68C3F3031352F82330B0FBF3F008BDA3
:10861800E83B01082DE9F0410446002853D04FF00B
:10862800B0439D68DE6803689B0605F00C0506F0FC
:10863800030668D5026A1DB10C2D46D1012E44D11E
:10864800002A40D04FF0B043A16A1A68170756BFF6
:10865800D3F894301B681B0903F0F00399421FD923
:108668000846FFF7EFFE00282DD14FF0B0421368FF
:1086780043F0080313601368A16A23F0F0030B4367
:108688001360606AFFF7CEFEFFF7B4FFAB4B1860CC
:10869800AB4B1868FAF718FA002834D0BDE8F08117
:1086A8004FF0B042136843F008031360136823F0D7
:1086B800F0030B431360606AFFF7B4FE0846FFF748
:1086C800C1FE0028E0D00120E8E74FF0B043002ABF
:1086D80054D01A6842F001021A60FAF7F7F907460F
:1086E800FFF79AFE002842D04FF0B042136843F0DB
:1086F800080313601368A16A23F0F0030B431360A7
:10870800606AFFF78FFE2368D80748D42368990763
:1087180000F18C8023681E0740F1FA80A3694FF0AE
:10872800B046002B00F0E180D6F89430E16903F000
:108738001002914200F0C48003F00302022AC2D062
:10874800D80740F1B380D6F8943023F00103C6F877
:108758009430FAF7BBF90746D6F89430990740F1F8
:10876800A580FAF7B3F9C31B112BF5D904E0FAF782
:10877800ADF9C01B0228B3D903208FE71A6822F08D
:1087880001021A60FAF7A2F90746FFF745FE00282A
:10879800B9D0FAF79BF9C01B0228F6D9ECE7082DE7
:1087A80003D00C2D05D1032E03D16368002BADD166
:1087B80089E74FF0B043A1681A6822F480120A438F
:1087C8001A606268B2F5803F10D11A6842F48032AC
:1087D8001A60FAF77BF90746FFF718FE002895D1CB
:1087E800FAF774F9C01B6428F6D9C5E7B2F5041F77
:1087F80004D11A6842F400121A60E6E7196821F4F5
:1088080080311960196821F400111960002AE0D13B
:10881800FAF75CF90746FFF7F9FD00283FF476AF51
:10882800FAF754F9C01B6428F5D9A5E7042D236984
:1088380003D00C2D0ED1022E0CD1002B3FF443AFE8
:108848004FF0B0426169536823F0FE4343EA016385
:1088580053605FE74FF0B046BBB1336843F48073B1
:108868003360FAF733F9074633685A0505D4FAF73F
:108878002DF9C31B022BF7D97EE77368626923F0D1
:10888800FE4343EA0263736044E7336823F480736A
:108898003360FAF71BF9074633685B057FF53AAF93
:1088A800FAF714F9C31B022BF6D965E74FF0B0426B
:1088B800E169D2F8943023F010030B43C2F89430E6
:1088C8004FF0B047D7F8943043F00103C7F894301D
:1088D800FAF7FCF80646D7F894309A0718D4FAF74E
:1088E800F5F8831B112BF6D946E7D6F8943023F018
:1088F8000103C6F89430FAF7E9F80746D6F8943039
:108908009B0705D5FAF7E2F8C31B112BF6D933E715
:108918002368580754D50B4F3B68D90514D4FFF783
:10892800EFFCFAF7D3F806463B68DA050CD4FAF7F9
:10893800CDF8831B022BF7D91EE700BF28080020BB
:108948002C08002000040058E3684FF0B046002BC4
:1089580058D023F08003052B02BFD6F8903043F09F
:108968000403C6F890304FF0B046FAF7AFF8D6F8DF
:10897800903043F001030746C6F8903041F288383A
:10898800D6F890309B0705D4FAF7A0F8C31B4345E7
:10899800F6D9F1E6E36823F00403812B1BD1FAF73B
:1089A80095F8D6F8903043F08003C6F89030074623
:1089B8004FF0B04641F28838D6F89030180504D503
:1089C800E36A002B4AD1002068E6FAF77FF8C01B5B
:1089D8004045F1D9D0E6FAF779F8D6F8903023F087
:1089E8008003C6F8903007464FF0B04641F2883809
:1089F800D6F890301905E3D5FAF768F8C01B40455A
:108A0800F6D9B9E6FAF762F8D6F8903023F0800381
:108A18000746C6F8903041F28838D6F890301A05E3
:108A280016D4FAF753F8D6F8903023F00103C6F8B5
:108A3800903007464FF0B04841F28836D8F8903069
:108A48009B07BDD5FAF742F8C31BB342F6D993E6A4
:108A5800FAF73CF8C01B4045DFD98DE60C2D4ED007
:108A6800022B4FF0B0431A6822F080721A6033D19B
:108A7800FAF72CF80546FFF7DEFC38BBD4E90C31D1
:108A88004FF0B0420B43D0682D4901400B43E16BD6
:108A98000B43216C0B43616C0B43A16B43EA01232D
:108AA800D360136843F080731360D36843F0805336
:108AB800D360FAF70BF80446FFF7BDFC002882D113
:108AC800FAF704F8001B0A28F6D955E6F9F7FEFF6D
:108AD800401B0A28CFD94FE6F9F7F8FF0446FFF7FD
:108AE800AAFC30B94FF0B042164BD1680B40D360A6
:108AF80069E7F9F7EBFF001B0A28F0D93CE6012BE0
:108B08003FF4E1AD4FF0B043D868236B00F00302A7
:108B18009A427FF4D8AD626B00F0700393427FF401
:108B2800D2ADA26B00F4FE43B3EB022F7FF4CBADC2
:108B3800636C00F06040C01A18BF0120AEE500BFAA
:108B48008C80C111FCFFFEEE2DE9F0410D46044674
:108B580010B90120BDE8F081684E336803F00703BF
:108B68008B4216D323689A0727D54FF0B047A268DF
:108B7800BB6823F0F0031343BB60F9F7A7FF064671
:108B8800BB68DB0319D4F9F7A1FF831B022BF7D9C4
:108B980011E0336823F007030B433360F9F796FFBE
:108BA8000746336803F00703AB42DBD0F9F78EFFC3
:108BB800C01B0228F5D90320CCE72368580617D52F
:108BC8004FF0B0476269D7F8083123F00F0343EA42
:108BD8001213C7F80831F9F779FF0646D7F80831B4
:108BE800D90305D4F9F772FF831B022BF6D9E2E704
:108BF80023685A0713D54FF0B047E268BB6823F4DF
:108C0800E0631343BB60F9F761FF0646BB689B034B
:108C180005D4F9F75BFF831B022BF7D9CBE7236851
:108C2800180714D54FF0B0472269BB6823F4605386
:108C380043EAC203BB60F9F749FF0646BB6859031C
:108C480005D4F9F743FF831B022BF7D9B3E7236851
:108C5800DA070FD4294C236803F00703AB4239D84D
:108C6800FFF7C8FC264B1860264BBDE8F041186892
:108C7800F9F72ABF6268022A1DD1FFF7C7FB00284F
:108C88003FF467AF4FF0B04641F28838B36823F03D
:108C980003031343B360F9F719FF0746B368626823
:108CA80003F00C03B3EB820FD4D0F9F70FFFC01B0E
:108CB8004045F3D97FE7032A02D1FFF7BCFBDEE783
:108CC80012B9FFF7A9FBDAE74FF0B0431B685B0561
:108CD800D8D43EE7236823F007032B432360F9F732
:108CE800F5FE0646236803F00703AB42B8D0F9F750
:108CF800EDFE801B0228F5D95DE700BF0040005853
:108D0800280800202C08002008B5FFF773FC4FF056
:108D1800B043044A9B68C3F3022352F82330D84077
:108D280008BD00BFC83B010808B5FFF763FC4FF05A
:108D3800B043044A9B68C3F3C22352F82330D84097
:108D480008BD00BFC83B01084FF0B043D3F89000FE
:108D5800C0F3400070474FF0B0410209D1F88830A5
:108D680002F47F22000123EA020300F47F20034378
:108D7800C1F8883070474FF0B041020CD1F8883004
:108D8800120423EA020343EA0040C1F8880070474E
:108D98000368DA0370B5044639D5FFF7B1FAF9F775
:108DA80095FE614E05463368DB0532D54FF0B0437A
:108DB800616BD3F8902002F4407291421DD0D3F831
:108DC8009010D3F8902042F48032C3F89020D3F862
:108DD800902021F4407022F480328D07C3F890204F
:108DE800C3F8900009D5F9F771FE41F288360546B7
:108DF800FFF7AAFF012840F090804FF0B042616B66
:108E0800D2F8903023F440730B43C2F89030002618
:108E180005E0F9F75BFE401B0228C4D90326256844
:108E2800E8070AD54FF0B0416268D1F8883023EAE4
:108E3800124392B21343C1F88830A9070AD54FF0FC
:108E4800B041A268D1F8883023EA124392B21343A2
:108E5800C1F88830AA0609D54FF0B0422169D2F886
:108E6800883023F440630B43C2F88830AB0502D541
:108E7800206AFFF780FF680502D5606AFFF77BFF6D
:108E8800290502D5A06AFFF776FF6A0602D5606950
:108E9800FFF761FF2B0602D5A069FFF75CFFE80525
:108EA80002D5E069FFF757FFE90610D54FF0B04249
:108EB800E168D2F8883023F440730B43C2F8883055
:108EC800B1F5807F02BFD36843F08073D3602A0472
:108ED8000ED54FF0B042216BD2F8883023F04043D2
:108EE8000B43C2F8883019B9D36843F08073D36054
:108EF8006B0410D54FF0B042E16AD2F8883023F005
:108F080040530B43B1F1005FC2F8883003D1D368F6
:108F180043F48033D360304670BDF9F7D7FD401B6A
:108F2800B0427FF665AF79E70004005830B590F895
:108F38002C30012B02464FF0020022D0174B82F84A
:108F48002D00CA24012582F82C505C6253245C62EF
:108F5800B1F5807F146B996914D121F48851996116
:108F6800596C24F0010421F0004159641463DD6553
:108F78000A4BFF2159620020012382F82D3082F824
:108F88002C0030BD21F408519961D96C24F00204F9
:108F980021F00041D9641463D865E9E7002800404E
:108FA80070B50B4E036B756D1D40EA07044603D57B
:108FB8000123F365F9F79DFEAB0704D50223F3659A
:108FC800204600F0C9F9012384F82D3070BD00BF98
:108FD8000028004038B50A4CE36823F02003E3601A
:108FE800F9F774FD0546E3689B0601D5002038BDF6
:108FF800F9F76CFD401BB0F57A7FF4D90320F6E74A
:1090080000280040F8B5114DEC6814F040040646FD
:109018001AD1EB6843F08003EB60F9F757FD23465C
:109028000746EC6814F0400401D1032B01D118461F
:10903800F8BDF9F74BFDC01BB0F57A7F234684BF16
:10904800032386F82D30ECE70023F0E700280040E2
:1090580038B50F4CE36823F08003E360A3699B06EF
:10906800054606D4FFF7B6FF10B1032085F82D009A
:1090780038BDA36923F02003A361FFF7ABFF10B14C
:10908800032085F82D00A36943F02003A361EFE7CF
:109098000028004038B5044600284BD090F82D3001
:1090A80003F0FF021BB980F82C20F9F7E7FA022336
:1090B800214D84F82D30EB68DB0636D4CA236B6269
:1090C80053236B622046FFF79DFF10B1FF236B62AD
:1090D80038BDAB6923F08E6323F04003AB6121698F
:1090E8006368AA690B431343A2691343AB61D4E9CC
:1090F800022343EA02432B61D4E90931EA680B43AE
:1091080022F4F8521343EB602046FFF7A1FF002832
:10911800DCD1D4E90713AA690B4322F06042134358
:1091280062691343AB61FF236B62012384F82D301E
:109138000020CDE70120CBE70028004000230928C4
:1091480003D840EA0310C0B270470A380133C0B2EE
:10915800F5E700002DE9F04790F82C30012B054683
:109168004FF0020069D0012385F82C304E4B85F86A
:109178002D00DE6806F44076B6F5807F78D04C691D
:10918800087891F8019091F802A091F82470002ACB
:1091980055D19B6913F0400308BFCB70FFF7CEFF92
:1091A80080464846FFF7CAFF02465046FFF7C6FF0B
:1091B80081463846FFF7C2FF0B6ACF78234343EA5C
:1091C800875343EA090343EA084343EA022343EA8D
:1091D8000063354ACA205062532050628C6A8869FD
:1091E800B4F5807F946945D124F4885494610124AE
:1091F800D465B6F5807F09BFCB6913640343536414
:1092080018BF5064284B4A681A672A6B42F001025B
:109218002A639A6942F488529A61244AD2F88030C3
:1092280043F40033C2F880301F4BFF225A620020FB
:10923800012385F82D3085F82C00BDE8F087B4F1BE
:10924800803F07D0B4F5000F04D09B6913F04003AA
:1092580008BFCB700B6ACA781C4344EA0A0444EA84
:10926800004343EA092343EA825343EA0763B0E72A
:109278000023AEE724F4085494610224D465B6F5BB
:10928800807F09BFCB6993640343D36418BFD0645C
:10929800054B4A685A672A6B42F002022A639A69A8
:1092A80042F40852B8E700BF002800400008005800
:1092B80090F82C20012A03464FF0020012D00A4AE7
:1092C80083F82D00CA21516253215162916941F0FE
:1092D80020019161FF2151620020012283F82D2095
:1092E80083F82C00704700BF0028004090F82C201D
:1092F800012A03464FF0020019D00D4A83F82D00C9
:10930800CA2151625321516291690A4841F0800192
:109318009161D0F8801041F48021C0F88010FF21BD
:1093280051620020012283F82D2083F82C00704719
:109338000028004000080058064B5A6D520610B528
:10934800044603D54022DA65F9F7D6FC012384F8F0
:109358002D3010BD002800407047890001F1804180
:1093680001F531410A607047890001F1804101F53A
:109378003141086870470000034AD2F8903043F43E
:109388000043C2F89030704700040058034AD2F8EE
:10939800903023F40043C2F890307047000400581E
:1093A800074B1A6822F040021A6040F441704FF4EB
:1093B800B85218605A601A6842F040021A60704742
:1093C8000000015837B5054600284ED0837903F0D0
:1093D800FF046BB1032C0BD0254B4FF400629A614C
:1093E8002868FFF7DDFF002401232B71AC602FE014
:1093F80000236B712846F9F783FA1E4AD2F8903099
:1094080043F48053C2F89030002CE5D102234FF08A
:10941800B042AB71D2F8943023F40043C2F89430D0
:10942800154B1B681C214B43DB0C64214B430193F8
:10943800019B93B90124AC60FFF79EFF0C4B9A681F
:1094480042F400629A604FF400629A61002CC7D01F
:109458000123AB71204603B030BD019B013B019352
:10946800D2F894305B04E3D4E6E70124F2E700BFC6
:1094780000040058000800582808002037B5174D88
:109488002B6802461C204343DB0C642043431448EA
:109498000193019B93B901209060114C21732B68B3
:1094A8001C214B43DB0C64214B430193019B6BB99B
:1094B800012090600A4BDB6803B030BD019B013B83
:1094C800019383689C07E4D50020E6E7019B013BF4
:1094D8000193A368DB07E9D5ECE700BF2808002063
:1094E8000000015837B5184D2B6802461C2043432D
:1094F800DB0C6420434315480193019BA3B9012069
:109508009060124CFF2323732B681C256B43DB0CE4
:1095180064256B430193019B73B9012090600B4B49
:10952800DB680B7003B030BD019B013B019383687E
:109538009C07E2D50020E4E7019B013B0193A36867
:10954800DB07E8D5EBE700BF28080020000001583A
:109558000E4B0F491B681822534382B01B0D64221F
:10956800534301934B69019AC3F3800322B9022341
:109578008360012002B07047019A013A01924A695A
:10958800920701D5002BEDD10020F3E72808002031
:109598000004005807B50379012B0FD10A4B1B684B
:1095A800182253431B0C0193FFF7F0FE019B013B6C
:1095B8000193019B002BF9D1FFF7DEFE03B05DF8A4
:1095C80004EBFFF7C5BF00BF28080020F8B51E460A
:1095D8008379012B154604460F46DAB22DD143791B
:1095E800012B2AD0022342718371FFF7D3FF0D218B
:1095F8002046FFF7CBFEFFF741FF390A2046FFF769
:109608003DFFF9B22046FFF739FF2E44B5420ED18F
:109618002046FFF7B1FEFFF79BFFA0680123003843
:10962800A3714FF0000318BF01206371F8BD15F84E
:10963800011B2046FFF722FFE8E70220F6E7F8B50E
:109648001E468379012B154604460F46DAB22FD100
:109658004379012B2CD04271FFF79CFF1D21204636
:10966800FFF794FEFFF70AFF390A2046FFF706FFC7
:10967800F9B22046FFF702FF00212046FFF7FEFE61
:109688002E44B5420ED12046FFF776FEFFF760FF65
:10969800A06801230038A3714FF0000318BF012010
:1096A8006371F8BD29462046FFF71CFF0135E8E73E
:1096B8000220F6E7F8B51F468379012B15460446C4
:1096C8000E46DAB22CD14379012B29D04271FFF72B
:1096D80061FF06F0EF03A3F1840253425341237163
:1096E80031462046FFF752FEFFF7C8FE2F44AF422F
:1096F80010D1FFF741FE842E02D02046FFF728FF45
:10970800A06801230038A3714FF0000318BF01209F
:109718006371F8BD15F8011B2046FFF7AFFEE6E7B9
:109728000220F6E7F8B51E468379012B1546044654
:109738000F46DAB227D14379012B24D04271FFF7C3
:1097480029FF39462046FFF721FEFFF797FE002143
:109758002046FFF793FE2E44B5420ED12046FFF770
:109768000BFEFFF7F5FEA06801230038A3714FF048
:10977800000318BF01206371F8BD29462046FFF792
:10978800B1FE0135E8E70220F6E737B50023ADF86A
:10979800043001AA022312210546FFF7C3FFBDF8D2
:1097A8000440022364BA01AAA4B219462846FFF766
:1097B80081FFE20702D5284609F0B4F9A30702D5CC
:1097C800284609F0B5F9600702D5284609F0DAF904
:1097D800210702D5284609F0DBF9E20602D528461A
:1097E80009F0DCF9A30602D5284609F0C5F9600698
:1097F80002D5284609F0A2F9210606D514F480718D
:1098080018BF0121284609F09FF9A20502D528466C
:1098180009F0AAF9630402D5284609F0C5F903B08E
:1098280030BDF8B51E468379012B154604460F4610
:10983800DAB227D14379012B24D04271FFF7AAFE6F
:109848000E212046FFF7A2FDFFF718FE39462046F5
:10985800FFF714FE2E44B5420ED12046FFF78CFDCB
:10986800FFF776FEA06801230038A3714FF00003CC
:1098780018BF01206371F8BD15F8011B2046FFF7DA
:10988800FDFDE8E70220F6E7F8B51E468379012BCF
:10989800154604460F46DAB22BD14379012B28D05E
:1098A8004271FFF777FE1E212046FFF76FFDFFF795
:1098B800E5FD39462046FFF7E1FD00212046FFF788
:1098C800DDFD2E44B5420ED12046FFF755FDFFF7CA
:1098D8003FFEA06801230038A3714FF0000318BFB2
:1098E80001206371F8BD29462046FFF7FBFD0135CD
:1098F800E8E70220F6E7026852E8003F23F0C003D9
:1099080042E8003102680029F5D102F1080353E862
:10991800003F23F4000302F1080C4CE80031002951
:10992800F3D12023C0F888307047000010B50268D2
:1099380052E8003F23F4907342E80031026800299E
:10994800F5D10F4C02F1080353E8003F234002F120
:10995800080C4CE800310029F4D1C36E012B07D163
:1099680052E8003F23F0100342E800310029F7D104
:109978002023C0F88C300023C366436710BD00BFA6
:10998800FEFFFFEF38B50546C8B12423C0F888307C
:1099980003681A68002422F001021A601C605C60E7
:1099A8009C60F9F755FAC5F8904085F88440C5F8E9
:1099B80088402046C5F88C40EC662C6738BD0120ED
:1099C800FCE70000F8B504461346D4F88850202D6B
:1099D80032D1F1B1EAB1E06FA4F85620A4F85420CE
:1099E80000262122C4F890602165C4F888202268E6
:1099F80088B1124FC762124F0763124F2832C0E96D
:109A08000D76FDF785FE30B11023C4F89030C4F808
:109A180088500120F8BD236840221A62226802F1AA
:109A2800080353E8003F43F0800302F1080141E8CE
:109A380000300028F3D1EDE70220EBE7519A000847
:109A4800999A0008A59A000808B50346806A1B6819
:109A58001B6813F0200317D1A0F85630026802F1F2
:109A6800080353E8003F23F08003083242E800313E
:109A780002680029F2D152E8003F43F0400342E86F
:109A880000310029F7D108BDF9F75CFAFBE7704708
:109A980008B5806AFFF7FBFF08BD7047806A38B5D4
:109AA8000468D0F88830D0F88C50A268120606D521
:109AB800212B04D10023A0F85630FFF71CFFA36820
:109AC8005B0606D5222D04D10023A0F85E30FFF7EF
:109AD8002DFFD0F8903043F01003C0F89030FFF716
:109AE800DCFF38BD70470000D0F88C20B0F860105B
:109AF800222A08B5036855D15B6A826D0B40137042
:109B0800836D01338365B0F85E30013B9BB2A0F8EA
:109B18005E30B0F85E309BB2002B42D1026852E84A
:109B2800003F23F4907342E8003103680029F5D11F
:109B380003F1080252E8002F22F0010203F1080C99
:109B48004CE800210029F3D12022C0F88C20184AC3
:109B580041679342016705D1C26E012A0ED0F9F719
:109B6800FFF91EE05A681102F6D553E8002F22F0DB
:109B7800806243E800210029F7D1EDE70022C266A0
:109B880053E8002F22F0100243E800210029F7D102
:109B9800DA69B0F85C10D20644BF10221A62FFF7E7
:109BA800A1FF08BD9A6942F008029A61F9E700BF6F
:109BB80000800040D0F88C20B0F86010222A08B548
:109BC800036852D15A6A1140826D22F8021B8265DD
:109BD800B0F85E20013A92B2A0F85E20B0F85E209C
:109BE80092B2002A40D153E8002F22F4907243E841
:109BF80000210029F7D103F1080252E8002F22F0D2
:109C0800010203F1080C4CE800210029F3D12022BD
:109C1800C0F88C20174A41679342016705D1C26E8C
:109C2800012A0ED0F9F79CF91EE05A681102F6D500
:109C380053E8002F22F0806243E800210029F7D181
:109C4800EDE70022C26653E8002F22F0100243E835
:109C580000210029F7D1DA69B0F85C10D20644BFB8
:109C680010221A62FFF73EFF08BD9A6942F0080207
:109C78009A61F9E7008000402DE9F84F0368B0F8D1
:109C88006060D3F81CB01F689D68D0F88C20222A29
:109C9800044640F0B980B0F8683043B1DFF87491F9
:109CA800DFF874A14FF000081BF0200F20D1B4F8A2
:109CB8005E309BB2D3B1B4F868209A4216D92268B4
:109CC80002F1080353E8003F23F08053083242E8CA
:109CD800003122680029F2D1504B636752E8003FF7
:109CE80043F0200342E800310029F7D1BDE8F88F9E
:109CF8002368A26D5B6A33401370A36D0133A365BB
:109D0800B4F85E30013B9BB2A4F85E302368D3F808
:109D18001CB01BF0070F2ED01BF0010F09D0F9055E
:109D280007D501221A62D4F8902042F00102C4F843
:109D380090201BF0020F09D0EA0707D502221A6209
:109D4800D4F8902042F00402C4F890201BF0040FCD
:109D580009D0E80707D504221A62D4F8903043F0F6
:109D68000203C4F89030D4F8903023B12046FFF7AE
:109D780094FEC4F89080B4F85E309BB2002B93D167
:109D8800226852E8003F23F4807342E800312368D8
:109D98000029F5D103F1080252E8002F02EA09026E
:109DA80003F1080040E800210029F3D1202253459F
:109DB800C4F88C20616721670AD05A68110207D558
:109DC80053E8002F22F0806243E800210029F7D1F0
:109DD800E26E012A14D10022E26653E8002F22F035
:109DE800100243E800210029F7D1DA69B4F85C10C1
:109DF800D20644BF10221A622046FFF773FE53E7CB
:109E08002046F9F7ADF84FE79A6942F008029A61DF
:109E18006CE700BFFEFFFFEF00800040F19A0008EA
:109E28002DE9F84F0368B0F86060D3F81CB01F68DC
:109E38009D68D0F88C20222A044640F0B780B0F8FC
:109E4800683043B1DFF87091DFF870A14FF0000877
:109E58001BF0200F20D1B4F85E309BB2D3B1B4F818
:109E680068209A4216D9226802F1080353E8003F95
:109E780023F08053083242E8003122680029F2D1E9
:109E88004F4B636752E8003F43F0200342E800313C
:109E98000029F7D1BDE8F88F2368A26D596A3140CF
:109EA80022F8021BA265B4F85E20013A92B2A4F827
:109EB8005E20D3F81CB01BF0070F2ED01BF0010F4B
:109EC80009D0F90507D501221A62D4F8902042F08A
:109ED8000102C4F890201BF0020F09D0EA0707D549
:109EE80002221A62D4F8902042F00402C4F89020AA
:109EF8001BF0040F09D0E80707D504221A62D4F82A
:109F0800903043F00203C4F89030D4F8903023B175
:109F18002046FFF7C2FDC4F89080B4F85E309BB2CB
:109F2800002B95D1226852E8003F23F4807342E861
:109F3800003123680029F5D103F1080252E8002F07
:109F480002EA090203F1080040E800210029F3D1E0
:109F580020225345C4F88C20616721670AD05A68CB
:109F6800110207D553E8002F22F0806243E8002150
:109F78000029F7D1E26E012A14D10022E26653E8E3
:109F8800002F22F0100243E800210029F7D1DA69F6
:109F9800B4F85C10D20644BF10221A622046FFF7BC
:109FA800A1FD55E72046F8F7DBFF51E79A6942F033
:109FB80008029A616EE700BFFEFFFFEF00800040D5
:109FC800BD9B000838B5044603682169A2681D686E
:109FD800C0690A4361690A437749024329400A4331
:109FE8001A605A68E16822F440520A435A60734A78
:109FF800A16993421CBF226A11439A6822F06E42FB
:10A0080022F430620A439A60DA6A616A22F00F0227
:10A018000A43DA626A4A934219D14FF0B043694A57
:10A02800D3F8883003F0030343F44033934200F03D
:10A03800B480B3F1031F24D0013A934240F0B580B5
:10A04800B0F5004F40F08F80FEF766FA6EE05E4A8A
:10A0580093421CD14FF0B0435C49D3F8883003F0E9
:10A068000C0343F440228A4200F0978006D8002B64
:10A078007CD0574B9A42E3D0012026E0B2F10C1F66
:10A08800FAD1B0F5004F53D04FF4004075E04B4A79
:10A098009342F1D14FF0B043D3F8883003F44063D2
:10A0A800B3F5006F18D006D85BB1B3F5806FE3D174
:10A0B800FEF732FA07E0B3F5406FDDD14FF4004008
:10A0C8000BE0FEF721FE40B900204FF00113A36614
:10A0D8000023C4E91D3338BD3E4865683E4B626ABB
:10A0E80005EB450133F81220B0FBF2F39942C3D8CF
:10A0F800B3EB053FC0D800231946F7F705FD090261
:10A1080041EA10616B080002C0182A464FF00003AC
:10A1180041F10001F7F7F8FC304BA0F540729A4284
:10A12800AAD82368D860CFE7FEF7EEFD0028CBD089
:10A138006168294B626A33F81220B0FBF2F24B08CF
:10A1480003EB42034FF6EF72B3FBF1F3A3F11001F7
:10A15800914291D823F00F02216892B2C3F34203CF
:10A168001343CB60B0E7FEF7D7F904E0B0F5004F32
:10A17800DAD0FEF7C9FD0028A6D06368616A164ADE
:10A1880032F81120B0FBF2F000EB5300B0FBF3F013
:10A198004FF6EF73A0F11002C1E7B0F5004F0D487C
:10A1A800EBD1C5E7FEF7C0FDC0E7B0F5004FF9D029
:10A1B800FEF7BAFDDFE700BFF369FFCF008000407C
:10A1C80000380140020003000044004008000C0071
:10A1D80004000C000024F400283C0108FFFC0F00D8
:10A1E800836ADA0710B506D50168C46A4A6822F49A
:10A1F800003222434A609C0706D50168046B4A680E
:10A2080022F4803222434A60590706D50168446B1C
:10A218004A6822F4802222434A601A0706D5016858
:10A22800846B4A6822F4004222434A60DC0606D561
:10A238000168C46B8A6822F4805222438A609906B6
:10A2480006D50168046C8A6822F4005222438A60A9
:10A258005A060FD50168446C4A6822F480122243DA
:10A26800B4F5801F4A6005D14A68846C22F4C002A4
:10A2780022434A601B0606D50268C16C536823F462
:10A2880000230B43536010BD2DE9F843DDF82090FF
:10A2980005460F46164698462A68D36937EA0303E7
:10A2A8000CBF01230023B34201D0002029E0B9F1FB
:10A2B800FF3FF2D0F8F70AFCA0EB080048452C68ED
:10A2C80002D8B9F1000F1ED154E8003F23F4D0732F
:10A2D80044E80032002AF7D104F1080353E8003FAC
:10A2E80023F0010304F1080141E80032002AF3D108
:10A2F8002023C5F88830C5F88C30002385F88430D1
:10A308000320BDE8F88323685A07C5D5E3691B0510
:10A31800C2D54FF40063236254E8003F23F4D0739E
:10A3280044E80032002AF7D104F1080353E8003F5B
:10A3380023F0010304F1080141E80032002AF3D1B7
:10A348002023C5F88830C5F88C30C5F89030D4E79C
:10A3580073B504460026C0F89060F8F7B7FB236889
:10A368001B681A07054619D423681B685B070AD5BA
:10A378006FF07E43009300222B464FF48001204665
:10A38800FFF782FFB0B900202023C4F8883084F892
:10A398008400C4F88C30E06620670CE06FF07E43E0
:10A3A8000093324603464FF400112046FFF76CFF36
:10A3B8000028D9D0032002B070BD10B5044650B3B0
:10A3C800D0F888301BB980F88430F8F7D1FC2268BF
:10A3D8002423C4F88830136823F00103136020464F
:10A3E800FFF7F0FD012816D0A36A13B12046FFF746
:10A3F800F7FE23685A6822F490425A609A6822F05D
:10A408002A029A601A6842F0010220461A60BDE8E2
:10A418001040FFF79DBF012010BD000030B58165D9
:10A428008168A0F85C200023B1F5805FA0F85E2069
:10A43800436735D10369002B40F2FF1318BFFF2390
:10A44800A0F860300023C0F890302223C0F88C3088
:10A45800016801F1080353E8003F43F001030831A4
:10A4680041E800340368002CF2D1456E8468016924
:10A47800B5F1005F32D1B0F8685095422ED8B4F5E6
:10A48800805F244A03D1244C002908BF2246426732
:10A49800B1B153E8002F42F4807243E80021F7E796
:10A4A80029B90369002B14BF7F23FF23C8E7B1F143
:10A4B800805FC5D10369002B14BF3F237F23BFE70B
:10A4C80003F1080252E8002F42F0805203F108001D
:10A4D80040E800210029F3D1002030BDB4F5805FA9
:10A4E8000E4A03D10E4C002908BF2246426741B1EB
:10A4F80053E8002F42F4907243E800210029F7D175
:10A50800EAE753E8002F42F0200243E8002100293F
:10A51800F7D1E1E7819C0008299E0008F19A00081C
:10A52800BD9B0008D0F88C30202B30B415D1B9B1C0
:10A53800B2B100230468C3660A4B9C420AD0636820
:10A548001B0207D554E8003F43F0806344E8003518
:10A55800002DF7D130BCFFF761BF022030BC704737
:10A568000120FBE700800040436E30B52BB9012382
:10A57800A0F86A30A0F8683030BD0368094D9A68C1
:10A588009968094C490FC2F342626B5C615CDB005D
:10A59800B3FBF1F3A0F86A30AB5CA25CDB00B3FB61
:10A5A800F2F3E7E7483C0108403C01081FB504AB5B
:10A5B80003E9060090F88430012B04463AD00123C1
:10A5C80080F884302423C0F8883003681A6822F0A1
:10A5D80001021A609A6822F440120A439A6071B91B
:10A5E8005A68BDF80C009DF80E1022F010020243C4
:10A5F8005A605A6822F07F4242EA01625A601A6839
:10A6080042F001021A60F8F761FA6FF07E420346E1
:10A6180000924FF4800100222046FFF735FE38B93A
:10A628002023C4F88830002384F8843004B010BD97
:10A638000320F8E70220F9E790F88430012B0FD0C7
:10A64800012380F88430016851E8002F42F00202AB
:10A6580041E80023002BF6D180F884301846704773
:10A668000220704710B590F88430012B044617D0AB
:10A678002423C0F8883003681A68196821F001019A
:10A68800196042F000524FF0005141661A60FFF71E
:10A698006BFF2023C0F88830002084F8840010BDA8
:10A6A8000220FCE770B590F88430012B044617D0DF
:10A6B80005682423C0F888302E682B6823F001032E
:10A6C8002B60AB6823F060431943A960FFF74CFF88
:10A6D80020232E60C0F88830002084F8840070BDE4
:10A6E8000220FCE738B5084D052455F8043B2BB982
:10A6F800013C14F0FF04F8D1204638BDDB689847C8
:10A708000028F5D0F9E700BF2C100020034BD870C3
:10A71800034B1B681B6C03B11847704714100020CB
:10A7280010100020034B1874034B1B685B6C03B1BB
:10A73800184770471410002010100020F0B5314D54
:10A74800314B95F90420314E91B00C46012795F90B
:10A7580005108DF8047002288DF809208DF80A106C
:10A7680010D18DF80800D8711C7202F063FD33789F
:10A7780003B114B101A803F0C1F9254B059A1A6079
:10A7880011B0F0BD59714FF480711A71D9801C72E3
:10A7980033788DF8087053BB1F2306A88DF81C204A
:10A7A8008DF8183002F024FF20238DF8183006A801
:10A7B8002B798DF81C3002F01BFF22238DF81830FE
:10A7C80006A86B798DF81C3002F012FF21238DF852
:10A7D800183006A86B798DF81C3002F009FF292380
:10A7E8008DF8183006A80B4B079302F001FF02F012
:10A7F80021FD012306A88DF818308DF81C3002F0D1
:10A80800F7FEB4E71410002060080020F00E0020C6
:10A81800E40F0020000400017FB5092301A88DF88A
:10A82800043003F06BF90038044B059A1A6018BF1E
:10A838000120404207B05DF804FB00BFE40F002090
:10A8480070B504460B46144962784A700020A27815
:10A858000A7208701A884A729A788A72DB780B74BE
:10A868006368CB600D4B1B68DA6A2AB1237803F062
:10A87800FB030A2B00D09047094E002556F8043BED
:10A888001BB15B6A0BB1204698470135EBB2052B2B
:10A898006DB2F3D170BD00BF300800201010002049
:10A8A8002C10002070B5044611480123037063780A
:10A8B8004370A3788372E368C360E37803762369FF
:10A8C8004376237943720B4B1B689B6A03B1984705
:10A8D800094E002556F8043B1BB19B690BB1204675
:10A8E80098470135EBB2052B6DB2F3D170BD00BFAF
:10A8F80044080020101000202C100020014B18687C
:10A90800704700BFE40F002000B58BB001236846F4
:10A918008DF8003002F046FD38B99DF80400003883
:10A9280018BF01200BB05DF804FB0020FAE7000017
:10A9380008B501F037FE40B9FFF7E6FF012806D059
:10A94800054B197AD879FFF7F9FE012008BDBDE853
:10A958000840FFF7C7BE00BF600800202DE9F0419E
:10A9680086B005460E46174601F01CFE002873D136
:10A9780001F030FE044640B9FFF7C6FF01280AD0AF
:10A988003D4B197AD879FFF7D9FE6FF002042046BB
:10A9980006B0BDE8F081DFF8E48088F80860003E82
:10A9A80018BF01268DF80460354E687833798DF824
:10A9B8001230694602F094FC00283FD08DF804401C
:10A9C8000394ADF810406FF0060495E803002D4B92
:10A9D80083E80300337988F80A30394601A803F080
:10A9E80091F9294B059A1A6011283FD801A353F809
:10A9F80020F000BF67AA000861AA000875AA00082D
:10AA080075AA000875AA000875AA000875AA0008A2
:10AA180093A9000875AA000875AA000875AA000875
:10AA28005BAA000875AA000875AA000861AA0008B0
:10AA380061AA000861AA00087BAA00082B788DF893
:10AA480008306B78ADF810306B6803934FF0FF3423
:10AA5800BBE76FF005049AE76FF0010497E70B4B2B
:10AA680000221A70E31D18BF144690E74FF0FF3418
:10AA78008DE76FF004048AE760080020440800208E
:10AA88001410002054080020E40F0020E30F0020D9
:10AA980037B501F0A9FD134D052455F8043B4BB11A
:10AAA8001A693AB19B682BB1984718B155F8043C1C
:10AAB8001B699847013C14F0FF04EED1FFF712FE22
:10AAC80068B9094D2B7853B1084BADF80040D978D7
:10AAD800019422466846FFF741FF00B92C7003B085
:10AAE80030BD00BF2C100020E30F00201410002000
:10AAF80030B58BB0044601F055FD0546002835D128
:10AB0800FFF702FF012834D168468DF8005002F0A3
:10AB180049FC40BB9DF80430A34204D0012C22D04C
:10AB2800022C12D014B100200BB030BD002BFAD08B
:10AB380068468DF8044002F05BFDA0B90E4B1B6817
:10AB48001B6B002BEFD09847EDE763B968468DF88B
:10AB5800044002F04DFD30B9074B1B681B6B002BFE
:10AB6800E1D02046EFE74FF0FF30DDE76FF001005E
:10AB7800DAE76FF00200D7E71010002010B504469E
:10AB88008AB018B94FF0FF300AB010BD00236846EC
:10AB98008DF8003002F006FC0028F3D19DF804304F
:10ABA8002370F1E77FB500220B4620498DF8072076
:10ABB80001220A7042784A700446002A33D1027989
:10ABC8000A721A884A729A788A72DB780B74036957
:10ABD800CB60C378164D8DF80830037B8DF80930AB
:10ABE800836803932B68DB6A0BB102A898472B682C
:10ABF8009B6B13B1227E02B198470E4E052556F87D
:10AC0800043B1BB1DB690BB120469847013D15F0A9
:10AC1800FF05F4D10DF10700FFF7B0FF637913B119
:10AC2800054B01221A7004B070BD00BF3008002027
:10AC3800101000202C100020E30F002010B504464F
:10AC48008AB018B94FF0FF300AB010BD202368460B
:10AC58008DF8003002F0A6FB0028F3D1024A9DF9D6
:10AC6800043023701371EFE71410002000B58BB087
:10AC78002323019068468DF8003002F0B9FC0038B3
:10AC880018BF012040420BB05DF804FB70B5654C5D
:10AC980001468EB01822204606F0C0F8624B00220A
:10ACA8001A70F9F761F923784068012202FA03F172
:10ACB800014004D15D4B084608F09CF8FEE75C496A
:10ACC8005C481A4602F0F8F818B14FF0FF300EB0A1
:10ACD80070BD272304A88DF8103002F089FC564E69
:10ACE800564D002870D1012333702B68DB690BB1F6
:10ACF80000209847272304A88DF8103002F052FB53
:10AD0800059B93F84820227093F8182193F81A317C
:10AD18006270A370464BD3E9020105F06FFF054648
:10AD28000028D2D1464E062304A88DF8103002F030
:10AD380039FB059B736104A802F05AFC022304A89E
:10AD48008DF81030059602F02DFB0836032304A871
:10AD58008DF81030059602F025FB0F2606F014F842
:10AD6800012304A88DF814308DF8106002F040FC1F
:10AD780010230DEB03008DF810308DF8145002F0FD
:10AD880037FC04238DF8103004A8A3788DF814300C
:10AD980002F02EFC3A238DF8103004A8636905935D
:10ADA80002F026FC02A920788DF8086004F09CF8CF
:10ADB800003818BF0120E0711420FFF757FFE07931
:10ADC80003F062F9284682E728238DF810302B68B3
:10ADD8001B6943B104A802F0E5FA2B6805981B69C2
:10ADE80040F2C4519847272304A88DF8103002F088
:10ADF800FFFB50B9012304A88DF8103002F0D2FAF5
:10AE08009DF81430002B7FF46EAF3378002B7FF45D
:10AE18006CAF052204A88DF81020059302F0E8FB1A
:10AE280078E700BF14100020E30F0020503C010811
:10AE3800E80F002000100020F00E00201010002065
:10AE48005010002037B500230D4601930446D0B9B1
:10AE580000F0A8FB0190019BD3B10F4A42F82430BF
:10AE68000E4A9A620E4A1268916B1963916C596383
:10AE780092690C49D9625A6128465B680A49F222EC
:10AE88009847002006E001A900F092FB0028E2D0D4
:10AE98004FF0FF3003B030BD2C10002045A700084C
:10AEA8001010002021A80008F10E0020194B07B54A
:10AEB8001860194B194A1A60194A5A60194A9A6057
:10AEC800194ADA60194B02681A6042685A60826847
:10AED8009A60C268DA60164A1A6182695A61154B2B
:10AEE800C26B5A60144A019119609A601946134A54
:10AEF800DA600020FFF7A6FF48B901A800F056FB6A
:10AF0800003818BF0120404203B05DF804FB4FF041
:10AF1800FF30F9E71010002000100020ADA800084D
:10AF2800ADAB0008C1AF000849A80008E80F002031
:10AF3800A1EE00084010002015A700082DA7000862
:10AF480049B118B1012804D000207047034B0B60A9
:10AF5800FAE7034BFBE74FF0FF30704700040001AE
:10AF68000100010208B503F0ABF8002814BF6FF028
:10AF78000100002008BD08B502F084F9002814BFBC
:10AF88006FF00100002008BD10B504468AB018B95A
:10AF98004FF0FF300AB010BD212368468DF800300D
:10AFA80002F000FA0028F3D1024A9DF90430237018
:10AFB8005371EFE7141000202DE9F0412F4D304F69
:10AFC80000232B7043786B703B689B6A8AB00446F9
:10AFD8000BB128469847DFF8AC80002658F8043BA8
:10AFE8001BB11B6A0BB1204698470136F3B2052BFB
:10AFF80076B2F3D12378052B2FD00B2B35D0012B2C
:10B0080025D1214C062368468DF8003002F0CAF994
:10B018000199E07905F038FE10B91C4B019A5A6184
:10B028001B48FFF70BFE1B48FFF7AEFF6B788BB989
:10B03800A371194B5878FFF75BFD3B685B6A0BB14E
:10B04800114898476B7813B9E07905F0AFFE0AB05C
:10B05800BDE8F081FF23A371EFE7104B01225A747A
:10B06800227A9A74627ADA74F1E76378002BEED068
:10B078000AB0BDE8F041FFF7CFBB00BF440800208D
:10B08800101000202C100020600800205010002014
:10B0980064080020650800201410002030080020F3
:10B0A80030B58BB0FFF767FF0446F0B903F0FCFE3C
:10B0B800831C1DD0F8B9134D2B685B69DBB12723BE
:10B0C80068468DF8003002F06DF92B6801985B69CD
:10B0D8004FF4B961984703F0F9FE78B92CB9094BD8
:10B0E8001B68DB690BB10120984720460BB030BDC7
:10B0F8006FF00704EFE74FF0FF34ECE74FF0FF3451
:10B10800F3E700BF10100020014B1878704700BF0C
:10B1180084100020014B5878704700BF841000202D
:10B1280070470000044B9A7A0AB101225A70034B07
:10B138005B6903B118477047841000206C08002031
:10B1480073B5224C6378002B33D008F03BF966685E
:10B158000546FFF7D3FB0644AE4214D2A37A93B157
:10B16800E0228DF800208DF80130217AE368019300
:10B1780001226846FFF7F2FB08B1073010D100231F
:10B188006370A372656094F83430EBB1002384F8DF
:10B1980034300F4B5B6BBBB102B0BDE87040184751
:10B1A80040F2DC510B4808F0D9F90A4808F09CF93C
:10B1B800E8E794F83520002AE5D094F8360084F8BA
:10B1C8003530FFF795FCDEE702B070BD8410002033
:10B1D8006C0800206810002037B5104D104CC8B11D
:10B1E800C1B16272012300222860E16023700D481A
:10B1F8000D4B00924FF0FF3108F0CAF800250B48BC
:10B2080025822022294605F01DFE6570A574A586B5
:10B2180003B030BD00232B602370EFE780100020BF
:10B2280084100020681000202DB10008981000201C
:10B238002DE9F0478E4C23788CB0002B56D0C2787D
:10B248000AB9837B13B1238A01332382437B002B02
:10B258004CD0E02A4AD10023A372876897F800806F
:10B26800B8F1220F27D8B8F1220F30D8DFE818F04C
:10B278004100FB0052005A0061006E0075008E000C
:10B288009D00B400C7002F002F002F002F002F00B3
:10B298002F002F002F002F002F002F002F002F002E
:10B2A8002F002F002F002F002F002F002F002F001E
:10B2B800C900D000D400B8F17E0F00F0CC80B8F1FE
:10B2C8007F0F00F0DF80B8F17D0F00F0AB80A57A2A
:10B2D800002D00F05B81674C637A3BB94FF47A71BB
:10B2E800204608F03BF9204608F0FEF80CB0BDE80F
:10B2F800F087E36801220021A2721970A37AE1683D
:10B308009818A0720620C854A37AE1689818A07209
:10B31800CA54DCE7584B9B6A002BD8D00121022085
:10B328009847D4E77B7884F83630012384F83530A1
:10B33800CDE704238DF804307B78003B18BF012348
:10B3480001A88DF8083002F053F9C0E77878003882
:10B3580018BF012002F098FEB9E7484E0FCE01ADA4
:10B368000FC50FCE0FC596E8070085E807007B7864
:10B378000A2BACD8424A12685268002AA7D00CA9F6
:10B3880001EB830353F82C0C9047A0E77878431E11
:10B39800012B9CD83A4B01381B6818BF012020723A
:10B3A8009B68002B93D0984791E7E2680123082116
:10B3B800A3721170627A057BA17AAA4228BF2A4635
:10B3C800934284D285685A1CEB5CE56801334E1CB5
:10B3D800A6726B54D3B2EDE7E3680122A272092288
:10B3E8001A70A37AE268218A581CA072D154A27AF2
:10B3F800238AE1681B0A501CA0728B5467E72382DA
:10B4080065E705238DF8043001A802F077FB5EE7B5
:10B41800194BDB6A98475AE7194B78781B686075AF
:10B42800DB68BEE7037B072B7FF451AF06238DF85B
:10B438000430B7F80130ADF808307B793A791B044D
:10B4480043EA0223FA781343642253430393BB79F4
:10B458008DF81030D8E73B2201A88DF804208DF82C
:10B46800083002F0C5F8012384F834302FE700BF14
:10B4780084100020681000206C0800203C3A010865
:10B48800801000202A2301A88DF8043001F08AFFDB
:10B4980094F80A90E6689DF808009DF809509DF810
:10B4A8000A709DF80BC09DF80D309DF80E209DF890
:10B4B8000F109DF80CE009F1010A84F80AA006F8BB
:10B4C8000980354E94F80A903668D4F80C8009F152
:10B4D800010A84F80AA096F803A008F809A094F8CD
:10B4E8000A90D4F80C8009F1010A84F80AA096F8A9
:10B4F80002A008F809A094F80A90D4F80C8009F181
:10B50800010A84F80AA096F801A008F809A094F89E
:10B518000A9009F1010A84F80AA096F80080E66802
:10B5280006F8098094F80A80E66808F1010984F8A9
:10B538000A9006F808C094F80AC0E6680CF10108F9
:10B5480084F80A8006F80C70A77AE66807F1010CFF
:10B5580084F80AC0F555A57AE6686F1CA77270557D
:10B56800A07AE568461CA6722954A17AE0684D1CA9
:10B57800A5724254A27AE168501CA0728B54A37A37
:10B58800E268591CA17202F803E0A0E6034807F03C
:10B598005DFF6570AAE600BF8010002068100020DB
:10B5A80070470000004870476C0800200020704772
:10B5B8004FF0FF3070470000044B054A93F81831EC
:10B5C800022B18BF062382F89034704728170020F2
:10B5D800EC1C0020034BD3F8483313B15B6903B16B
:10B5E80018477047EC1C0020034A137843F0040303
:10B5F8001370FFF7EFBF00BFD01000201FB50A4B34
:10B608008DF8090093F87C208DF80A2093F88C2097
:10B6180093F848000D3202A98DF8082003F064FC65
:10B62800C0B205B05DF804FB2817002008B507482C
:10B6380007F00CFF064B93F81A2412B1012283F885
:10B648001924BDE80840FFF7C5BF00BFEC20002063
:10B65800EC1C002010B50C4CD4F8403343F08003A8
:10B66800C4F8403394F81A3413B10020FFF7DEFF12
:10B6780094F8913423F0120343F0120384F89134C0
:10B68800BDE81040FFF798BFEC1C00202DE9F04101
:10B69800DFF8AC8098F81831022B06460D4602D028
:10B6A800284BDB6A984702F0A6FD044628B1022021
:10B6B80002F097FD002002F099FD98F81831012B4F
:10B6C80017D102F09AFD074630B1002002F08AFD3A
:10B6D800002002F08CFD3C4602F091FD48B10020AC
:10B6E80002F081FD002002F083FDBDE8F041FFF784
:10B6F80063BF002CF9D1144C94F8902494F81A34B0
:10B70800BAB90BB184F84164304602F017FFD8F893
:10B718002C0007F061FED4F8B4339842E5D30B4807
:10B7280007F094FE94F8913443F0100384F89134B0
:10B73800DBE70BB184F84154284602F0FFFEF1E73D
:10B7480028170020CC430108EC1C0020842000208E
:10B75800074A10B5137843F002031370FFF73AFF56
:10B76800BDE81040034B01220021022007F042BB34
:10B77800D0100020993C0108074A10B5137843F00F
:10B7880008031370FFF726FFBDE81040034B0122A2
:10B798000021022007F02EBBD0100020A93C010890
:10B7A8002DE9F0410F4616461D46804607F00AFE71
:10B7B8000B4A0C4C1378278123F0110343F0110333
:10B7C800C4E90008137066812573FFF703FFBDE81D
:10B7D800F041054B01220021022007F00BBB00BFFE
:10B7E800D0100020BC100020B93C010813B507F0A8
:10B7F800E9FD0D4B6C461860204607F037FD94E8CC
:10B8080003000A4A0A4B83E80300137843F0200335
:10B818001370FFF7DFFE074B01220021022002B060
:10B82800BDE8104007F0E6BACC100020D010002088
:10B8380024200020C63C01082DE9F04192B00646BC
:10B8480002F0D9FC002840F05881AD4D95F8183128
:10B85800012B09D02B6BAB4C93B194F80431BBB1DD
:10B86800042B6FD0032003E002F0C7FC18B10F20AF
:10B8780012B0BDE8F08102F0C2FC0028EAD0F6E779
:10B88800B5F82031D4F81C24013B53432B63E4E77B
:10B898009D4803F060FA002840F0128194F80C31BA
:10B8A80023802B6B0C930DF1180895F839308DF81F
:10B8B8003830404695F81C318DF83A3007F0FCFCDA
:10B8C800D5F82831009302AF98E80600D5F824315E
:10B8D800384607F088FC97E803000FAB83E80300BD
:10B8E800EB6A0D9300238DF844302388ADF8463079
:10B8F80095F8303101228DF839201BB98DF8442094
:10B908008DF83930814B0093814B95F84800A3F1AD
:10B9180079020CA903F05DFBC0B10B28A8D1D4F8BB
:10B92800941499B1002EA3D0D4F84033794843F049
:10B938002003C4F8403307F011FE764807F0D4FD21
:10B94800002095E7704803F03AFAA4E795F84870A4
:10B9580095F9693095F9392095F87D106E4E38467D
:10B9680003F044FB009641B2EB6C95F85020384642
:10B97800183603F0DFFA0096EB6C95F8502095F92D
:10B98800701095F8480003F0D5FAD4F8C413AB6DDD
:10B99800D4F8DC230B44C4F8B033EB6D1344C4F87B
:10B9A800B43394F80431042B07D02B6E0B44C4F83D
:10B9B800B0336B6E1344C4F8B4330023089395F87E
:10B9C8003031002B40D100238DF8133095F83930F1
:10B9D8008DF8213095F838308DF82230D5F8803040
:10B9E8000993D5F884300A932388ADF82C3095F85C
:10B9F800303194F81B648DF82E3095F84800474B89
:10BA08008DF820600DF1130208A903F0A7FA0123AD
:10BA180084F8413495F8393084F842349DF813306D
:10BA280084F84334D4F81C34C4F85064C4F8483457
:10BA3800C4F8583402F0E5FBC8B1D4F81C0402F08D
:10BA4800F2FBA0B1102013E708A802F0A7FC60B928
:10BA580095F9390094F837629DF82070FFF7CEFD0C
:10BA68003E44B042AFD2082002E7132000E795F821
:10BA78001831012B01D102F0D8FB02F0C5FB0023DD
:10BA8800059394F8043195F9395094F81B649BB1E7
:10BA9800042B7FF4E7AE05A802F0B4FE58BB94F877
:10BAA800183413B1059B013B0593174B0598324693
:10BAB800E9B202F00DFF02E0134802F0DDFE08B122
:10BAC8001120D5E6D4F8403394F80C11218043F0C6
:10BAD8000203C4F8403394F8183411480133DBB238
:10BAE80084F8183484F845340E4B00259B6AC4F852
:10BAF8009854984724E71220BAE60E20B8E600BF0B
:10BB080028170020EC1C0020F41D002058170020E6
:10BB18008021002054200020A4200020082100209B
:10BB2800EE1C0020CC43010873B5134D134E00964C
:10BB3800EB6C95F8502095F9781095F8480003F0CB
:10BB4800F9F995F83031337595F8480040F201233A
:10BB580006F13C023146738203F0F8F950B196F8C9
:10BB68003C3086F88230064B00205B6B9847F37CAC
:10BB780086F8A83002B070BD28170020D420002015
:10BB8800CC430108F8B5324C94F81831012B05461E
:10BB98000ED0022B4ED0002B57D138B9D4E91B0157
:10BBA80004F1740383E803000020F8BD012806D1DE
:10BBB80002F02CFB0028F8D184F81851F5E7022888
:10BBC80043D1244E84F8180106F5747CBCE80F00B4
:10BBD80006F57A770FC79CE8030094F8E92094F8F3
:10BBE800003187E8030086F8FB53D2B1022B18D145
:10BBF800D4F804316367C6F8EC3394F87D3094F8D0
:10BC0800082186F8F83394F88C3084F8782086F880
:10BC1800F93396F81B2486F8E82340F20133A6F896
:10BC2800FA33002386F81A340B4BDB6A9847FFF780
:10BC38007BFFB9E748B9074B84F81801062283F857
:10BC48009024054BDB6A9847AEE70320ADE700BFB9
:10BC580028170020EC1C0020CC430108F0B5504CFC
:10BC6800504EB4F8DC202287D4E92D0194F8B12095
:10BC780084F8692004F16C0282E80300D4E92F01FA
:10BC880004F1740282E80300B4F8C420A4F87C200C
:10BC980091B0D4F8CC20D4F8C810C4F8842000257A
:10BCA800D4F8D020C4F888200123A4F82031C4F89F
:10BCB800801084F83051A56284F81B5184F83A50FA
:10BCC80084F81D5184F81E51C4F83451C6F89854AC
:10BCD800A6F8185486F81A54A4F838518DF8183074
:10BCE80004F50973039304F50A7394F84800049360
:10BCF80003A92D4B84F84551C4E94F55A4F8465182
:10BD0800059303F0FFF8E36EC6F8D43394F87D305A
:10BD180086F8E03394F88C3086F8E1334FF480737A
:10BD2800A6F8E23386F8D05394F8303186F8E43335
:10BD380006F574770FCF06F57A740FC497E80300F9
:10BD480040F2012384E80300A6F8FA33D6F8483312
:10BD580086F81B54CDE901551BB15A685B690192FD
:10BD68000293124B0793A3F148020892A3F114021D
:10BD780009920F4A0B9229330A93A2F19C030C9360
:10BD8800A2F198030D93131D0E9301A902F14C0320
:10BD980007A802F599620F9302F022FA11B0F0BDDC
:10BDA80028170020EC1C0020D4100020542100206B
:10BDB8000C180020F8B50D4F0D4E0C4607F046FB49
:10BDC8003B6B98470B4A96F84800214603F0BEF8AB
:10BDD80050B1094D706D95F8243485F86A347B6B41
:10BDE8009847E37C85F89034F8BD00BFCC43010840
:10BDF8002817002010210020EC1C00200F4890F884
:10BE08001B3480F8B8330E4B93F8692080F8BB23B5
:10BE180093F87D2080F8C82393F88C2080F8C923F4
:10BE280093F8303180F8CC330022A0F8CA2300F50B
:10BE38006E7100F56070FFF7BDBF00BFEC1C0020FD
:10BE480028170020114890F89034EBB190F81B3473
:10BE580080F8D0330E4BDA6EC0F8D42393F87D20E7
:10BE680080F8E02393F88C2080F8E12393F83031B0
:10BE780080F8E4334FF48072A0F8E22300F574717F
:10BE880000F56670FFF796BF704700BFEC1C0020F6
:10BE98002817002070B5344C2421204604F0D4FF24
:10BEA800636A984218BF60624FF01C012F4814BFA4
:10BEB8000125002504F0C8FF636C984218BF606430
:10BEC8004FF480712A4818BF45F0020504F0BCFF02
:10BED800D4F84831984218BFC4F848014FF0D4014B
:10BEE800244818BF45F0040504F0AEFFD4F820320A
:10BEF800984218BFC4F820024FF000011E4818BF2E
:10BF080045F0080504F0A0FFD4F82432984218BF81
:10BF1800C4F824024FF46071184818BF45F01005A2
:10BF280004F092FFD4F8A835984218BFC4F8A805C1
:10BF38004FF01401124818BF45F0200504F084FFA3
:10BF4800D4F8C03598420F4B18BFC4F8C005D3F8D1
:10BF5800483318BF45F040052BB11B691BB1284673
:10BF6800BDE87040184770BD281700205017002002
:10BF780070170020741800204C1900205019002058
:10BF8800D41C0020EC1C00202DE9F04F8FB04FF09E
:10BF98000009012B06460F4690468DF80D90ADF826
:10BFA800109002D84C46BC4202D30FB0BDE8F08FC7
:10BFB800305D02F033FA2044B842F6DC335D651C8C
:10BFC800023BEDB2112BF0D801A252F823F000BFCA
:10BFD80021C000084BC0000849C1000871C1000811
:10BFE800EFC1000815C200087BC20008A3C2000800
:10BFF80029C30008B3BF0008B3BF00087DC3000809
:10C00800B3BF0008B3BF000825C400084DC400082A
:10C0180085C40008B9C40008052002F0A7FA70B169
:10C028000521002002F068FA725DBA4BE51C023463
:10C03800E4B283F85C24325D83F85D24EDB22C46CB
:10C04800B1E700238DF80E308DF80F308DF81430DD
:10C058008DF81830B9F1000F6DD1AF4C4FF00509CC
:10C0680094F87C208DF831206B1E94F839208DF8D7
:10C078003320334494F838200B938DF8342094F807
:10C088001A3194F868208DF83520D4F82C218DF8D1
:10C0980032300A9273B37B1C5B1BDBB28DF83030F5
:10C0A80006AB019305AB009394F848000DF10F031C
:10C0B8000DF10E020AA902F05DFF8DF80D0000F0E7
:10C0C8000700072813D194F939209DF90E3084F818
:10C0D80039309A429DF80F3084F83830B8BF0122C1
:10C0E8009DF81430B8BF84F81D2184F868304FF0EB
:10C0F800000A09E00523D1E701220DF10D01032013
:10C1080002F0A4F80AF1010A5FFA8AF29DF81830E1
:10C11800B3FBF9F19142EFD82B44DDB26B1EDBB2D1
:10C128009F420BD9F25C032A9AD0AF4288BF1D46C2
:10C138004FF0010983E70534E5B2F9E71D46F7E753
:10C14800735D754903F00F03012281F81B31023436
:10C1580002FA03F3A1F82031E4B2002204A9042072
:10C1680002F074F825466AE707238DF80D30735DF1
:10C17800C3F3021203F00F038DF82830E31CDBB27F
:10C188008DF82920F25C231DDBB2651DF35C0234B7
:10C19800E4B21B0443EA0223325D5F4C134364227A
:10C1A800534394F848000B930AA902F0F2FE00F0FA
:10C1B8000703072BEDB28DF80D000CD19DF8283040
:10C1C80084F8703084F878300B9BE36663679DF8D9
:10C1D800293084F869308DF81000012204A905205F
:10C1E80002F034F82BE74B4BD3F8483363B11B68A4
:10C1F80053B1984708F03F038DF810008DF81130BF
:10C20800022204A90620EBE7FF20F3E703238DF8B9
:10C218000D30735D8DF81C300AAB0693E31CDBB25E
:10C22800A51DF25C231DDBB206A9F35C1B0443EADF
:10C238000223A21CD2B20534B25C134364225343D6
:10C24800E4B20A9300230B93335D8DF83030324B00
:10C2580093F8480002F0A3FEC3B20028EDB28DF8AF
:10C268000D30FFF6ECAE8DF81030012204A907203E
:10C27800B6E7735D03F00F03012B4FF47A7238BFF2
:10C2880001235343244A0234936503F57A73D36533
:10C29800E4B2002204A9082062E7735D1E4DC3F3CF
:10C2A80040128DF8152095F84800C3F3001205A92F
:10C2B80003F00F038DF814208DF8163002F075FE88
:10C2C80002340130E4B23FF44DAFBDF81430134AE4
:10C2D800A5F87C309DF816309DF814A0D05CF5F7D1
:10C2E80095FB0223C5F880000AA995F848008DF847
:10C2F80028308DF82AA002F0F7FD95F9393006901C
:10C3080040B29842B8BF184685F83900002204A9FF
:10C31800092025E7EC1C002028170020D33C010841
:10C3280003238DF80D30735D8DF82830E31CDBB2E4
:10C33800651DF25C231DDBB20234F35CE4B21B041E
:10C3480043EA0223325D1343642253430B93644B45
:10C358000AA993F8480002F02EFEC3B20028EDB2F5
:10C368008DF80D30FFF66BAE8DF81030012204A960
:10C378000A2035E7092002F0F9F8DFF868B100284B
:10C3880049D00921002002F0B7F80023ADF81E308B
:10C39800A31CDBB2F25CE31CDBB216F803A0735DEE
:10C3A8004FEA0A4A4AEA022A4AEA030A231DDBB28A
:10C3B800A51D0534F35CE4B24AEA036A335D4FF421
:10C3C8007A7253430AAC1B122046ADF81C3006F0B3
:10C3D8004DFF454B53440693DBF83C3300930DF176
:10C3E800180A9AE80600DBF8383308A806F0FBFEBE
:10C3F800099B009394E80600089B504606F0D8FE77
:10C408009AE8030006F00AFF01F00AFF0123EDB2E3
:10C418008BF8383413E68BF8380410E60C2002F059
:10C42800A5F800283FF40BAE0C21002002F064F8B8
:10C438002C4B93F89034043B012B7FF600AE01F0AF
:10C44800EBFEFCE5A31CDBB2725DF15CE31CDBB226
:10C45800651DF35C0434E4B21B04305D43EA012338
:10C4680013436421594300F00F0001F0D6FEEDB2EA
:10C478008DF81000012204A91120B1E60D2002F068
:10C4880075F800283FF4DBAD0D21002002F034F8E8
:10C49800A31CDBB2154AF05C735D1268251D0334DA
:10C4A800E4B243EA0020315DEDB201F0B8FEC6E522
:10C4B800725DA31C251D0334DBB2E4B2F15C335D6D
:10C4C8001B0443EA012313436420584301F0A9FEE7
:10C4D800EDB28DF81000012204A9132080E600BFF8
:10C4E80028170020EC1C0020803DD512BC1000202D
:10C4F8000E4B93F89124920703D593F88F24012AC1
:10C5080008D90B4991F81A2122B18A6A501C18BF20
:10C5180001328A620022A3F8182483F81A24D3F877
:10C52800402322F00202C3F840237047EC1C00208D
:10C538002817002070B5184C1848194D06F086FFCA
:10C54800D4F84033D4F89804D5F8906023F0200349
:10C55800C4F8403338B106F03FFF864203D20023C7
:10C5680085F83A3070BD0120FFF766F90028F9D048
:10C578000B28F7D095F8393084F84234092094F81C
:10C58800183484F8453484F8410401F0D7FFBDE835
:10C598007040FFF7ADBF00BFEC1C00205420002006
:10C5A80028170020094BD3F84023012A0AD008494C
:10C5B8000978C90708D43AB993F89204013818BF22
:10C5C800012070470020704701207047EC1C0020B4
:10C5D800D0100020034BD3F84003431E5842584163
:10C5E800704700BFEC1C00202DE9F04FA9B0EFF315
:10C5F800108272B6DFF8F0B20021DBF80030CBF819
:10C60800001082F31088B94C002B00F0E180DAB2F8
:10C618009B06039264D5B64D95F81831022B02D0CB
:10C62800B44BDB6A9847EFF3108872B6B24F06F046
:10C63800C9FE3E68D4F8B013361A3144AF4806F044
:10C648008DFFAE4806F050FFD4F8B413AC4831441F
:10C6580006F084FFAA4806F047FF88F3108894F88C
:10C668001A34002B00F06B81152312A995F84800A5
:10C678008DF8483002F038FCD4F8B4130F90014418
:10C68800A04806F06BFF9F4806F02EFF3B6894F821
:10C698001B24EB620DAF38468DF870201D9306F011
:10C6A8000BFED5F82831009306AE97E80600D5F8BA
:10C6B8002431304606F097FD96E803001FAB83E867
:10C6C8000300D4F81C341E9395F8303195F84800CF
:10C6D800003B18BF01231CA98DF8713002F00DFC36
:10C6E800039BDF0648D5824DDFF81CA2D5F8E4206D
:10C6F80004929BF80020BAF90A809AF90C90A4F8E1
:10C708008C84002363F300020A9384F84434A4F869
:10C71800223484F82534C4F82834A4F82C3484F856
:10C728002E34C4F8303484F82034C4F8343484F80F
:10C738003834C4F83C346F4B8BF8002094F89024BC
:10C74800DB6A84F88E9484F88F24DAF80470BAF8D7
:10C758000860984794F88F3413B9694806F076FE54
:10C768003146384601F045FD8346002800F0EA804E
:10C77800A4F87E8484F88094039B19071AD55C4B2F
:10C7880093F81831022B02D05A4BDB6A98470220E3
:10C79800FEF712FF84F8410401F0D0FE94F81A3431
:10C7A80013B1012384F8193494F8913443F0100339
:10C7B80084F89134039B5A0703D506210520FEF718
:10C7C80065FF039B9B0703D504210320FEF75EFF4B
:10C7D80001F02DFD94F89124D7065FD5002384F845
:10C7E8009234D4F840331E0644BF23F08203C4F8C1
:10C7F800403312F0050F00F0FB820B2001F0B6FE6B
:10C80800002800F0F58294F89134DD0700F1F082F9
:10C81800580740F10783D4F8403323F00203C4F8E3
:10C828004033D4F8402382BB94F8915415F00101A9
:10C838001EBF2B4662F3000384F8913494F89134B8
:10C848005E0744BF6FF3820384F89134012384F8B0
:10C85800923421B1D4F844332C481B6898476D07AB
:10C868000BD52B4801F08EFE01F0BCFE28B194F8E0
:10C87800913443F0040384F8913401F0C6FC94F831
:10C8880091346FF3041384F89134012384F89234BB
:10C8980094F8913443F0200384F8913494F8913457
:10C8A80018070AD56FF3C3031A4984F89134D4F8EA
:10C8B8004433A1F12400DB68984794F89134990730
:10C8C8000AD56FF34103134984F89134D4F84433FB
:10C8D800A1F16C005B68984794F89034022B1BD147
:10C8E800FFF722F918E000BFD0100020EC1C002050
:10C8F80028170020CC430108CC1000206C20002011
:10C9080084200020EC200020BC1000202C210020D6
:10C91800402100207821002094F891349A0640F1B3
:10C92800C4826FF3451384F89134D4F84033002B54
:10C9380040F0BB8229B0BDE8F04FFFF7ABBA84F8EE
:10C948004134A3E695F81831012B0CD101F055FCC0
:10C95800804668B1584601F045FC584601F047FC4E
:10C96800042384F88F347EB9012384F821344FE1FD
:10C9780001F045FC0028F6D0404601F034FC404662
:10C9880001F036FC0523ECE73B7805935B09013B96
:10C99800062B00F21782DFE813F007001502950056
:10C9A8001502920015020602102EDDD995F83031D5
:10C9B8001297F6B28DF84C60002BD5D11CA804F064
:10C9C80055F912AA1CA9FF2002F09EF89DF85830CC
:10C9D800C3F3030307468DF82C3095F8480095F803
:10C9E8007D308DF82D3007220BA902F090FA002F28
:10C9F8005DD100285BD09DF853309DF852201599E1
:10CA0800C5F8E4101B0443EA02239DF851200220D4
:10CA18001343C5F8E03004F037F99DF8583095F81D
:10CA2800480085F82E71C3F30212C3F3030385F897
:10CA3800703085F878309DF8593085F86920012BD9
:10CA480038BF01234FF47A725343AB651344EB6547
:10CA58000DF15A034FF001081093113E94F81B345E
:10CA68008DF83C300FA985F868808DF8446002F095
:10CA780056FA0223404685F8303101F077FD18B1A7
:10CA88004146384601F038FD94F88F34012B00F206
:10CA9800A78194F81A34002B40F09A8194F89134C5
:10CAA80043F0100384F89134FEF786FD64E6012014
:10CAB80001F05CFD0028E7D001210720E2E701230F
:10CAC80084F8203495F87D308DF82E3094F824348D
:10CAD8008DF82D3095F88C3095F848000D330BA95A
:10CAE8008DF82C3002F000FAA6F10D031BB2099064
:10CAF80023EAE37300B283423FF736AF0B2E7FF68B
:10CB080033AFBA4B25931CA8FF231C978DF874608C
:10CB18008DF8983002F0C4F8074600287FF424AF57
:10CB280095F81831012B13D101F067FB002872D05A
:10CB3800384601F057FB384601F059FB04239DF8AD
:10CB48007C101E9884F88F34C1F3001101F06EFB3D
:10CB58009DF87C301E99C4F8341413F00F0203D0EA
:10CB68009DF89000002862D19DF89800002861D0B7
:10CB7800002A7FF4F9AE9DF89020002A14BF4FF0E8
:10CB880003084FF0020800220A92D5F8EC2095F825
:10CB9800E900914251D100284FD0D5F80C1195F8F1
:10CBA800EAB009680A9195F81811022902D10321FF
:10CBB80084F88F14B8F1030F7FF4D6AE13F0600F2A
:10CBC8007FF4D2AE0492012795F82E31BBF1000F05
:10CBD80036D0BBF1010F13D1012B33D16FF0090609
:10CBE80046FA08F606F00106C6F10206F6B2BDF8E6
:10CBF8007E100AAA304601F011FE38B3072823D068
:10CC0800012384F821340A9BC4F83034C4F86C3406
:10CC1800FEF720FDB0E501F0F2FA002898D038467A
:10CC280001F0E1FA384601F0E3FA052387E74FF00F
:10CC38000008A8E74FF00108A5E74FF0010BC3E78C
:10CC48000426D4E70326D2E70823DAE71CAB0093CF
:10CC580004990A9B3246584601F0A2FE20B10228E8
:10CC680014BF0B230A2380E60A9BC4F83034C4F8A7
:10CC78006C349DF87C3084F82104C3F3401384F8A5
:10CC88002E3484F8443494F88F3484F82274012BB9
:10CC98009EBF0122A86285F81E21012FC4F828042E
:10CCA80084F82C0484F8410438D1022284F8202422
:10CCB80095F83A20002A4AD19DF87C20D60646D419
:10CCC800012B94F840149DF87C2005D8012901D146
:10CCD800900601D501F04CFBB8F1020F94F88F349F
:10CCE80043D0B8F1030F0AD09DF87C10B8F1010FBA
:10CCF8004A4601F00F0120A83BD0FFF745F99DF8FF
:10CD0800903084F82334259BC4F828349DF8983053
:10CD180084F82C34012384F82D3430E0059A02F08D
:10CD2800E002A02A1BD195F82E11012285F83A209D
:10CD380009B927996963012B84F8202407D9D5F804
:10CD48009020C4F83C24DAF80020C4F8982495F818
:10CD58001821002AB4D1012284F82524B0E7002242
:10CD680085F83A2084F82024A6E79DF8981025989D
:10CD78004A46FFF709F99DF8903084F823349DF866
:10CD88009020E02A08D195F81F312BB984F8232484
:10CD9800C4F82834A4F82C3494F8913443F00203EE
:10CDA80084F8913470E6114D013EB2B2791C2846E0
:10CDB80004F034F80323A4F82034C4F8285484F881
:10CDC8002C64E9E7012384F82134FEF743FC5BE691
:10CDD80094F84434002B3FF461AE0020FEF726FCA3
:10CDE80094F88F34022B3FF45FAE57E6241F0020DF
:10CDF80094F89134590715D5012001F0B7FB60B1BB
:10CE0800012001F08BFB08B984F81804D4F84033EA
:10CE180023F00203C4F8403304E0062001F0A6FB27
:10CE28000028F3D194F89134DA077FF5FAAC94F836
:10CE380040240AB1032A18D11D4A94F8181492F80C
:10CE48006820914205D29B0723D594F88F34012B93
:10CE58001FD8184806F0FAFAD4F8403323F0200314
:10CE6800C4F84033FFF744FBDBE4012A11D194F8FE
:10CE78001924002A3FF4D5AC0D4A94F8181492F8F6
:10CE880068209142E5D29F0703D594F84434002BDB
:10CE9800DFD194F8913400206FF3041384F89134AF
:10CEA80084F81904FFF746FBBBE429B0BDE8F08F0E
:10CEB80028170020542000202DE9F04F89468DB016
:10CEC80090460746002800F08F81002900F08C81E9
:10CED8000368002B00F088814368002B00F08481F0
:10CEE8008368002B00F08081C368002B00F07C81F0
:10CEF800104601F0F5FF002800F07881BD4CBE4DCA
:10CF0800384601F0AFFA40F2C4520021204603F03F
:10CF180099FF40F21C520021284603F093FFB74BBB
:10CF2800C4F82C3104F50973089304F50A73002634
:10CF38004046099308A9B24B84F848800A9384F8BC
:10CF4800186184F88C608DF82C6001F0DBFF0F23EA
:10CF580006A994F848008DF8183001F0C5FF801B29
:10CF680018BF01204FF00A0B84F81C0106A994F899
:10CF780048008DF818B001F0B7FF4FF0060A84F8A2
:10CF8800DC0006A994F848008DF818A001F0ACFF61
:10CF9800102384F8DD0006A994F848008DF81830AD
:10CFA80001F0A2FF1123C4F89C0006A994F84800D8
:10CFB8008DF8183001F098FF1223C4F8A00006A9D4
:10CFC80094F848008DF8183001F08EFF1323C4F848
:10CFD800A40006A994F848008DF8183001F084FFE1
:10CFE8001423C4F8A80006A994F848008DF818304E
:10CFF80001F07AFF1623C4F8AC0006A994F848009B
:10D008008DF8183001F070FF172384F8B10006A9D5
:10D0180094F848008DF8183001F066FF18230DEBDE
:10D028000301C4F8B400C4F8BC0094F848008DF8B3
:10D03800183001F059FFC0B21D2384F8B80084F8F5
:10D04800C00006A994F848008DF8183001F04CFF8C
:10D058001E2384F8C40006A994F848008DF81830F7
:10D0680001F042FF1F2384F8C50006A994F8480080
:10D078008DF8183001F038FF2023C4F8C80006A93D
:10D0880094F848008DF8183001F02EFF0B23C4F8EF
:10D09800CC0006A994F848008DF8183001F024FF58
:10D0A8000C2306A9A4F8D00094F848008DF818308D
:10D0B80001F01AFFD4F89C306365D4F8A030A3655A
:10D0C800D4F8A430E365D4F8A83023664FF00108FB
:10D0D800D4F8AC300590A4F8D200636684F8B08028
:10D0E800C4F894B084F898A0C4F84CB084F850A060
:10D0F80084F8688084F81F81C5F84893FEF7AEFD70
:10D10800C5F84473C4E90B663E4B84F8198185F869
:10D118009164C5F8408332464FF0FF31009605F51B
:10D128005A7006F035F9384B009632464FF0FF3109
:10D1380005F5607006F02CF9344B009632464FF036
:10D14800FF3105F5667006F023F902AF304B009603
:10D1580032464FF0FF3105F5806006F019F9384680
:10D1680006F0AAF897E8030004F5927383E8030031
:10D17800284B294F1E60294BC5F84C33284BC5F85E
:10D188005433284BC5F85C33274BC5F85033274B2D
:10D19800C5F8583305F553703B68984704F5A670F1
:10D1A80003F080FB20B1112630460DB0BDE8F08FAA
:10D1B800204601F003FB0028F5D101F039F8B8B991
:10D1C8001B4801F04DFB06460028ECD17B699847C7
:10D1D80003F002FEBB6D94F819019847FB6A984763
:10D1E800012385F89234DFE70326DDE70926DBE72C
:10D1F8001326D9E728170020EC1C002000040001A2
:10D20800D41000203DC5000805BE00084DBE00082A
:10D2180035B60008D0100020CC430108F5B7000847
:10D22800A9B70008F1B5000881B7000859B7000888
:10D238001018002008B5034B0020C3F84003FEF780
:10D24800BBF908BDEC1C002010B5FFF7ABF90A4C80
:10D2580060B90A4B93F81831022B02D1084BDB6AEC
:10D2680098470123C4F84033002010BDD4F8400388
:10D27800013818BF0120F8E7EC1C0020281700200F
:10D28800CC43010838B5124C204606F0DFF804F10B
:10D29800180006F0DBF804F1300006F0D7F804F1C6
:10D2A800980006F0D3F800F0AFFF0A4B0025DB6AC0
:10D2B800984744F8285CFEF7EDFD0749074840F217
:10D2C800C45203F0ABFD012344F8283C284638BD7E
:10D2D80054200020CC4301082817002064110020A6
:10D2E80070B52E4B8AB0054693F8DD008DF809001D
:10D2F80093F8DC008DF80A0029489A6A90F8180417
:10D30800039200268DF80B0004960C46002940D0A5
:10D318000692D3F8882007921A8F93F81A118DF87D
:10D32800151052BAADF8202093F87C2093F84830B5
:10D338008DF8243003AB8DF822008DF8232000935C
:10D348000DF10A020DF10B030DF1090105A88DF885
:10D35800146000F0D7FE9DF90900FEF74FF96070E0
:10D3680004A801F01BF8B0B9049A0F2A0DD8637805
:10D378009A420AD81544AB42A3EB02012CBF002005
:10D3880001202170C0000AB070BD0023237008205E
:10D39800F9E70320F7E71320F5E700BF2817002077
:10D3A800EC1C00201FB50446002800F0108103780B
:10D3B800412B00F20781DFE813F0420049004D00DD
:10D3C8005100550059005E000501050105010501E0
:10D3D8000501050105010501650069006D0078007A
:10D3E8007F00820085008A0088008C0090009300EE
:10D3F800960099009C009F00AE00B200BA00B600EB
:10D40800BE00C100C500CE00CA00CC000501D20094
:10D4180005010501050105010501050105010501D4
:10D428000501050105010501050105010501DA00F0
:10D43800DE00E200E700EB00EF00F300FC00664BC3
:10D4480093F818312371002004B010BD624B93F893
:10D458003031F7E7406803F0C3FBF4E7406803F0B6
:10D4680005FCF0E75C4B93F81A31EBE75A4BD3F81D
:10D47800E0306360E7E7584B011D93F8300103F093
:10D488000DFCE0E7544B93F81931DBE7524B93F866
:10D498008C30D7E71C238DF808304F4B02A993F83E
:10D4A800480001F021FD6060CDE74C4B043493E85F
:10D4B800030084E80300C6E7494B0434F7E7494B07
:10D4C8000434F4E7484B0434F1E71A23E3E719235B
:10D4D800E1E7414B93F86830B4E73F4B5B6DC8E731
:10D4E8003D4B9B6DC5E73C4BDB6DC2E73A4B1B6E72
:10D4F800BFE7394B5B6EBCE702238DF80830364B2B
:10D5080002A993F87C2093F848008DF80A2001F0CE
:10D51800EBFC207197E7304B93F8DD3092E72E4B08
:10D5280093F839308EE72C4B93F8DC308AE72A4B96
:10D5380093F8383086E7284BDB6C9AE7264B93F84C
:10D5480050307FE7244BD3F8843063607BE7224B6D
:10D558008FE7264B8DE7204BD3F8CC30F5E71E4BF1
:10D56800D3F82C31436001F04DFDA0606BE71A4BF6
:10D57800D3F890307DE7184B93F81F3162E7164BCC
:10D58800B3F88830A3805EE7134BB3F88A30F9E725
:10D59800114BB3F8D030F5E70F4BB3F8D230F1E7C1
:10D5A8000D4B93F848200AB1062A12D1B3F8A035DA
:10D5B800E8E7094B93F848200AB1062A09D1D3F8BD
:10D5C800A43556E704B0BDE8104000F021BE0320A2
:10D5D8003AE7182038E700BF2817002094170020E2
:10D5E800DC1700209C170020E4170020641100209D
:10D5F8007FB5044610B9032004B070BDA34DD5F81B
:10D6080040339A0700F16F820278412A00F268825B
:10D61800DFE812F04200470055005B005F0064003D
:10D6280069007600810087008D00930099009F00B3
:10D63800A500AB00B5006602BA00DC00EF001601D9
:10D648003801290142014B014F01530157015B0188
:10D6580066025F01710199018701AB01B101B8014F
:10D66800BD01C201660228026602660266026602FF
:10D678006602660266026602660266026602660262
:10D688006602660266026602340239023E024302FC
:10D6980048024D0252025C020079FEF773FA30B17B
:10D6A800AAE70379022BA6D0794A82F8303195F897
:10D6B800913443F0200385F8913400209CE74068BA
:10D6C80003F080FA0028F2D095E7406803F0BEFA2C
:10D6D800F8E76F4B027983F81A21E8E76C4B426848
:10D6E800C3F8E020E3E76A4E416896F8300103F09A
:10D6F800CBFA00287FF47FAF6368C6F8E430D6E73A
:10D70800416800293FF477AF002001F0DDF90028D7
:10D71800CDD0112070E7416800293FF46CAF01209B
:10D72800F3E7416800293FF466AF0820EDE7416858
:10D7380000293FF460AF0920E7E7416800293FF47A
:10D748005AAF0C20E1E7416800293FF454AF0D209F
:10D75800DBE7416800293FF44EAF0E20D5E741686A
:10D7680000293FF448AF0F20CFE74A4C484B0079D7
:10D7780083F81901A36D9847E36A984797E7444BE4
:10D78800027983F88C2092E7414E037A8DF80430B1
:10D7980096F8480096F87D308DF80530072201A9E3
:10D7A80001F0B5FB00283FF426AF636896F84800FF
:10D7B8000193002201A901F0AAFB00283FF41BAF46
:10D7C8006C36D4E9010186E8030070E7304E037A2D
:10D7D8008DF8043096F8480096F87D308DF80530BD
:10D7E800072201A901F093FB00283FF404AFB436E7
:10D7F800E7E7274E037A8DF8043096F8480096F844
:10D808007D308DF80530072201A901F080FB002842
:10D818003FF4F1AED4E9010106F1740383E8030093
:10D8280096F81831022B7FF442AF96F83031002B6E
:10D838003FF43DAF174BDB6A9847FEF775F936E7BB
:10D84800134E037A8DF8043096F8480096F87D3028
:10D858008DF80530072201A901F059FB00283FF493
:10D86800CAAEBC36ADE74368029301238DF80C308D
:10D87800074B02A993F8480001F056FB00287FF4F3
:10D8880016AFB8E6436802930023EFE7EC1C0020CC
:10D8980028170020CC43010803795A1E0E2A3FF6A8
:10D8A800AAAE934A82F8683001E7914B42685A65FC
:10D8B800FDE68F4B42689A65F9E68D4B4268DA655A
:10D8C800F5E68B4B42681A66F1E6894B42685A6660
:10D8D800EDE6874C037994F848008DF80430062269
:10D8E80001A901F014FB00283FF485AE9DF804302F
:10D8F80084F8DD30DBE67E4C03798DF8043094F84B
:10D90800480094F87C308DF80630052201A901F012
:10D91800FEFA00283FF46FAE9DF8043084F83930E1
:10D92800C5E6734C037994F848008DF804300A2250
:10D9380001A901F0ECFA00283FF45DAE9DF804302F
:10D9480084F8DC30B3E66A4C037994F848008DF823
:10D958000430092201A901F0DAFA00283FF44BAE9D
:10D968009DF8043084F83830A1E6614B4268C3F86A
:10D978009420DA649BE65E4B027983F8982083F85A
:10D98800502094E65A4B4268C3F884208FE6584BDF
:10D998004268C3F8CC208AE6012B40F0A480554C9D
:10D9A8002421204603F050FA636A984201D01720D8
:10D9B80022E61C2104F1280003F046FA636C984221
:10D9C800F5D14FF4807104F1480003F03DFAD4F822
:10D9D80048319842EBD1D42104F5A67003F034FA0B
:10D9E800D4F820329842E2D1002104F5097003F0FE
:10D9F8002BFAD4F824329842D9D14FF4607104F547
:10DA08000A7003F021FAD4F8A8359842CFD114212E
:10DA180004F2AC5003F018FAD4F8C0359842C6D1D5
:10DA2800334E2146304640F2C45203F0F7F92046FF
:10DA380040F2C452002103F005FA95F81B3485F82A
:10DA4800E833736FC5F8EC3396F87D3085F8F83312
:10DA580040F20123A5F8FA33274B96F819019B6D7C
:10DA6800984724E68379012B3FF6C5AD204B4268E1
:10DA78004068C3F82C2100F0BDFE48E61C4B426804
:10DA8800C3F8902013E61A4B027983F81F210EE69B
:10DA9800174B8288A3F8882009E6154B8288A3F8DB
:10DAA8008A2004E6124B8288A3F8D020FFE5104BA9
:10DAB8008288A3F8D220FAE50D4B93F848200AB1E2
:10DAC800062A12D1A288A3F8A025F0E5084B93F8FE
:10DAD80048200AB1062A08D16268C3F8A425E6E5F9
:10DAE80000F098FBDBE5012086E5182084E500BFFF
:10DAF8002817002064110020CC4301082DE9F043C9
:10DB080087B00023ADF800300646002800F0EE800C
:10DB18000361FEF747FD20B10124204607B0BDE8A8
:10DB2800F08300F065FD0028F6D100F05BFD0146AA
:10DB380018B96F48142203F085F96E4D95F89134A1
:10DB4800012243F0040385F8552485F8913433788D
:10DB58008DF804300021013B8DF80520ADF8061042
:10DB68000C2B00F2BB80DFE803F007B9B9B9798262
:10DB7800B9B990B9AD9AA900D5F8407317F0200744
:10DB8800CAD196F80480B8F1020F46D1DFF868814F
:10DB98005A4CFEF763F896F9051098F848003A468B
:10DBA80001F00FFA88F83900B37988F83830384628
:10DBB80007238DF80530FDF7E5FFFF2304F5867090
:10DBC800A5F80C31C5F8084185F8047103F04EF842
:10DBD80004F58A7003F004F83846FDF72DFE044674
:10DBE800002839D096F9051098F84800012201F06C
:10DBF800E8F988F83900D5F894343361002C71D0ED
:10DC080000F0F0FC002888D195F8913485F81A04C2
:10DC180060F3820385F891347FE7B8F1010F4FF084
:10DC28000204E8D1DFF8D0908DF8144099F8480044
:10DC380089F81D7102A901F065F9337989F8303145
:10DC48008DF805708DF80680FDF7C4FC95F89134C1
:10DC580043F0100385F891340024CCE7002269468C
:10DC6800022000F0F3FA0028F6D01324C3E7244B6F
:10DC7800B288DB6B96F90C10B0689847D5F840333A
:10DC880043F00203C5F84033E6E702A90D2000F08F
:10DC980053FB0028E0D0002269460D20E1E7164B2F
:10DCA80093F81831D3B9347904F0070000F0ABFACF
:10DCB8008DF80040012269461020D2E7002269460B
:10DCC8001220CEE78DF8072000F08EFA044638B906
:10DCD80000F087FA204600F089FABDE702248AE7B7
:10DCE800012488E701A800F0D1FB16E7032414E714
:10DCF80040210020EC1C002028170020EE1C0020EA
:10DD0800CC4301082DE9F04F99B08046059118B928
:10DD1800032019B0BDE8F08F00230361FEF742FC31
:10DD28000446002840F0A58046460FCE0EAD0FC52C
:10DD38001422524898F800A0B8F80C7098F90EB060
:10DD48004F4E214603F07EF84E4B012283F84124C2
:10DD580096F83021022A25460BD196F81821022A76
:10DD680007D196F81E2122B9BAF1010F38BF4FF03A
:10DD7800010ABAF1010F2BD0BAF1030F2AD0BAF178
:10DD8800000F33D102229DF83C30DDF84090029319
:10DD980062F34715012496F87C108DF832100222A0
:10DDA8000CA996F848008DF8302001F09DF896F8F7
:10DDB8001A3196F830C196F81D1140B2002B63D085
:10DDC800BCF1010F57D1002955D1002C61D153E086
:10DDD8000422D8E70023DDF83C90BDF840709DF997
:10DDE80042B0029365F01F050124D4E74FF0000B01
:10DDF800D946CDF808B0CEE74FF0010084F81A04F0
:10DE0800D2E005F29A420BA900F0D4FA002800F0FB
:10DE180015811320049B33871A4B002283F81A2498
:10DE280023E105F29A452A460BA900F0C3FA002817
:10DE3800EFD10B9B84F82801C4F82C5184F83031B9
:10DE4800FCE0B9F1000F00F0F980002A00F0F6803C
:10DE58004946E01C02F0E2FF94F837320133238090
:10DE6800ECE01220D6E70220D4E70720D4E71320FD
:10DE7800D2E701204DE7FCB90220F6E02C21002072
:10DE880028170020EC1C0020002CF5D05845B8BFFE
:10DE9800584696F87C308DF82000052296F8480000
:10DEA8008DF8223008A901F032F800283FF430AF8D
:10DEB8009DF8203086F839306F4A704BD2F89804B4
:10DEC800D3F8904038B105F087FA6C4B84423CBFD8
:10DED800002283F83A20198F1A8F93F830010491A1
:10DEE800996A099152BA0028BFD093F81B0100B96A
:10DEF800186393F81801ADF85820013893F87C207E
:10DF080093F81A411491D0F1000BD3F888108DF8CA
:10DF18005B204BEB000B93F8482093F83A0093F8FA
:10DF280068308DF85A3009AB0093554B03904FF089
:10DF380001008DF84C0015918DF85C20A3F12F019C
:10DF4800A3F1300213A88DF84D4000F0DBF8039BD5
:10DF58004FEA0B1B4BEA431B00264BEA801B4BEA9C
:10DF6800C413B145444C039308BF37463A46494663
:10DF780004F59C70CDE90A669B46268084F81A64ED
:10DF880002F04CFFE9B2A570C5F34215FAB2042DB0
:10DF98003A4E039B84F837223FF42EAF072D3FF407
:10DFA80050AF022D7FF45FAF364D84F80D11042079
:10DFB800029984F80401FF2084F80C0184F82811E0
:10DFC80084F81431D6F8E410C4F8085105F59B73A9
:10DFD8000AA8C4F8101184F83021C4F82C3100F0D4
:10DFE80011FC00287FF43DAF0A9BA4F844040BA859
:10DFF800A4F81631C4F84C3400F0D0F900287FF4A6
:10E0080008AF0B9BD3B196F93900FDF7F7FA94F8EE
:10E018003732002B3FF405AF0B9B0F2B3FF6F1AEC9
:10E0280005F58B720BA90F2000F0C4F900287FF4C6
:10E03800F0AE0B9B63F3030B84F814B10598FDF75E
:10E04800FBFB00287FF4E6AE099B86F83A00B36232
:10E0580000F080F900287FF40AAF94F8913484F82E
:10E0680040A443F0010384F89134034BD3F894346B
:10E07800C8F810304DE600BFEC1C0020281700201F
:10E0880090170020EE1C002037B50B4D8DF80400CA
:10E0980004460F2295F8480001A900F038FF40B166
:10E0A800064A85F81C4192F8913443F0200382F81F
:10E0B800913403B030BD00BF28170020EC1C0020AD
:10E0C80010B5FFF7C1F8044688B90A4805F0BEF94B
:10E0D800094805F0BBF9094805F0B8F900F094F8CB
:10E0E800FDF7BCFD064BDB6A9847204610BD0124AE
:10E0F800FBE700BF542000206C2000208420002073
:10E10800CC4301082DE9F04F8BB047780093149B5E
:10E1180090F90C8090F90D6090F80EB08A4641682D
:10E12800196004469146002F58D002238DF810300C
:10E1380004A9C37B007C8DF8123000F0D5FEB4F83A
:10E1480008C0618943B26068984545466144B8BFD4
:10E158001D46604534BF00270127884209D30A219C
:10E168008DF81010207C019304A900F0BDFE019BDE
:10E1780046B2B4F808C0608961680CEB400E71457E
:10E1880019D3A1EB0C01B1FBF0FC00FB1C1191B9F8
:10E19800984503DC2378CBB94FF0010B21238DF888
:10E1A8001030207CE37B8DF8115004A98DF81230D3
:10E1B80000F09AFE45B2009B8AF80050384689F86C
:10E1C800006083F800B00BB0BDE8F08F0223207C1C
:10E1D8008DF8243006A900F095FEDDE74546EAE70C
:10E1E8007047704770477047002070477047704706
:10E1F80070470020704700207047002070470020BB
:10E20800704700207047704770477047022070477A
:10E2180002207047022070477047002070477047FF
:10E22800704700207047002070477047704770475C
:10E2380010B5054C4FF403722046002102F002FE8F
:10E248000020C4E9000010BD082200202DE9F84391
:10E258008146904600293CD01F4C2023224604F1D9
:10E26800100012F8017F6FBB8242FAD11B4E33684F
:10E27800013403B93460736803B11C60002525605C
:10E28800C4F8088074601FFA88F284F80490601D4E
:10E2980002F0C4FDB9F1110F4FF0000398BF104D03
:10E2A8006373D6F8083298BF25FA09F503F101031C
:10E2B80098BF05F0010543442573C6F8083238466F
:10E2C800BDE8F883013B13F0FF030446C6D10227DB
:10E2D800F5E70127F3E700BF0F22002008220020FE
:10E2E8002007020010B518B3124A1368984204D1E7
:10E2F80003681360002305E00B46002BFAD0196869
:10E308008842F9D15168884208BF53600BB101684F
:10E318001960D2F808328168013B00245B1A046056
:10E328002146C2F80832102202F08CFD204610BDAA
:10E338000120FCE708220020054B1B6813B11A795D
:10E348008242FAD1002B0B600CBF032000207047DB
:10E358000822002010B5054B186800B910BD037BD2
:10E3680004680BB9FFF7BEFF2046F6E70822002035
:10E3780038B5084B084C186800B938BD03790568EA
:10E38800112B05D824FA03F3DB0701D5FFF7AAFF01
:10E398002846F1E7082200202007020028B1044B94
:10E3A800D3F808320360002070470120704700BF8F
:10E3B800082200202DE9F04107460E46154642B3D3
:10E3C80039B3154B1C6800232CB93046FFF7E6FF1C
:10E3D8000020BDE8F081A268F91A0132914215D3F4
:10E3E8002279EA54581C22895FFA80F8611D55FA8F
:10E3F80080F002F013FDA368246898445FFA88F35C
:10E40800E2E720462568FFF76DFF2C46002CF8D17F
:10E41800DBE70120DDE700BF082200200238C0B298
:10E4280011289ABF014B185C00207047E33C010893
:10E4380030B50B4B93F820200446084672B10021F2
:10E448001C330578A54208D001319842CDB214BFDB
:10E4580004301038AA42F4D8002030BD1046FCE73A
:10E468001424002010B5084C00232060142204F165
:10E478000C00FF2184F82030C4E9010002F0E2FC1E
:10E48800012384F8213010BD1424002010B50E4A51
:10E4980092F82010042915D8936804781C704478E1
:10E4A8005C70C478807898700131DC7082F8201034
:10E4B80002F11C018B4214BF043302F10C03936078
:10E4C800012010BD0020FCE714240020094B93F81C
:10E4D800200068B15A6803F11C018A4200F1FF303C
:10E4E80014BF043203F10C0283F820005A600120A3
:10E4F800704700BF1424002010B5074B93F8202064
:10E508000446084632B15968FFF792FF10B101235B
:10E518004470837010BD00BF1424002008B5064B5A
:10E5280093F820202AB15968FFF782FF08B1407894
:10E5380008BD0120FCE700BF1424002030B50A4ABA
:10E5480092F82010536882F8210061B19168012483
:10E558001C32DD78587005B99C70934214BF04339F
:10E56800103B9942F5D130BD1424002008B5044B66
:10E578005968FFF75DFF003818BF012008BD00BFCC
:10E5880014240020F7B50422154E044600210DEB93
:10E59800020096F8207002F055FC0025EBB29F426D
:10E5A80001D803B0F0BD7368197821705A78627089
:10E5B800987838B1336820469B689847FFF786FFFC
:10E5C8000135EBE7DB788DF804108DF805208DF820
:10E5D8000730FFF77BFF01A8FFF758FFF0E700BF00
:10E5E80014240020014B93F82000704714240020C5
:10E5F800034B93F82000042894BF002001207047A3
:10E60800142400201FB50024CDE90244C41F8DF84E
:10E6180000408DF801100C0AADF80420090C120C0A
:10E628008DF803108DF806208DF8073002461B0A76
:10E63800012168468DF802408DF8083002F05DFA35
:10E64800002818BF0E2004B010BD2DE9F04188B095
:10E6580090460D460F9A0746002847D0002401210E
:10E66800CDE904448DF810109DF838108DF8151078
:10E67800ADF81630190CCDE900441B0ECDE9024463
:10E688008DF81930ADF81A20130C120E07948DF876
:10E6980018108DF81C308DF81D20E3B21E01002DD6
:10E6A800F6B203DC002008B0BDE8F0810133102188
:10E6B8008DF81F3042466B460DEB010002F0B3F9AE
:10E6C8000346A8B9102D28463E44A8BF1020694625
:10E6D800327811F801CB013382EA0C02984206F82D
:10E6E800012BF5DC103D2DB20134D6E70920DAE71D
:10E6F8000E20D8E70138032815D8DFE800F0020813
:10E708000C100A4B1B681B690B6000207047074BF5
:10E718001B685B69F8E7054B1B689B69F4E7034BCB
:10E728001B68DB69F0E70520704700BF382400202C
:10E738002DE9F041C4B00C464A9E17461D46804656
:10E74800B8B3B1F5807F36D84FF488720021684697
:10E7580002F078FB492300934FF48073ADF804303E
:10E768002B0C8DF80830330CADF80650ADF80A6064
:10E778008DF80C3022460023414604A82D0E360E93
:10E788008DF80E308DF809508DF80D608DF80F401A
:10E7980002F044FB04F110014B9A3B4689B26846EB
:10E7A80002F02BF910B1012818BF0E2044B0BDE8C3
:10E7B800F0810920FAE70D20F8E7000010B590B1C4
:10E7C8000A4C28220021206002F03CFB2368084AFA
:10E7D8001A6000204FF0FF32C3E90302C3E90522A3
:10E7E800C3E9072210BD0820FCE700BF3824002039
:10E7F80000010101024B1B6818600020704700BF30
:10E808003824002030B1044B1B68DB6801330360F7
:10E8180000207047092070473824002013B50023D2
:10E828000C460193CAB101A9FFF764FF18B9019B0F
:10E83800591C02D1146002B010BD99B2611A0029A6
:10E8480001DD5C18F6E702D113600720F3E71B0C23
:10E858001B0403F580331C44ECE70920EBE70000B8
:10E8680028B1044B1B681C33436200207047092001
:10E87800704700BF382400201FB5044600B30023AA
:10E8880003A8039302F090F9104ABDF80C301268FF
:10E8980020469380E38200F05EFA98B904F11803E9
:10E8A800009321680123132202F09CF860B92046E6
:10E8B80000F051FA003818BF0120000104B010BD63
:10E8C8000920FBE71020F9E70E20F7E7382400209D
:10E8D800F0B5054687B01C4613B9092007B0F0BD4E
:10E8E8002E4E3368DB68834255D894F82020002ADE
:10E8F8000CBF08220922834205D3204600F05FFAA4
:10E9080068B11020EAE7002301900093A36894F807
:10E918002810606AFFF799FE0028EED0DEE7237919
:10E928002168B4F808C0A768043B9AB20029D4D07B
:10E93800B2F5807F2DD8ADF80EC08DF817304FEAAC
:10E94800174C04F12C033F0E8DF8117000932F0C17
:10E9580008234FF0490EADF80C008DF814708DF8AF
:10E9680016002F0E0DEB0300CDF808E08DF810C04F
:10E97800ADF812508DF8157002F034F808B10E2079
:10E98800ACE7204600F01BFA0028BAD13368DD60F6
:10E99800A4E70D20A2E70620A0E700BF3824002046
:10E9A8002DE9FF410A9D80460F4616461C46002D5C
:10E9B8005AD0002303A910460393FFF79BFE18B112
:10E9C800062004B0BDE8F081039B9C4201D80133C6
:10E9D800F6D1284600F064F9002847D1264B1A786A
:10E9E800424503D01A79424542D10120AA68BA4269
:10E9F80040D103EB8002EB6A92F801802979CDE9D6
:10EA080000430439927828683B4689B2FFF790FEA4
:10EA18000028D6D195F820300194002B4FF001033F
:10EA2800009314BF4246082295F82810686A3B46AE
:10EA3800FFF70BFE0028C4D1013E032EC1D8DFE842
:10EA480006F002070B0F0D4B1B681C611C62B8E730
:10EA58000A4B1B685C61F9E7084B1B689C61F5E78A
:10EA6800064B1B68DC61ACE70920AAE70F20A8E782
:10EA78000B20A6E70220A4E7A408002038240020E1
:10EA88001FB50B294FF00003CDE90033CDE9023360
:10EA98000A4607D00C2914D00A2910D00A2005B03C
:10EAA8005DF804FB012802D120238DF800300021F5
:10EAB800684602F022F8002818BF0E20EFE730233E
:10EAC800F3E70B21F4E7000038B5054602F010F82B
:10EAD800044610B10E24204638BD002DFBD1094B49
:10EAE8001B680B219878FFF7CBFF0028F2D10C2187
:10EAF800FFF7C6FF0028EDD10A21FFF7C1FF002864
:10EB0800E9D0E7E7382400202DE9F04380468FB0AC
:10EB18000C461746002A6BD0002969D000252946E3
:10EB28001D2206A8059504F0A7FE8DF81350344D54
:10EB38002B680DF114099E88CDF804900DF113038C
:10EB480002933B7900933B6832462146404601F0E8
:10EB5800F0FF00284ED138683A79494602F05EF94C
:10EB6800384600F04FF8002846D13C7AFA79BB794C
:10EB7800240444EA02241C432B689A6894423DD931
:10EB88009C609DF813000B21FFF77AFF034658BBE2
:10EB98000C21FFF775FF034630BB0A21FFF770FF12
:10EBA800034608BB7B7ABA7AFF7A3F0447EA022712
:10EBB8001F433A46334621460920FFF723FD034603
:10EBC80090B933463A4621460820FFF71BFD034615
:10EBD80050B92A689DF8131091700021D1604FF048
:10EBE800FF31C2E90411916118460FB0BDE8F08306
:10EBF8000923F9E70E23F7E70F23F5E70323F3E7E4
:10EC08003824002010B50446002845D001680029A2
:10EC180042D011F8013B43710322063002F0FEF89E
:10EC28002046032250F8091B043102F0F7F8216846
:10EC3800CB79E3600A7A43EA0223E3604A7A43EA3B
:10EC48000243E3608A7A43EA0263E360CB7A23747F
:10EC58000B7B63742379212B1AD110220D3104F117
:10EC6800120002F0DBF81D222168501C8B5C6362E5
:10EC7800085C43EA0023901C6362085C033243EAA1
:10EC8800004363628A5C43EA02636362002010BD4A
:10EC9800112B03DC0D22E7E70220F8E70120F6E755
:10ECA80010B50446002854D00168002951D00B78CB
:10ECB80043714B7883608A7843EA02238360CA7879
:10ECC80043EA024383600A7943EA026383604B792B
:10ECD80003738B79C381CA7943EA0223027BC38118
:10ECE80002F00F020831103002F098F8237B00225E
:10ECF80003F00F0384F8202084F82820227903F1F8
:10ED08000800111A04290DDD21680933043AD21AC2
:10ED1800085C84F82000D2B2606A84F8282019447C
:10ED280002F07CF8237922681A44002012F8043C87
:10ED3800E36212F8031C43EA0123E36212F8021C9F
:10ED480043EA0143E36212F8012C43EA0263E362F7
:10ED580010BD0220FCE710B5044660B3036853B346
:10ED68000279162A29D942791A700146082251F8DF
:10ED7800060B013002F05CF82146082251F80E0B10
:10ED8800093002F055F82368E28A5A74E38A226847
:10ED98001B0A93742368A269DA74A36922681B0AA0
:10EDA80013752368628B5A752368E27E9A75172358
:10EDB8002371002010BD0120FCE70220FAE738B5D6
:10EDC8000446002863D00168002960D0037B90F8CE
:10EDD800282003F00F03002A57D108332079043282
:10EDE8001344984255D363790B702368A2685A700C
:10EDF800A36822681B0A937023686289DA70236803
:10EE0800E27A1A712368227B5A712368E2899A711F
:10EE1800E38922681B0A2146D371227B51F8100B23
:10EE280002F00F02083001F0F9FF237B94F8282044
:10EE380003F00F0303F108052AB1226894F82010A3
:10EE4800515503F10905206894F82820616A28447F
:10EE580001F0E4FF94F828302268E16A2B44D15489
:10EE68005A1CE16A206892B2090A81549A1C2168E6
:10EE7800E08D92B28854DA1C216894F82F0092B27F
:10EE8800043388542371002038BD0933A6E70120D4
:10EE9800FAE70220F8E70000024B1A8810431880AE
:10EEA800704700BF3C24002008B5074B1B883BB1C6
:10EEB800FEF7CAF9002814BF6FF00200002008BD51
:10EEC8006FF00100FBE700BF3C24002010B5034BA6
:10EED80000241C80FEF7AEF9204610BD3C2400201B
:10EEE800B0FA80F04009704782B018B9084602B0FD
:10EEF80000F0CAB8002002B0704710B9084600F008
:10EF080077B9704710B9084600F08EB970470346C4
:10EF1800084611460BB900F0E5B90020704710B952
:10EF2800084600F06DBD704710B9084600F006BAF3
:10EF38000020704710B40446084611461A46019B43
:10EF480014B910BC00F014BA10BC70470346084648
:10EF580011460BB900F03EBA0020704710B40446C1
:10EF6800084611461A4614B910BC00F0ABBA002086
:10EF780010BC704730B40546084611461A46DDE90C
:10EF880002341DB9029430BC00F02ABB002030BC0A
:10EF9800704710B9084600F0DBBB0020704710B975
:10EFA800084600F06BBD0020704710B9084600F015
:10EFB800EABB0020704710B9084600F0E7BB002004
:10EFC80070470346084611460BB900F001BC002003
:10EFD800704710B40446084611461A46019B14B9F6
:10EFE80010BC00F0F7BB092010BC704710B40446F1
:10EFF800084611461A4614B910BC00F061BDC8B2E3
:10F0080010BC70470048704701000102064B10B55C
:10F018001B6A0446984730B10448054B204498427F
:10F028008CBF0020012010BDCC43010840C220C97C
:10F0380080B92A00F0B5114B85B00C4610491F560F
:10F04800054601F04BF80F4BE4B25E6A072D4FF00E
:10F058000103CDE9024301460AD105220023CDE987
:10F0680000234FF47A727A431846B04705B0F0BDD2
:10F0780008220020CDE900203A46F5E7B03D010816
:10F08800903D0108CC4301081FB500230093037885
:10F09800013B372B21D8DFE803F01C242020201E59
:10F0A800202020204143454E2055585B5E61642056
:10F0B8006C1E6E73787A20207D81262020202020E7
:10F0C800202020202020202083858A2020838A2039
:10F0D8008C90C3780BB102230093009805B05DF8BB
:10F0E80004FB8378F6E743788DF8043005238DF820
:10F0F80005308378003B18BF01235B008DF806308C
:10F1080010238DF80730304B1B6801A803F558729F
:10F11800CDE9022300F0C2FF0090DEE74023DBE7E1
:10F128002023D9E7827890F9013012B9274AD35CB5
:10F13800D2E7274AFBE7827890F90130002AF8D114
:10F14800244AF4E740F6B833C6E74FF47A73C3E7C6
:10F158004FF4FA63C0E741F28833BDE741F27073B8
:10F16800BAE71D484FF47A7101F03CFE00F5FA60E9
:10F17800D2E71A4BB0E7144B1B6803F55873ABE79B
:10F18800114B1B6803F55B73A6E71023A4E70E4B2E
:10F198001B68A1E74FF0834300939EE7104BFBE702
:10F1A800104B99E740F21113ADF8003095E70323AF
:10F1B80092E790F901300C4AB9E70C4990F901003F
:10F1C80000F08CFFA8E700BF44240020853D01081B
:10F1D800753D01087D3D010818FCFFFF00EA063770
:10F1E8009A99094040F70937B03D0108903D010858
:10F1F80037B50B4B02781B680C2101FB02335B7A95
:10F2080003EB4304074B1D6803690093C368427806
:10F21800816805EBC40000F0DDFC03B030BD00BF21
:10F22800442400204024002070B586B0027B64236B
:10F23800ADF80030012A4FF00003CDE90133CDE9E4
:10F2480003338DF802308DF8143030D0022A39D0CB
:10F258005ABB03684BB343683BB31F4D80682B60B0
:10F268001E4B18226946186001F0D8FD1C4B2C680B
:10F2780093E807000C3384E8070093E8070004F1DB
:10F288000C06032386E80700A4F86C33012204F572
:10F298005B7104F5587000F08EFC2B684FF6B07265
:10F2A800A3F878230522C3F87C2306B070BD0A4969
:10F2B80008684360036100F55B7100F5587000F061
:10F2C8007AFCF2E7044B1B68B3F86023B3F86C13BD
:10F2D8000A43A3F86023E8E74424002040240020E0
:10F2E800683A010808B503460A2924D8DFE801F07E
:10F2F80006232323230B161B23212100BDE80840E6
:10F308000068FFF783BE90F900009978052271B96B
:10F3180000F011FC003818BF012008BD052293F940
:10F3280000000021F4E790F900005978EEE7022187
:10F33800EEE70722F3E70020EFE7000008B50279BF
:10F348001AB1012A0BD0002008BD084B01681B68C0
:10F35800012203F5587000F02EFC0120F4E7034B5E
:10F3680001681B6803F55B70F5E700BF44240020C3
:10F37800F7B50528144D1C46A8BF052058700E4641
:10F388002946174600F0AAFE94F90130A070072B11
:10F3980013D1322000F0A2FD0C4BDB6D05469847D7
:10F3A80004F10C0208340346019200943A463146AF
:10F3B800284600F098FD03B0F0BD054A55F8231023
:10F3C800D05C00F083FDE7E7903D0108CC430108DD
:10F3D800B03D01082DE9F04F344F90F901607B688A
:10F3E800D0F804908BB00446884698470546002814
:10F3F80059D1E37C73B92E4A2378126803EB43038F
:10F40800990002EB8303D3F80490B9F1000F01D1FE
:10F4180052F80190274B484613F906B0FB68984705
:10F42800A37C2289D7F818A00993072E28D1002396
:10F438000121CDE90223204A0693CDE90431CDE923
:10F4480007330521CDE900214FF47A7202FB0BF254
:10F458004CF250311846D047637C13B3174B995D73
:10F468007B6D0D31C9B228469847E07C3246494643
:10F4780000F046FE88F8006001200BB0BDE8F08F70
:10F48800002101250823CDE90013CDE90715CDE9B1
:10F498000511CDE903110292A1782B465A46284658
:10F4A800D9E7074BDBE70020E7E700BFCC430108BB
:10F4B80044240020B03D0108854501007D3D010838
:10F4C800853D01082DE9F04F8DB090F90130DFF846
:10F4D800FCA0DFF8FC90CDE90A123E4A12F903B00D
:10F4E8000278DAF800300C2505FB02333A4A5B7AD9
:10F4F800126803EB430302EBC303044693F90210BB
:10F5080090F9020000F0E5FD3449064694F901003F
:10F5180000F0E4FDA26861688046304600F00BFD0B
:10F528002178DAF80020D9F80C306943074650589A
:10F538009847D9F81C309C4694F901300025072BD0
:10F548004FF47A63CDE90753CDE905552DD1012351
:10F55800CDE903530523CDE901534FF47A7303FB37
:10F568000BF300933946434646F2A81228466746ED
:10F57800B8472378DAF800200C214B4394F901109E
:10F58800D05800F0DFFDA18994F90100FFF752FD82
:10F598000B9B217B1860D9F85430284698470A9B62
:10F5A80001201E700DB0BDE8F08F01200823CDE9C1
:10F5B8000350CDE901032A46CDF800B0654643461D
:10F5C8003946A84701200546D3E700BF4424002058
:10F5D800CC430108B03D010840240020903D0108BB
:10F5E8002DE9F04F8FB0002405468A46914698468B
:10F5F8000494ADF81440ADF8024007264FF0010B13
:10F608002B7AA34206D9686804A9204400F0F6FBC7
:10F6180000285ED102238DF8083002A86B7A8DF895
:10F628000A30FFF731FDAB7A8DF81D309DF81130A7
:10F638008DF81E309DF812308DF81F309DF810306F
:10F648008DF82030EB7A8DF821302B7B8DF8223025
:10F658006B7B8DF8233010238DF81C608DF82430D7
:10F668003A4E8DF82C000DF102030A9305238DF80C
:10F678002D3033680C930723ADF834302B6806938C
:10F688000DF1120204AB0DF1110106A800F0D0FB38
:10F69800072805460BD130680C22002100F5587068
:10F6A80001F0D0FB3368BDF80220A3F860239DF871
:10F6B80011308AF800309DF8123089F800309DF832
:10F6C800103088F80030189B28461C700FB0BDE831
:10F6D800F08F9DF81330BDF81470ADF80270204417
:10F6E800C4B2F3B917B3194A0020116807260246B5
:10F6F8004FF00C0C062B1BD10CFB00FE51F80EE052
:10F70800BEF1000F04D00BFA00F23A4397B201227F
:10F7180001301028EED1002A3FF472AFADF8027024
:10F728006EE75A1E042A01D9062BDCD0062667E7A5
:10F7380047FA00FE1EF0010FEAD00CFB00FE51F85C
:10F748000EE0BEF1000F08BF0626E1E744240020C2
:10F7580038B505464068FFF759FC0522841D00218D
:10F7680095F90000E4B200F0E6F908B904F0FD04E8
:10F7780095F901000722002100F0DDF908B904F02D
:10F78800FB04204638BD00207047000010B5037800
:10F798000F2B044618D84068FFF738FC22780B492D
:10F7A80002EB42020968831C01EB820051F8222017
:10F7B800DBB21AB903F0FD0358B210BD032B06BF24
:10F7C800626842600223F7E70020F6E7442400203D
:10F7D800022070472DE9F04FDFF838810446D8F849
:10F7E800000099B08946174600211E4601220323CE
:10F7F80000F55870CDE90611CDE908118DF81410FF
:10F808008DF81510ADF8163000F0B7F938B9D8F8FA
:10F818000020B2F8603343F00303A2F86033D8F84D
:10F828000020637A8DF8283002F55871CDE90B1263
:10F83800394A94F9083012680D920DF116020F92A8
:10F848002268109262681192D4E90301A27A8DF8B5
:10F85800482001228DF8492013AA82E803001025C8
:10F86800227DE18A8DF8293018468DF85420ADF8AC
:10F878003850FFF7DFFB0AAB17930DF1150316900D
:10F8880000933146019705AB06AA10A800F0C2FB09
:10F89800064698BB9DF81410204F013901F0A2FAD2
:10F8A8001F4B1B690393C4B24FF00C0B04F16003A8
:10F8B8006B44D8F8000013F848AC9DF814300BFBE3
:10F8C8000AFC01343946B4FBF3F203FB1244D0F8C6
:10F8D8007C33B0F9782350F80C00DDF80CC0E4B2A2
:10F8E800E04728B189F800A0304619B0BDE8F08F8C
:10F8F800013D15F0FF05D9D10D26F5E70C2801BF0C
:10F90800D8F80020B2F8603343F00303A2F860335C
:10F91800EAE700BF4424002040240020400D0300F3
:10F92800CC430108F8B50679012E054648D90F2EB3
:10F9380048D80368187A40F303000522002140B232
:10F9480000F0F9F82B680446187A40F303100522F2
:10F95800002140B200F0EFF8B8B1B4FA84F46409B9
:10F9680029680B7A086843F3030243F303135BB275
:10F9780052B29A42C8BF0124FFF748FB80F0010346
:10F98800DBB224B10533D8B2F8BD0124E8E7DBB90E
:10F998000E4F29683B6806EB460003EB80000C22FB
:10F9A80001F03CFA3A680C2303FB062320465C72FC
:10F9B800B2F860130123B3400B43A2F86033E3E7C6
:10F9C8000620E1E70320DFE70420DDE744240020E8
:10F9D80010B4017801290ED9084B18680C234B4341
:10F9E800C4180022C250C4E9012200F5587010BCA6
:10F9F800102200F0A9B8002010BC70474424002051
:10FA08002DE9F04186B050238DF81430037A102B7D
:10FA1800074630D14368DD7B6DBB0224A8466426C7
:10FA2800062C14D87A68535D03932A44517843EA24
:10FA380001230393927843EA02437343CDE90338E1
:10FA480063B968468DF80040FFF7C2FF0DE0CDF8B6
:10FA58000C808DF81480CDF81080F2E703AB01A874
:10FA680001938DF80840FFF75DFF0134E4B2102CD4
:10FA780005F10305D4D106B0BDE8F0811FB50268D1
:10FA88000379116849B901A88DF80430FFF7A0FF80
:10FA980078B1032005B05DF804FB02A802928DF846
:10FAA8000C30FFF73FFF042805D0052805D00028B3
:10FAB800EFD00020EEE70220ECE70120EAE70000A3
:10FAC800C90020B9034B0B449856C0B27047024B8B
:10FAD800F9E700BF353D0108F53C0108F0B59A4249
:10FAE800069D03DB9DF914309A4220DD0020F0BD0D
:10FAF80003EB430331F814C005EB830300264CFAEB
:10FB080006F7FF0707D51F7A07F00F0E964502DCA8
:10FB1800B2EB171F0DDD0136102E03F10C03EED1E9
:10FB28000134E4B22301DBB29842E1D8DEE70024D5
:10FB3800F8E70120DBE7884204DB9042CCBF0020D5
:10FB4800012070470020704710B51409B4EB111F4D
:10FB580003464FEA11100ED391420CD202B201F0C3
:10FB68000F0133F81240012000FA01F124EA0101E3
:10FB780023F8121010BD0020FCE7F0B528B100EB07
:10FB8800410501270020914200D3F0BD002435F83B
:10FB980002CB234607FA04F636EA0C0608BF0133FF
:10FBA80004F1010408BFDBB2102CF3D11844013171
:10FBB800C0B2C9B2E7E710B500B149B910BD31F814
:10FBC800134020F813400133DCB2A242F7D8F5E71E
:10FBD8000023F9E782B030B504880493D2B9B3F5AD
:10FBE800616F15D349F6AF2542F21072AB4298BF48
:10FBF8004FF47A72944238BF14466143BDE83040EE
:10FC0800C3688B428CBF5B1A0023C36002B0704785
:10FC18006422EFE7012C38BF0124EEE72DE9F04F0D
:10FC28008FB01546199F03939DF8603007930C46D3
:10FC3800804603F0C7FB6A4A0590A7F5F633303BC8
:10FC4800B3FBF2F3534303F5F63B0493182313FB7A
:10FC580005430BF1300B069300254FF0FF3A069B46
:10FC68009C4207D1002D14BF50464FF0FF300FB013
:10FC7800BDE8F08FBDF96830ADF8243009991997BF
:10FC88003846089703F02EFB2688B8F1000F5FD19D
:10FC9800B7F5616F5AD349F6AF2242F21073974213
:10FCA80098BF4FF47A739E4238BF1E46642E59D1CE
:10FCB800DFF83091A060A1680CA803F035FB0D9B1C
:10FCC8000093DDE908120C9B0AA803F08CFA039A4A
:10FCD8000A9B0AB9079A2AB122694A4502D1424ABF
:10FCE80093420ED9414BC4F80C909F4209D9002386
:10FCF800ADF82C300B99CDF828B0584603F0F2FA3D
:10FD0800A060606808B9C4F80C90C4F81090B8F105
:10FD1800000F04D003F060FBE3680344E360D4E918
:10FD280003329342059B88BFE26063601B9BE168D6
:10FD38007343994204D20398E8B9B8F1000F1AD076
:10FD480001231D442375EDB2183488E76423AAE71C
:10FD5800039B0BB9234BE360012EDFF8889038BF73
:10FD68000126CEE7B6F57A7F0ABFDFF88490DFF880
:10FD78008490A0609FE700209342207506D85B1A04
:10FD88009A4505F1010528BF9A46EDB2B8F1000F72
:10FD9800DAD1642E184AADF82C801DD049F6B0236C
:10FDA800B6F57A7F18BF1346974281BF049A02F5C9
:10FDB800A83202F5C0729B180A931A9B00930AAEE8
:10FDC80096E80600199B304603F00DFA96E8030002
:10FDD80003F088FA8246B7E74FF46163E4E700BFAF
:10FDE8008051010040771B007F5101002FEC01007A
:10FDF80080A81201002E930230EC01000378032B37
:10FE080014D1437803F00F021B098A704B70837872
:10FE18008B80C27843EA02238B800379C3F30212F2
:10FE280003F00F03CA700B7005207047002070475D
:10FE38002DE9F3479A464379057990F90760914689
:10FE4800044690F906208846D3B190F90870002D31
:10FE580037D00F2A1BD194F909200F2E27D194F9F6
:10FE68000A00072D02D1002F08BF012788F80020BB
:10FE780089F8000028468AF8007002B0BDE8F087CB
:10FE880090F90B7090F9092090F90A60DFE7A369EF
:10FE9800019394F91530009394F914302169207B6B
:10FEA800FFF71CFE0028D8D105F0FD05D5E794F929
:10FEB8001D00B042D5DC94F91C30B34203DA05F0DA
:10FEC800FB053046D2E73046CBE70000024B03FA89
:10FED80000F0B0FBF1F0704740420F004FF4FA53C6
:10FEE800B3FBF0F0704730B54FF47A750C1F6A43D6
:10FEF80000FB042252001EBF00F1FF341219B2FBAE
:10FF0800F0F2914238BF1146039A116082004843CB
:10FF18001CBF013040084FF47A71121A01FB1323F9
:10FF2800002BCABF03F2E73393FBF1F1B3FBF1F106
:10FF3800049B196030BD38B5400014460D46F1F7F2
:10FF480065FD01462846F1F7AFFC2146F1F7ACFC08
:10FF5800F1F79EFB03F0DCFCF1F77AFC40B238BD08
:10FF68002DE9F74F019300239C469E46048A1E0103
:10FF7800F6B2B44246D906EB46054FEA4309AD004E
:10FF88000024476837F809702741FF0729D5876893
:10FF980007EB050A7F5927B3077837B9476927B1AF
:10FFA80037F809702741FF071BD59AF8087090F9B0
:10FFB80001B047F303084FFA88F8D84511DC47F336
:10FFC80003177FB25F450CDB9AF8097007EB470807
:10FFD800C76807EBC8073F7D5FB90CF1010C5FFAF2
:10FFE8008CFC0134102C05F10C05CAD10133DBB2AD
:08FFF800BCE70EF1010706EB66
:020000040801F1
:10000000040801F80E805FFA87FEEEE7019B82F894
:1000100000E083F800C003B0BDE8F08F2DE9FF4792
:1000200004464068DDE90C671D468A46914603F0A8
:10003000D7F923681B1A3B604FF000080123337087
:1000400085F80080636813B12368834224D8D4F80C
:100050001CC0CAF80080A3699CF800E00393D4E9AF
:10006000030101AB83E80300237D0093DCF80C104F
:10007000237A627A7046FFF7D5FD334638602A4608
:10008000E0694946FFF770FF2B782BB1C7F8008075
:10009000002004B0BDE8F0873378002B0CBF0C20A3
:1000A0000B20F6E737B590F9002090F90250954201
:1000B00004460FD0013A52B295420BD0A368019387
:1000C00094F9013000936168E0782B46FFF70AFD50
:1000D0000028EFD0104603B030BD8842B8BF0846B4
:1000E0007047000051F82000054B984205D0054BA1
:1000F000C31A58425841400070470120704700BF62
:1001000090D0030020A1070005281FB50ED80C4B86
:1001100053F820300093CDE901120A4B012200214F
:10012000022002F06BFE05B05DF804FBCDE9001281
:10013000054B01220021022002F060FEF3E700BF20
:10014000243E0108B83D0108D73D010807B5054B1D
:10015000CDE9000101220021022002F04FFE03B090
:100160005DF804FBF33D010810B5102204460021A0
:10017000F13000F06BFE0021C4F814112046F0228B
:10018000BDE8104000F062BE02460846102100F0B3
:10019000A5B92DE9F0430446D0F8140185B00E4608
:1001A000154604F2011988B3C0F11008904547467E
:1001B00028BF1746BAB2484400F034FED4F81431D0
:1001C0003B440F2BC4F814312DD9A8452BD204F190
:1001D000F00304F5807113F8012F187C8B4282EA3A
:1001E00000021A70F7D104F1F10810224146684666
:1001F00000F018FE22466946684600F0F1F9102228
:100200006946404600F00EFE3E44ED1B04F5807842
:1002100004F1F107102D09D8AAB23146484600F082
:1002200001FEC4F8145105B0BDE8F08304F1F003F9
:10023000711E13F8012F11F8010F434582EA0002E5
:100240001A70F6D110223946684600F0EBFD2246BE
:100250006946684600F0C4F910226946384600F045
:10026000E1FD1036103DD5E7F0B589B00C461022FF
:1002700000210546684600F0E9FD224669466846C9
:1002800000F0AEF99DF90030002B6A464FF00001F6
:1002900043DA137812F8010F01315B0043EAD013FF
:1002A0000F2902F8013CF4D19DF80F305B0083F078
:1002B0008703D4F81401DBB210288DF80F303BD13E
:1002C00004F58073694604F5887013F8016F11F81E
:1002D000012B984282EA06021A70F6D104F1F0036B
:1002E00004F5807113F8012F187C8B4282EA00021A
:1002F0001A70F7D110220DEB020004F1F10100F0A9
:1003000091FD2246294604A800F06AF91022002136
:10031000684600F09BFD09B0F0BD137812F8010F9C
:1003200001315B0043EAD0130F2902F8013CF4D1FC
:100330009DF80F305B00BCE79DF90030002B6A464A
:100340004FF0000137DA137812F8016F01315B00CA
:1003500043EAD6130F2902F8013CF4D19DF80F307F
:100360005B0083F08703471CDBB28DF80F30102F42
:1003700004EB0003C0F10F064FF0800288BF002697
:1003800000F5817083F801210021324620443E446B
:1003900003F076FAC4F8146104F58073694604F535
:1003A000887013F8016F11F8012B984282EA060257
:1003B0001A70F6D192E7137812F8016F01315B00E1
:1003C00043EAD6130F2902F8013CF4D19DF80F300F
:1003D0005B00C8E70A780378534003704A78437893
:1003E000534043708A78837853408370CA78C378C7
:1003F0005340C3700A790379534003714A794379B2
:10040000534043718A79837953408371CA79C379A0
:100410005340C3710A7A037A534003724A7A437A8B
:10042000534043728A7A837A53408372CA7AC37A7A
:100430005340C3720A7B037B534003734A7B437B65
:10044000534043738A7B837B53408373CA7BC37B54
:100450005340C373704710B50B7814786340037032
:1004600054784B786340437094788B786340837002
:10047000D478CB786340C37014790B7963400371EF
:1004800054794B796340437194798B7963408371DC
:10049000D479CB796340C371147A0B7A63400372C9
:1004A000547A4B7A634043728B7A947A63408372B6
:1004B000D47ACB7A6340C372147B0B7B63400373A3
:1004C000547B4B7B63404373947B8B7B6340837390
:1004D000CB7BD27B5340C37310BD0000A1F110034E
:1004E000DBB2102B2DE9F047044604D83A4820FA35
:1004F00003F3DB0705D4002382F8F030FF20BDE8CA
:10050000F087561E254615F8013B06F8013F631B90
:100510000B4413F0FF00F6D101F11C039B005FFABE
:1005200083FCC3F30313013BDFF8B09082F8F03093
:10053000884653184FF0010EB8FBF1FA01FB1A8AF6
:100540001AF0FF0A13F8047C13F8036C13F8025C2A
:1005500013F8014C30D119F806A019F8056019F804
:10056000045019F807404FEADE1707EB47078EEAF9
:100570000A0A07EBC7074FEA4E0EFFB25FFA8EFE7C
:1005800087EA0E0E574692F800A087EA0A071F7006
:1005900057787E405E70967875409D70D57808F1EA
:1005A00004085FFA88F86C40C445DC7002F104026C
:1005B00003F10403C0D8A2E71829E4D9BAF1100F57
:1005C000E1D1DFF818A01AF807701AF806601AF8D7
:1005D00005501AF80440D6E7010101003C4001082B
:1005E0002DE9F04FA3B092F8F0301D911B920193CA
:1005F000002B00F0538101461EA8FFF72CFF1B9B28
:10060000A74CA84DA84E10330293002303939DF8E6
:100610007C0004909DF886000590205C06909DF873
:100620007B000790205C089004989DF881C0205CB6
:10063000099014F80C000A909DF880000B909DF82A
:1006400085009DF878809DF87DE09DF882A09DF85A
:1006500087900C909DF87A00029B1C9314F80A2056
:1006600014F8093014F8081014F80E700D90205C7E
:100670000E909DF87F000F90205C10900B98205CEE
:1006800011900C98205C12909DF8840013909DF8B6
:10069000790014909DF87E001590205C16909DF8CE
:1006A00083001790205C18901398205C1990149880
:1006B000205C1A900398013003900298DDF804B092
:1006C000103002909DF80C00834536D88DF87810D4
:1006D0008DF87A2009990E9A8DF87C108DF8822079
:1006E0001199069A8DF880108DF87E201999169A26
:1006F0008DF884108DF886200A99189A8DF87D104F
:100700008DF887201299109A8DF87B301B9B8DF8FD
:1007100081108DF883201A99089A1D988DF88510FC
:100720008DF87F201EA903EB0B128DF87970FFF76F
:1007300092FE002023B0BDE8F08F15F808B082EAE1
:1007400003008BEA000016F80EB080EA0B008DF86B
:10075000780015F80E004B40434016F80A0043405D
:100760008DF8793081EA070315F80A10594016F818
:100770000930594016F808308DF87A107A40534005
:1007800015F8092053408DF87B30089A069B53409A
:10079000049AAA5C534016F80C2053408DF87C3024
:1007A000DDE908325A4015F80C305340059AB25C26
:1007B00053408DF87D30DDE909325A40059BEB5CF2
:1007C0005340079AB25C53408DF87E30069B0A9ADC
:1007D0005340049AB25C5A40079BEB5C5A408DF838
:1007E0007F200E9B109A53400B9AAA5C53400C9AA0
:1007F000B25C53408DF88030DDE910325A400C9BDA
:10080000EB5C53400D9AB25C53408DF88130DDE9CA
:1008100011325A400D9BEB5C53400F9AB25C53402F
:100820008DF88230129A0E9B53400B9AB25C5A405C
:100830000F9BEB5C1C995A408DF88320169B189AED
:100840005340139AAA5C5340149AB25C53408DF8FB
:100850008430DDE918325A40149BEB5C5340159A02
:10086000B25C53408DF88530DDE919325A40159B52
:10087000EB5C5340179AB25C53408DF886301A9A5D
:10088000169B5340139AB25C5340179AAA5C1EA859
:1008900053408DF88730FFF79DFDB8E6FF2049E70C
:1008A0003C4001083C3F01083C3E010808B538B116
:1008B000044A05491060D82200F0B4FA002008BDAF
:1008C0000220FCE7482400206C4501080A4B1A6806
:1008D00070B5002302F1180503EB03142E5D864268
:1008E00004D1183422440A60002070BD01330B2B60
:1008F000F2D10320F9E700BF482400202DE9F041A0
:10090000CCB00646DDF8488117461C460D4631B38B
:10091000B8F1000F23D006A8FFF726FC204601A956
:10092000FFF7D4FF0446B0B9019906A80131FFF7DB
:100930002BFC26B11022314606A8FFF72AFC3A46C6
:10094000294606A8FFF725FC06A902A8FFF78CFC9C
:10095000029BC8F8003020464CB0BDE8F08102246C
:10096000F9E7000030B595B013A90446FFF7AEFFD4
:10097000002830D11B4B0C2101FB00F2D5189A5CEA
:10098000A2422AD1139B1A7C1092DA7B0F929A7B97
:100990000E925A7B0D921A7B0C92DA7A0B929A7A0B
:1009A0000A925A7A09921A7A0892DA7907929A790F
:1009B00006925A7905921A790492DA7803929A7813
:1009C00002925B7801930022AB6800931146064BBC
:1009D000022002F013FA15B030BD01300B28CBD144
:1009E000F9E700BFB44201083C41010810B40B2BE9
:1009F000019C03D8019410BCFFF780BF032010BCFA
:100A0000704730B50D4685B01446014668B103AA5B
:100A1000002000922A460390FFF770FF18B9039850
:100A2000001B18BF012005B030BD0220FBE72DE9F7
:100A3000F0430D46BFB014469946804620B31BB321
:100A400011F00F0122D1F02201A800F0FFF9204699
:100A50006946FFF73BFF044648B9009801AA1021F8
:100A60000130FFF73BFD2E46AF1BFFB21EB92046FB
:100A70003FB0BDE8F08301AA09EB070108EB0700CE
:100A8000FFF7AEFD103EEFE70224F0E70524EEE7A6
:100A9000F0B5184E3468024685B00846002304F1CC
:100AA000180103EB03154F5D97421ED10D2A05F186
:100AB000190513D10023CDE90033CDE902330C220F
:100AC00010216B46FFF7B3FF0446306810226946D9
:100AD000284400F0A7F9204605B0F0BD01461022D9
:100AE000601900F09FF90024F5E701330B2BD8D1F2
:100AF0000324F0E74824002009B1FFF7C9BF022012
:100B000070471FB51446A0B10C2A01D10B2912D190
:100B10000023CDE90033CDE902330A466B461021AC
:100B2000FFF785FF18B969462046FFF7B1FF04B00B
:100B300010BD0220FBE70320F9E7F8B51E46DDE90A
:100B400007479DF818505BB354B34FB3212D29D8F4
:100B500019462A46204600F065F90122631C691EE9
:100B6000B018FFF764FFF8B9E37ADB093B70EBB923
:100B70006319204613F8012C13F8021C120642EAEE
:100B8000014213F8041C0A4313F8031C012342EA30
:100B90000122291FFFF735FF003818BF0120F8BDDB
:100BA0000220FCE70520FAE70720F8E70420F6E733
:100BB00010B5044628B1044B5B69984720600020BB
:100BC00010BD0220FCE700BFCC43010808B5014678
:100BD00030B1044B0822186800F024F9002008BD49
:100BE0000220FCE74824002008B530B1044B08225D
:100BF000196800F017F9002008BD0220FCE700BFCB
:100C0000482400207FB5124E0023044602A8019319
:100C10000D46FFF7E9FF33685B6901936CB102AAE7
:100C2000082312F8011B41B9013B13F0FF03F8D16F
:100C300002A8A04702A8FFF7C9FF35B1019B23B95D
:100C400001A8A8473368019A5A61002004B070BD1A
:100C50004824002008B5014638B1054B1868082221
:100C6000104400F0DFF8002008BD0220FCE700BFC0
:100C70004824002008B538B1044B196808221144F3
:100C800000F0D0F8002008BD0220FCE74824002036
:100C9000034B1B6802280CBF196159610020704783
:100CA0004824002049B1064B1B68D3E904230228DD
:100CB00008BF13460B60002070470220704700BF3A
:100CC0004824002030B58FB0002405460CA80994B4
:100CD000FFF78AFF9DF8373007939DF8363006936B
:100CE0009DF8353005939DF8343004939DF83330EA
:100CF00003939DF8323002939DF8313001939DF8B3
:100D000030300093224621461E4B022002F076F836
:100D10000AA8FFF7AFFF9DF82F3007939DF82E30FC
:100D200006939DF82D3005939DF82C3004939DF883
:100D30002B3003939DF82A3002939DF829300193BC
:100D40009DF82830009322460F4B2146022002F0E6
:100D500055F809A92846FFF7A5FF9DF8243003930D
:100D60009DF8253002939DF8263001939DF8273099
:100D700000932246054B2146022002F03FF80FB0B7
:100D800030BD00BF98410108D64101081442010856
:100D900008B50020FFF7E6FD0120FFF7E3FD09207D
:100DA000FFF7E0FD0820FFF7DDFD0020FFF78AFFD9
:100DB000002008BD10B504460B20FFF7D3FD0C2022
:100DC000FFF7D0FD0920FFF7CDFD0820FFF7CAFD92
:100DD0000A20FFF7C7FD2046FFF774FF002010BD73
:100DE000014B1860704700BFAC0800200B4A30B5BB
:100DF00014680B4D43F2390305FB04331360091AE1
:100E00006FF00042B3FBF2F2C2EBC27201319B1AE7
:100E100093FBF1F201FB1233184430BDAC08002003
:100E20006D4EC64101380A44914200D1704711F815
:100E3000013B00F8013FF7E710440A44914200D11A
:100E4000704711F8013B00F8013DF7E702F018BDCB
:100E500030B530B10A4D01444FF0FF33814201D12A
:100E6000D84330BD10F8012B5340082243F300044F
:100E7000013A2C4092B284EA5303002AF6D1EDE7FE
:100E80002083B8ED01207047054B4FF400529A6261
:100E9000044B1B6813B15B6803B11847704700BF70
:100EA00000040048D8240020054B4FF480529A6279
:100EB000044B1B6813B1DB6803B11847704700BFD0
:100EC00000040048D824002001207047012070470A
:100ED00001F03EB901F02CB910B501F00FFE0E2162
:100EE000044640F61F1001F023F92046012101F0CD
:100EF000EFFDBDE8104001F0CDBA000070B50C4E1A
:100F000001EB40030D46B3654FF6FF710023044625
:100F10001A46084601F054FB96F85600002101F0ED
:100F2000D7FD29462046BDE8704001F08BBA00BFCE
:100F30007C24002010B5044601F0A0FE01281CD13D
:100F400001F0A4FE34B11248214602F00BFB104818
:100F500002F0CEFA0F4C104B00214FF48052A165E5
:100F60009A6194F8560001F0B3FD63786BB16FF0AD
:100F70007F40BDE8104001F049BA002340F26221F1
:100F80001A46084601F01CFBDCE7A0688001F0E788
:100F90004C2400207C24002000040048002001F0A4
:100FA000B5B9000008B501F0BDF80438C0B2032897
:100FB00096BF024B0020185C08BD00BF9643010895
:100FC00008B501F0B0FD033008BD01F03FB901F0F4
:100FD000FFB808B501F0F6FC08BD000038B50D46B5
:100FE000144601F053FB284601F088FD0E2105460A
:100FF00040F61F1001F09CF828460121074D01F032
:1010000067FD01F047FA4FF47A716143284602F018
:10101000A9FA2846BDE8384002F06ABA64240020E4
:1010200001F034BB08B5084B002193F8560001F0DD
:101030004FFD00234FF4C0711A46084601F0C0FA74
:10104000BDE8084001F01ABA7C24002010B504461F
:1010500001F014FE01281CD101F018FE34B1124831
:10106000214602F07FFA104802F042FA0F4C104B72
:1010700000214FF48052A1659A6194F8560001F066
:1010800027FD63786BB16FF07F40BDE8104001F041
:1010900073B9002340F262211A46084601F090FA23
:1010A000DCE7A0688001F0E74C2400207C240020CD
:1010B0000004004808B54FF0040001F00DF9BDE848
:1010C00008400220F1F70EBD08B500231A46194664
:1010D000184601F075FABDE8084001F063B9000058
:1010E0001D4B73B51D4D186000241D486C70C5E97B
:1010F0000144AC6501F08EFAAC8101F0F9F92146AA
:10110000204601F041FC21460422012001F0F2FAC0
:10111000144E154D4FF6FF7123462246084601F046
:101120004FFAFFF7C7FF2246104B00944FF0FF31F4
:10113000304602F031F90E4B009422464FF0FF3159
:10114000284602F029F9304602F084F9284602B018
:10115000BDE8704002F07EB9D82400207C24002035
:1011600015210108642400204C240020890E010868
:10117000A90E01080128084805D1084BC17719704C
:101180000E3001F09DBB437D012B03D1034B8175D4
:101190001970F5E7704700BF7C240020B0080020DC
:1011A0000D4B10B5044618735873012000F016F863
:1011B0005CB134214FF4E86000F0BAFF4421BDE88F
:1011C000104040F2417000F0B3BF14214FF4E860CA
:1011D00000F0AEFF2421F2E77C24002038B5114C4A
:1011E0000546207001F057FD052D04D8DFE805F015
:1011F000090B03171709032001F066FA0023637334
:1012000038BD0020F8E7012001F05EFA207B637B07
:101210008342F5D06073BDE83840FFF7C1BF0220BC
:10122000EAE700BF7C2400202DE9F0431E4687B08A
:1012300000230546CDE901330C46174601F01DFD9C
:10124000032D5BD8DFE815F07A00C1000C01040023
:10125000A27C082A69D8A16801A801F0D5FE2168FE
:10126000002962D042F210729142E37C874D50D83F
:101270000322AA7385F83820E96385F844304FF0DB
:1012800002086368A17DDB002B820423AB74A37C7E
:10129000DB00EB7402294FF000032B75637D02D055
:1012A000227D022A46D103F10F02D2B2012A01D9CE
:1012B000012B3AD1764B774A196803944FF0010914
:1012C00003A88DF8149001F0D5FC70BB287685F842
:1012D00017906875FFF762FE4046FFF77FFF6E4884
:1012E00001F082FA6D4801F0EBFA01A800F080FFEE
:1012F000208A00F051FFA08900F096FF384601F0E7
:10130000FDFB624C84F8560001F0BCFC66600020D6
:101310000DE04FF00008E963890885F80E8085F834
:10132000388085F844302964ABE74FF0FF3007B0D0
:10133000BDE8F083EB7529766A75CBE72368002B4F
:10134000F3D0A27C082AF0D8504DA16801A801F082
:101350005BFE002385F838302268EA63E27C85F87A
:101360004420A269AB732A646268D2002A820422F4
:10137000AA74A27C2B75D200EA74A27D022A02D044
:10138000237D022B1CD1627D02F10F03DBB2012B06
:1013900001D9012AC9D13E4B3E4A196803944FF046
:1013A000010803A88DF8148001F064FC0028BCD16A
:1013B000287685F817806875FFF7F0FD00208CE728
:1013C000617DE9752A766B75F6E7304D012185F868
:1013D0003810227885F85020637885F85130A3784A
:1013E00085F85230E3788B4202D0022B03D03BB910
:1013F00085F8533004E00B3A012A29D885F85310B8
:101400004FF0010885F80E80A388AB83A379AB77F2
:10141000E37985F82030237A85F82130FFF7BEFD87
:101420004046FFF7DBFE1C4801F0DEF91B4801F0E7
:1014300047FA95F85130062B40F689000AD100F0A2
:1014400087FE00F0FB0140F6890000F071FE55E7D1
:101450000023CDE700F07CFE40F00401C9B2F2E7C2
:101460002368013BB3F57A7FBFF45FAF0320FFF73A
:10147000B5FE0648022380F83830236883641623BB
:1014800080F84C30383001F0AFF937E77C24002089
:10149000D824002064240020B42400208A240020C2
:1014A000F0B51E4687B00023CDE901331446074648
:1014B0000D4601F0E2FB002C724C16BF0123002305
:1014C0000026637027B1012F7AD0002007B0F0BD4D
:1014D000AB68002B00F0D280EB68002B00F0CE80D0
:1014E000AA7F082A00F2CA80296901A801F08CFDB0
:1014F0002868003818BF012000F0D6FF84F8387043
:10150000AB68E36395F8203084F84430686801F0F4
:1015100057FBA77384F84500EB68DB002382EB7F61
:10152000A374AB7FDB00E37495F82130237595F845
:101530002230002B3ED12A7D95F82410A275022975
:1015400095F8232001D0022B36D102F10F03DBB234
:10155000012B02D9012A40F0918000238DF814302C
:10156000494B4A4A1968049503A801F083FB0028F7
:1015700040F0848001232076E3756075FFF70EFD4F
:101580000020FFF72BFE424801F02EF9414801F000
:1015900097F901A800F02CFEA88B00F0FDFD288B28
:1015A00000F042FE4FF4FA53AA687343B3FBF2F320
:1015B000A3608AE7FF22BFE7E27521766375DDE766
:1015C0002B8E002B5AD095F83230A86A012B0CBF15
:1015D0002F7DFF27003818BF012000F065FFF0B213
:1015E00000F06EFF012184F8381095F82C2084F863
:1015F000502095F82D3084F8513095F82E3084F82D
:10160000523095F82F308B4202D0022B03D03BB9D9
:1016100084F8533004E00B3A012A27D884F8531099
:101620002B8EA38395F83230A3770126AB8E2384CB
:10163000A673E777FFF7B2FC3046FFF7CFFD1448FB
:1016400001F0D2F8134801F03BF994F82130B3428D
:1016500040F236700CD100F07BFD00F0FB0140F24F
:10166000367000F065FD4FF6FF73A1E70023CFE76A
:1016700000F06EFD40F00401C9B2F0E74FF0FF301A
:1016800024E700BF7C240020D82400204C24002024
:10169000B42400208A2400202DE9F04F85B0824632
:1016A0000E9DBDF840809DF844709DF848900191D2
:1016B00093461E4601F0E1FABAF1010F524C54D0A4
:1016C000BAF1040F00F09180BAF1000F3AD10B2269
:1016D000304684F8442084F838A0E56301F070FABD
:1016E0004FEAC803B9F1000F238241F60403638275
:1016F0000CBF0123F223E37587F001070123237652
:1017000084F84500C4F840B084F80EA084F814A012
:101710006775FFF743FC5046FFF760FD04F13800A2
:1017200001F062F804F10E0001F0CAF8374A1068BF
:10173000516802AB03C302A800F05AFD40F2FF104B
:1017400000F02AFD019801F0D9F90E2184F8560025
:1017500040F61F1000F0ECFC94F8560001F092FAED
:10176000169B636005B0BDE8F08F294984F838A066
:10177000EAB2895D84F8502076BB0B3D012D8CBF09
:1017800000250125053A012A04D8B8F10C0F38BF0D
:101790004FF00C081F4B9DF83C201B7884F85350E9
:1017A000E37701259DF8543084F8511084F85220D5
:1017B00084F82130A573A4F81C80A77784F82090C2
:1017C000FFF7ECFB2846FFF709FD134801F00CF882
:1017D000124801F075F8B5E7012E04D1A5F10C030C
:1017E0005D425D41CEE70025CCE75046FFF7F6FCB1
:1017F000022384F8383004F138001623A56484F8F5
:101800004C3000F0F1FF9DE77C240020803A010875
:10181000C8430108B0080020B42400208A24002016
:101820002DE9F04F87B0DFF8B4B29DF864A09DF8C1
:101830004C90029314469DF854309DF85020BDF80A
:101840004880039205468BF801A0BDF844600193DF
:101850000F4601F012FABAF1000F18BF4FF000085E
:10186000DFF87CA2039AB9F1000F08BFFF22012D17
:101870008AF8002000F0C880052D48D0002D40F0E7
:10188000C080284600F010FE0B2238468BF844201A
:101890008BF83850CBF83C4001F092F9019B8BF863
:1018A000450041F60402002BABF812209AF8002004
:1018B0008BF816200CBF0122F2228BF81720F600BD
:1018C000012289F001098BF818208BF80E50ABF833
:1018D00010608BF814508BF81590FFF75FFB2846CB
:1018E000FFF77CFC0BF1380000F07EFF0BF10E00DF
:1018F00000F0E6FF7B490868496804AA03C204A80F
:1019000000F076FC40F2FF1000F046FC71E0012090
:1019100000F0CAFD09224FF000098BF84420384638
:101920004FF44872CBF840208BF83890CBF83C400D
:1019300001F046F94FF48052ABF812209AF80020DB
:101940008BF845008BF8162028460122F6008BF80C
:1019500017208BF80E90ABF81060ABF814908BF852
:101960001890FFF73BFC0BF1380000F03DFF0BF146
:101970000E0000F0A5FF5B498868C96804AA03C28D
:1019800004A800F035FC40F2FF1000F005FC40F622
:10199000B80000F0DDFB00F0EF0140F6B80000F009
:1019A000C7FB042140F6B90000F0C2FB40F69B00E3
:1019B00000F0CEFB00F0E30141F0080140F69B008F
:1019C00000F0B6FB40F2D16000F0C2FB40F018011D
:1019D000C9B240F2D16000F0ABFB40F2AC6000F065
:1019E000B7FB00F08F0141F0500140F2AC6000F015
:1019F0009FFB4FF4FA5202FB08F2B2FBF4F2CBF871
:101A0000082007B0BDE8F08F002000F04DFD3649FA
:101A10008BF83850E2B2C95D8BF85020002F4DD1C1
:101A20000B3C012C8CBF00240124053A012A02D86A
:101A30000C2E38BF0C26029B9AF800208BF85230EF
:101A40008BF85340019B8BF81F2001249DF86020E8
:101A50008BF821208BF851108BF820308BF80E403A
:101A6000ABF81C608BF81E90FFF798FA2046FFF742
:101A7000B5FB1E4800F0B8FE1D4800F021FF5FFADC
:101A800088F000F01DFD40F6A30000F061FB00EAC5
:101A9000040140F6A30000F04BFB9BF82120A2427A
:101AA00040F2367013D100F053FB00F0FB0140F21E
:101AB000367000F03DFB4FF6FF72A0E7012F04D116
:101AC000A4F10C035C425C41AFE70024ADE700F0F9
:101AD0003FFB40F00401C9B2E9E700BF7C240020CD
:101AE000B0080020803A0108C8430108B42400204F
:101AF0008A240020F0B58BB00D46044617461E46DA
:101B0000FFF74CFA0020FFF769FB204600F0BEFD0E
:101B100000240123CDE9084303234FF4167229461C
:101B20002046CDE90644CDE90444CDE90244CDE99F
:101B300000532346FFF774FE2046FFF787FAFFF7AE
:101B40003FFAF0F7CFFF01F041FC0446204601F0D8
:101B500047FCB04205D30124FFF720FA20460BB022
:101B6000F0BD00F02FFF8742F0DA0024F4E7000018
:101B7000F7B500230C4640F201211A4606460846F6
:101B800000F01EFD644B654D4FF400529A6195F8CC
:101B90005600012100F09CFF2B78012B40F68900B4
:101BA00013D195F85130062B0FD100F0D1FA00F087
:101BB000FB0140F6890000F0BBFA2B78042B6CD8AF
:101BC000DFE803F0524B527F090000F0C1FA40F009
:101BD0000401C9B2EDE7524A731E1046C6F101076F
:101BE0004FF0000CF9188C426FDC0022E70013461E
:101BF000BA4271D19A0142EAC3125B0183F0200319
